 Rally

 Timestamp is 32869e46 (Mon Nov 11 12:32:22 1996)

 Preferred load address is 00400000

 Start         Length     Name                   Class
 0001:00000000 001057dcH .text                   CODE
 0002:00000000 00000790H .rdata                  DATA
 0002:00000790 00000028H .xdata$x                DATA
 0002:000007b8 00000000H .edata                  DATA
 0003:00000000 00000004H .CRT$XCA                DATA
 0003:00000004 00000004H .CRT$XCC                DATA
 0003:00000008 00000004H .CRT$XCZ                DATA
 0003:0000000c 00000004H .CRT$XIA                DATA
 0003:00000010 00000008H .CRT$XIC                DATA
 0003:00000018 00000004H .CRT$XIZ                DATA
 0003:0000001c 00000004H .CRT$XPA                DATA
 0003:00000020 00000004H .CRT$XPX                DATA
 0003:00000024 00000004H .CRT$XPZ                DATA
 0003:00000028 00000004H .CRT$XTA                DATA
 0003:0000002c 00000004H .CRT$XTZ                DATA
 0003:00000030 001339dcH .data                   DATA
 0003:00133a10 00d4f31cH .bss                    DATA
 0004:00000000 000000c8H .idata$2                DATA
 0004:000000c8 00000014H .idata$3                DATA
 0004:000000dc 000002d8H .idata$4                DATA
 0004:000003b4 000002d8H .idata$5                DATA
 0004:0000068c 00000af2H .idata$6                DATA
 0005:00000000 00000328H .rsrc$01                DATA
 0005:00000330 000024d0H .rsrc$02                DATA

  Address         Publics by Value              Rva+Base   Lib:Object

 0001:00000000       normal_ctrl_plset          00401000   PLCTRL.obj
 0001:00000074       myline_ctrl_plset          00401074   PLCTRL.obj
 0001:00000098       vs_ctrl_plset              00401098   PLCTRL.obj
 0001:0000010c       net_ctrl_plset             0040110c   PLCTRL.obj
 0001:00000180       other_set_mors             00401180   PLCTRL.obj
 0001:00000184       normal_plinit              00401184   PLCTRL.obj
 0001:000002f0       myline_plinit              004012f0   PLCTRL.obj
 0001:000003b4       mycar_init                 004013b4   PLCTRL.obj
 0001:00000644       vs_plinit1p                00401644   PLCTRL.obj
 0001:00000788       vs_plinit2p                00401788   PLCTRL.obj
 0001:000008a4       net_plinit1p               004018a4   PLCTRL.obj
 0001:000009e8       net_plinit2p               004019e8   PLCTRL.obj
 0001:00000b04       normal_otinit              00401b04   PLCTRL.obj
 0001:00000b6c       normal_plstart_wait        00401b6c   PLCTRL.obj
 0001:00000c38       myline_plstart_wait        00401c38   PLCTRL.obj
 0001:00000ccc       vs_plstart_wait1p          00401ccc   PLCTRL.obj
 0001:00000df8       vs_plstart_wait2p          00401df8   PLCTRL.obj
 0001:00000f24       net_plstart_wait1p         00401f24   PLCTRL.obj
 0001:0000111c       net_plstart_wait2p         0040211c   PLCTRL.obj
 0001:0000126c       normal_plmove              0040226c   PLCTRL.obj
 0001:000013c8       myline_plmove              004023c8   PLCTRL.obj
 0001:0000145c       vs_plmove1p                0040245c   PLCTRL.obj
 0001:000015a8       vs_plmove2p                004025a8   PLCTRL.obj
 0001:000016f4       net_plmove1p               004026f4   PLCTRL.obj
 0001:000018c8       net_plmove2p               004028c8   PLCTRL.obj
 0001:00001a9c       gover_plmove               00402a9c   PLCTRL.obj
 0001:00001b44       goali_plmove               00402b44   PLCTRL.obj
 0001:00001dc6       goal_plmove                00402dc6   PLCTRL.obj
 0001:00001e60       goali_plmove1p             00402e60   PLCTRL.obj
 0001:00001f75       goal_plmove1p              00402f75   PLCTRL.obj
 0001:00002018       goali_plmove2p             00403018   PLCTRL.obj
 0001:0000212d       goal_plmove2p              0040312d   PLCTRL.obj
 0001:000021d0       goal_plmove2p_sub          004031d0   PLCTRL.obj
 0001:00002298       normal_plmt_start          00403298   PLCTRL.obj
 0001:000023c0       calc_pmap_sub              004033c0   PLCTRL.obj
 0001:00002434       vs_plmt_start1p            00403434   PLCTRL.obj
 0001:00002590       vs_plmt_start2p            00403590   PLCTRL.obj
 0001:000026f4       net_plmt_start1p           004036f4   PLCTRL.obj
 0001:000028d8       net_plmt_start2p           004038d8   PLCTRL.obj
 0001:00002ac8       ending_plmt_start          00403ac8   PLCTRL.obj
 0001:00002b3c       replay_plmt_start          00403b3c   PLCTRL.obj
 0001:00002ce0       normal_plmt                00403ce0   PLCTRL.obj
 0001:000030c4       p2sync_ctrl                004040c4   PLCTRL.obj
 0001:000031bc       sync_ctrl                  004041bc   PLCTRL.obj
 0001:000032f0       replay_plmt                004042f0   PLCTRL.obj
 0001:00003470       ending_plmt                00404470   PLCTRL.obj
 0001:000034bc       vs1p_plmt                  004044bc   PLCTRL.obj
 0001:00003664       vs2p_plmt                  00404664   PLCTRL.obj
 0001:00003814       net1p_plmt                 00404814   PLCTRL.obj
 0001:000039bc       net2p_plmt                 004049bc   PLCTRL.obj
 0001:00003b6c       goal_plmt                  00404b6c   PLCTRL.obj
 0001:00003ca4       goal_plmt1p                00404ca4   PLCTRL.obj
 0001:00003d98       goal_plmt2p                00404d98   PLCTRL.obj
 0001:00004084       normal_otmt                00405084   PLCTRL.obj
 0001:000040ac       normal_otmtn               004050ac   PLCTRL.obj
 0001:000040b0       game_exit                  004050b0   PLCTRL.obj
 0001:00004988       set_gover                  00405988   PLCTRL.obj
 0001:000049e8       normal_rmove               004059e8   PLCTRL.obj
 0001:00004a10       replay_rmove               00405a10   PLCTRL.obj
 0001:00004a5c       normal_endmove             00405a5c   PLCTRL.obj
 0001:00004a84       normal_rmove2p             00405a84   PLCTRL.obj
 0001:00004aac       res_cmark_act              00405aac   RES_CMARKACT.obj
 0001:00004c88       res2_player_act            00405c88   RES_CMARKACT.obj
 0001:00004f4a       res2_timeobi_act           00405f4a   RES_CMARKACT.obj
 0001:000050f2       res2_winner_act            004060f2   RES_CMARKACT.obj
 0001:000053a8       record_RA                  004063a8   REC_RA.obj
 0001:00005b4c       setting_init               00406b4c   CS_SETTING.obj
 0001:00006025       setting_main               00407025   CS_SETTING.obj
 0001:000063ea       cslay0                     004073ea   CS_SETTING.obj
 0001:0000681b       cs_wait                    0040781b   CS_SETTING.obj
 0001:00006864       cslay1                     00407864   CS_SETTING.obj
 0001:00006b62       cslay2                     00407b62   CS_SETTING.obj
 0001:000070b0       cs_goto_blink              004080b0   CS_SETTING.obj
 0001:000071dc       cs_backto_save             004081dc   CS_SETTING.obj
 0001:000072cd       end_setting                004082cd   CS_SETTING.obj
 0001:0000734f       cs_cansel                  0040834f   CS_SETTING.obj
 0001:000073b6       cslay1to2                  004083b6   CS_SETTING.obj
 0001:0000741c       cslay2to1                  0040841c   CS_SETTING.obj
 0001:000074f9       cslay2to3                  004084f9   CS_SETTING.obj
 0001:00007586       line_scrl_m0               00408586   CS_SETTING.obj
 0001:000078ca       line_scrl_p0               004088ca   CS_SETTING.obj
 0001:00007b61       line_scrl_p1               00408b61   CS_SETTING.obj
 0001:00007d08       line_scrl_m1               00408d08   CS_SETTING.obj
 0001:00007e63       line_scrl_m2               00408e63   CS_SETTING.obj
 0001:00008137       line_scrl_p2               00409137   CS_SETTING.obj
 0001:000083bf       initial_parts_value        004093bf   CS_SETTING.obj
 0001:00008434       sel_new_car                00409434   CS_SETTING.obj
 0001:00008573       sel_tune_car               00409573   CS_SETTING.obj
 0001:00008702       check_padposi              00409702   CS_SETTING.obj
 0001:00008766       cs_put_parts_value         00409766   CS_SETTING.obj
 0001:000087e8       save_set_data              004097e8   CS_SETTING.obj
 0001:00008a40       put_car_type               00409a40   CS_SETTING.obj
 0001:00008ae1       cs_white_out               00409ae1   CS_SETTING.obj
 0001:00008b69       cs_white_out2              00409b69   CS_SETTING.obj
 0001:00008bf4       name_car_act               00409bf4   NAME_CAR.obj
 0001:00008d5c       _gfc_cmdload               00409d5c   tmp.obj
 0001:00008d60       _scroll_start_init         00409d60 f NScroll.obj
 0001:00008db0       _ChgSaturnColor2           00409db0 f NScroll.obj
 0001:00008e70       _DeleteScrollBitmapTable16 00409e70 f NScroll.obj
 0001:00008ec0       _LoadScrollBitmap16bit     00409ec0 f NScroll.obj
 0001:00008f00       _LoadScrollBitmap16bit_all 00409f00 f NScroll.obj
 0001:00008f30       _testCreateSurface16bit    00409f30 f NScroll.obj
 0001:00009120       _sprite_data_load          0040a120 f NScroll.obj
 0001:00009190       _make_pal                  0040a190 f NScroll.obj
 0001:000091a0       _sprite_init               0040a1a0 f NScroll.obj
 0001:00009200       _sprite_write              0040a200 f NScroll.obj
 0001:00009260       _sprite_rewrite            0040a260 f NScroll.obj
 0001:000092a0       _sprite_erace              0040a2a0 f NScroll.obj
 0001:00009310       _sprite_erace_all          0040a310 f NScroll.obj
 0001:00009370       _sprite_disp               0040a370 f NScroll.obj
 0001:000093b0       _sprite_move               0040a3b0 f NScroll.obj
 0001:00009400       _sprite_scroll             0040a400 f NScroll.obj
 0001:00009430       _sprite_change_scroll      0040a430 f NScroll.obj
 0001:00009470       _sprite_change_window      0040a470 f NScroll.obj
 0001:000094b0       _sprite_set_window         0040a4b0 f NScroll.obj
 0001:00009500       _sprite_reload             0040a500 f NScroll.obj
 0001:00009540       _sprite_remove             0040a540 f NScroll.obj
 0001:00009580       _scroll_init               0040a580 f NScroll.obj
 0001:000095e0       _scroll_write              0040a5e0 f NScroll.obj
 0001:00009640       _scroll_erace              0040a640 f NScroll.obj
 0001:000096b0       _scroll_disp               0040a6b0 f NScroll.obj
 0001:000096f0       _scroll_move               0040a6f0 f NScroll.obj
 0001:00009740       _scroll_scroll             0040a740 f NScroll.obj
 0001:00009770       _scroll_change             0040a770 f NScroll.obj
 0001:000097b0       _scroll_change_window      0040a7b0 f NScroll.obj
 0001:000097f0       _scroll_window_set         0040a7f0 f NScroll.obj
 0001:00009840       _scroll_reload             0040a840 f NScroll.obj
 0001:00009890       _scroll_data_read_16bit    0040a890 f NScroll.obj
 0001:00009950       _scroll_data_read          0040a950 f NScroll.obj
 0001:00009a10       _delete_allsurface         0040aa10 f NScroll.obj
 0001:00009a70       _scroll_data_erace         0040aa70 f NScroll.obj
 0001:00009ae0       _testCreateSurface         0040aae0 f NScroll.obj
 0001:00009d30       _testDestroySurface        0040ad30 f NScroll.obj
 0001:00009d80       _set_color_change_palette  0040ad80 f NScroll.obj
 0001:00009e00       _set_color_change_palette2 0040ae00 f NScroll.obj
 0001:00009e60       _rewrite_surface           0040ae60 f NScroll.obj
 0001:0000a020       _color_change_surface      0040b020 f NScroll.obj
 0001:0000a1d0       _get_change_color          0040b1d0 f NScroll.obj
 0001:0000a300       _write_surface             0040b300 f NScroll.obj
 0001:0000a490       _sprite_write_record_init  0040b490 f NScroll.obj
 0001:0000a500       _sprite_write_record_best  0040b500 f NScroll.obj
 0001:0000a910       _sprite_write_record_fast  0040b910 f NScroll.obj
 0001:0000ac90       sample_init                0040bc90   SAMPLE.obj
 0001:0000aeb2       sample_main                0040beb2   SAMPLE.obj
 0001:0000b2a3       camera_move                0040c2a3   SAMPLE.obj
 0001:0000b484       cube_act                   0040c484   SAMPLE.obj
 0001:0000b4e8       cube_init                  0040c4e8   SAMPLE.obj
 0001:0000b80f       object_control             0040c80f   SAMPLE.obj
 0001:0000b97d       draw_cube                  0040c97d   SAMPLE.obj
 0001:0000bc08       radar_act                  0040cc08   SAMPLE.obj
 0001:0000bd24       draw_radar                 0040cd24   SAMPLE.obj
 0001:0000bddc       draw_course_block          0040cddc   SAMPLE.obj
 0001:0000bef0       _setting_scroll_act_1      0040cef0 f setting.obj
 0001:0000bf60       _setting_scroll_act_2      0040cf60 f setting.obj
 0001:0000c000       _car_setting_init          0040d000 f setting.obj
 0001:0000c170       _car_setting_main          0040d170 f setting.obj
 0001:0000c380       _cs_lay0                   0040d380 f setting.obj
 0001:0000c630       _cs_lay1                   0040d630 f setting.obj
 0001:0000c750       _cs_lay2                   0040d750 f setting.obj
 0001:0000cda0       _init_parts_value          0040dda0 f setting.obj
 0001:0000ce60       _save_car_data             0040de60 f setting.obj
 0001:0000cf20       _set_sprite_disp           0040df20 f setting.obj
 0001:0000d200       _cs_sprite_bright          0040e200 f setting.obj
 0001:0000d500       _cslay2_sprite             0040e500 f setting.obj
 0001:0000d5c0       _button_sprite             0040e5c0 f setting.obj
 0001:0000d660       _setting_end               0040e660 f setting.obj
 0001:0000d680       _cs_cancel                 0040e680 f setting.obj
 0001:0000d6a0       _setting_scroll_change     0040e6a0 f setting.obj
 0001:0000dcd0       _setting_line_scroll       0040ecd0 f setting.obj
 0001:0000de10       _setting_scroll_init       0040ee10 f setting.obj
 0001:0000dee0       _setting_scroll_set        0040eee0 f setting.obj
 0001:0000e010       _setting_scroll_set_poly   0040f010 f setting.obj
 0001:0000e070       init_game_disp             0040f070   display.obj
 0001:0000e490       turn_around_disp           0040f490   display.obj
 0001:0000e508       turn_around_disp2p         0040f508   display.obj
 0001:0000e550       race_prac_title            0040f550   display.obj
 0001:0000e554       timeat_title               0040f554   display.obj
 0001:0000e555       record_sub                 0040f555   display.obj
 0001:0000e55c       freerun_title              0040f55c   display.obj
 0001:0000e560       vs_title                   0040f560   display.obj
 0001:0000e564       itacho_kmh                 0040f564   display.obj
 0001:0000e588       itacho_kmh1p               0040f588   display.obj
 0001:0000e5ac       base_position_disp         0040f5ac   display.obj
 0001:0000e5b0       best_number_disp           0040f5b0   display.obj
 0001:0000e5d4       best_number_disp_t         0040f5d4   display.obj
 0001:0000e5d8       re_1x1time_ft              0040f5d8   display.obj
 0001:0000e5e2       re_1x1time_2p              0040f5e2   display.obj
 0001:0000e664       laps_number_disp           0040f664   display.obj
 0001:0000e668       laps_number_disp_f         0040f668   display.obj
 0001:0000e66c       laps_number_disp_r         0040f66c   display.obj
 0001:0000e670       iresult_disp               0040f670   display.obj
 0001:0000e674       init_game_over             0040f674   display.obj
 0001:0000e678       reverse_display            0040f678   display.obj
 0001:0000e7ac       shift_display              0040f7ac   display.obj
 0001:0000e7cf       shift_display2p            0040f7cf   display.obj
 0001:0000e818       rank_display               0040f818   display.obj
 0001:0000e83c       lap_display2p              0040f83c   display.obj
 0001:0000e840       speed_display              0040f840   display.obj
 0001:0000e863       speed_display2p            0040f863   display.obj
 0001:0000e8ac       extend_time_display        0040f8ac   display.obj
 0001:0000eabc       extend_start_display       0040fabc   display.obj
 0001:0000ed38       sp_write                   0040fd38   display.obj
 0001:0000edbc       laptime_display            0040fdbc   display.obj
 0001:0000edf0       laptime_displayp           0040fdf0   display.obj
 0001:0000ee10       ld_sub                     0040fe10   display.obj
 0001:0000ee11       ld_sub2                    0040fe11   display.obj
 0001:0000ef3c       laptime_display1p          0040ff3c   display.obj
 0001:0000ef3c       laptime_display2p          0040ff3c   display.obj
 0001:0000efb4       laptime_displaylag         0040ffb4   display.obj
 0001:0000f00c       lap_rewrite                0041000c   display.obj
 0001:0000f010       lap_rewrite2p              00410010   display.obj
 0001:0000f03c       area_rewrite               0041003c   display.obj
 0001:0000f0dc       time1x1_display            004100dc   display.obj
 0001:0000f0e0       game_display               004100e0   display.obj
 0001:0000f2ac       timeattack                 004102ac   display.obj
 0001:0000f2ac       setting                    004102ac   display.obj
 0001:0000fdaf       speed_tbl                  00410daf   display.obj
 0001:0000ffb7       time10_tbl                 00410fb7   display.obj
 0001:0000ffb7       time_tbl                   00410fb7   display.obj
 0001:0000fff4       time100_tbl                00410ff4   display.obj
 0001:00010014       ending_init                00411014   ENDING.obj
 0001:00010014       __ending_init              00411014   ENDING.obj
 0001:0001033c       s_ending_init_poly         0041133c   ENDING.obj
 0001:0001039c       init_ending_work_start     0041139c   ENDING.obj
 0001:0001071c       ending_main                0041171c   ENDING.obj
 0001:0001071c       __ending_main              0041171c   ENDING.obj
 0001:00010887       game_main_ecom_ening       00411887   ENDING.obj
 0001:00010d26       get_staff_time             00411d26   ENDING.obj
 0001:00010ebc       set_staff_cg               00411ebc   ENDING.obj
 0001:00010f56       set_replay_camera_data     00411f56   ENDING.obj
 0001:00011028       staff_act_init             00412028   ENDING.obj
 0001:000110dc       staff_act                  004120dc   ENDING.obj
 0001:00011216       disp_staff_frame           00412216   ENDING.obj
 0001:0001134a       disp_staff_msg             0041234a   ENDING.obj
 0001:00011400       disp_staff_asc             00412400   ENDING.obj
 0001:0001151d       replay_camera_act          0041251d   ENDING.obj
 0001:0001151d       ending_camera_act          0041251d   ENDING.obj
 0001:00011588       replay_camera_main         00412588   ENDING.obj
 0001:000115e0       endcamera_turn             004125e0   ENDING.obj
 0001:00011611       endcamera_fix              00412611   ENDING.obj
 0001:000116ea       set_endcamera_type         004126ea   ENDING.obj
 0001:000117e0       set_endcamera_para         004127e0   ENDING.obj
 0001:000118c3       calc_endcamera_matrix      004128c3   ENDING.obj
 0001:00011a09       replay_pers_ctrl           00412a09   ENDING.obj
 0001:00011b57       set_game_pers              00412b57   ENDING.obj
 0001:00011b80       _PauseGame                 00412b80 f WinMain.obj
 0001:00011ba0       _UnPauseGame               00412ba0 f WinMain.obj
 0001:00011be0       _RestoreGame               00412be0 f WinMain.obj
 0001:00011c80       _GameMain                  00412c80 f WinMain.obj
 0001:00011da0       _initNumSurface            00412da0 f WinMain.obj
 0001:00011ff0       _DisplayFrameRate          00412ff0 f WinMain.obj
 0001:00012bf0       _MabikiCheck               00413bf0 f WinMain.obj
 0001:00012c40       _CheckMarkScreenRes        00413c40 f WinMain.obj
 0001:00012d10       _ChangeScreenRes           00413d10 f WinMain.obj
 0001:00012ef0       _SystemPause_SoundPause    00413ef0 f WinMain.obj
 0001:00012f00       _SystemPause_SoundResume   00413f00 f WinMain.obj
 0001:00012f20       _SystemPause               00413f20 f WinMain.obj
 0001:000131a0       _restart_game              004141a0 f WinMain.obj
 0001:000131d0       _ChangeScreenMode          004141d0 f WinMain.obj
 0001:00013360       _MainWndProc@16            00414360 f WinMain.obj
 0001:00014500       _ExitGame                  00415500 f WinMain.obj
 0001:00014560       _GetPixelShift             00415560 f WinMain.obj
 0001:00014660       _LoadPalette               00415660 f WinMain.obj
 0001:000146a0       _ChangePalette             004156a0 f WinMain.obj
 0001:000146e0       _InitGame                  004156e0 f WinMain.obj
 0001:00014ad0       _getint                    00415ad0 f WinMain.obj
 0001:00014b60       _WinMain@16                00415b60 f WinMain.obj
 0001:000151d0       _ChangeScale               004161d0 f WinMain.obj
 0001:00015210       _ChangePolyType            00416210 f WinMain.obj
 0001:00015240       _CheckRestatRace           00416240 f WinMain.obj
 0001:00015270       _InitMenuCheck             00416270 f WinMain.obj
 0001:00015600       sincos_tbl                 00416600   SINTBL.obj
 0001:00019600       atan_tbl                   0041a600   SINTBL.obj
 0001:00019a04       res_cmark_act_2            0041aa04   RES2_PLAYER.obj
 0001:00019c3c       timeact_init               0041ac3c   RES_TIMEACT.obj
 0001:00019ebf       timeact_act                0041aebf   RES_TIMEACT.obj
 0001:0001a3ac       rcopy                      0041b3ac   ETC.obj
 0001:0001a3f6       rcopyw                     0041b3f6   ETC.obj
 0001:0001a444       rfill                      0041b444   ETC.obj
 0001:0001a47c       rfillf                     0041b47c   ETC.obj
 0001:0001a48e       rfillff                    0041b48e   ETC.obj
 0001:0001a4c4       boxwrt_a                   0041b4c4   ETC.obj
 0001:0001a4d4       boxwrt_a2                  0041b4d4   ETC.obj
 0001:0001a4e4       boxwrt_a3                  0041b4e4   ETC.obj
 0001:0001a4f4       boxwrt_a4                  0041b4f4   ETC.obj
 0001:0001a504       boxwrt_b                   0041b504   ETC.obj
 0001:0001a514       boxwrt_b2                  0041b514   ETC.obj
 0001:0001a524       boxwrt_c                   0041b524   ETC.obj
 0001:0001a530       boxwrt_c2                  0041b530   ETC.obj
 0001:0001a53c       boxwrt_d                   0041b53c   ETC.obj
 0001:0001a548       boxwrt_d2                  0041b548   ETC.obj
 0001:0001a554       boxwrt_d3                  0041b554   ETC.obj
 0001:0001a560       boxwrt_a_nmap              0041b560   ETC.obj
 0001:0001a56c       boxwrt_b_nmap              0041b56c   ETC.obj
 0001:0001a578       boxwrt_c_nmap              0041b578   ETC.obj
 0001:0001a584       boxwrt_d_nmap              0041b584   ETC.obj
 0001:0001a590       boxwrt_word                0041b590   ETC.obj
 0001:0001a594       boxwrt_word2               0041b594   ETC.obj
 0001:0001a598       boxwrt_word3               0041b598   ETC.obj
 0001:0001a59c       boxwrt_long                0041b59c   ETC.obj
 0001:0001a5a0       boxwrt_long2               0041b5a0   ETC.obj
 0001:0001a5a4       boxwrt_long3               0041b5a4   ETC.obj
 0001:0001a5a8       boxwrt_long4               0041b5a8   ETC.obj
 0001:0001a5ac       boxwrt_word_nmap           0041b5ac   ETC.obj
 0001:0001a5b0       boxwrt_long_nmap           0041b5b0   ETC.obj
 0001:0001a5b4       boxclr_long                0041b5b4   ETC.obj
 0001:0001a634       boxclr_word                0041b634   ETC.obj
 0001:0001a6b8       fade_color_init            0041b6b8   ETC.obj
 0001:0001a868       get_time                   0041b868   ETC.obj
 0001:0001a86c       cd_open_check2             0041b86c   ETC.obj
 0001:0001a8f0       cd_open_check              0041b8f0   ETC.obj
 0001:0001a9e0       cd_open_checkg             0041b9e0   ETC.obj
 0001:0001aa70       clr_cmdtblbuf              0041ba70   SPRITE.obj
 0001:0001ab02       init_cmdtbl                0041bb02   SPRITE.obj
 0001:0001ab3c       set_cmdtbl                 0041bb3c   SPRITE.obj
 0001:0001abf6       set_sclip_cmd              0041bbf6   SPRITE.obj
 0001:0001ac9d       set_uclip_cmd              0041bc9d   SPRITE.obj
 0001:0001ad6c       set_lcoord_cmd             0041bd6c   SPRITE.obj
 0001:0001ae13       set_drawend_cmd            0041be13   SPRITE.obj
 0001:0001ae92       set_dummy_skip             0041be92   SPRITE.obj
 0001:0001af34       set_skip_assign            0041bf34   SPRITE.obj
 0001:0001afb3       chg_jump_cmd               0041bfb3   SPRITE.obj
 0001:0001aff2       set_erase_poly             0041bff2   SPRITE.obj
 0001:0001b179       set_demo_cmdtbl            0041c179   SPRITE.obj
 0001:0001b179       set_game_syscmdtbl         0041c179   SPRITE.obj
 0001:0001b235       draw_sprite                0041c235   SPRITE.obj
 0001:0001b238       record_connect             0041c238   REC_CONNECT.obj
 0001:0001b74b       time_disp                  0041c74b   REC_CONNECT.obj
 0001:0001b74b       putnum_1x2                 0041c74b   REC_CONNECT.obj
 0001:0001b74b       putnum_name2               0041c74b   REC_CONNECT.obj
 0001:0001b74b       putnum_rank2               0041c74b   REC_CONNECT.obj
 0001:0001b74b       putnum_Grn                 0041c74b   REC_CONNECT.obj
 0001:0001b74b       putnum_name                0041c74b   REC_CONNECT.obj
 0001:0001b74b       putnum_rank                0041c74b   REC_CONNECT.obj
 0001:0001b74b       putnum_rec                 0041c74b   REC_CONNECT.obj
 0001:0001b74b       putnum_Grn2                0041c74b   REC_CONNECT.obj
 0001:0001b74c       record_connect2            0041c74c   REC_CONNECT.obj
 0001:0001bf68       guide_africa               0041cf68   ndafrica.obj
 0001:0001d258       navi_display               0041e258   display3.obj
 0001:0001d417       init_navi                  0041e417   display3.obj
 0001:0001d418       count_down_start           0041e418   display3.obj
 0001:0001d4a0       count_init                 0041e4a0   display3.obj
 0001:0001d570       count_wait                 0041e570   display3.obj
 0001:0001d960       count_go                   0041e960   display3.obj
 0001:0001dbe4       count_down_start1p         0041ebe4   display3.obj
 0001:0001e160       set_bgmda_vs               0041f160   display3.obj
 0001:0001e25c       count_down_start2p         0041f25c   display3.obj
 0001:0001e924       count_down_start1p_net     0041f924   display3.obj
 0001:0001eec8       count_down_start2p_net     0041fec8   display3.obj
 0001:0001f4cc       timecmp_display_vs         004204cc   display3.obj
 0001:0001f584       vscmp_ndisp                00420584   display3.obj
 0001:0001f868       vscmp_disp_off             00420868   display3.obj
 0001:0001f910       vscmp_disp_end             00420910   display3.obj
 0001:0001fd34       timecmp_display_lag        00420d34   display3.obj
 0001:0001fe2c       lagcmp_disp_init           00420e2c   display3.obj
 0001:000200d0       reverse_display2p          004210d0   display3.obj
 0001:00020424       result_display2p           00421424   display3.obj
 0001:00020b7c       result_displaylag          00421b7c   display3.obj
 0001:00020e08       vs1st_display              00421e08   display3.obj
 0001:00020ecc       replay_display             00421ecc   display3.obj
 0001:00020fc4       init_replay_win            00421fc4   display3.obj
 0001:00020fc8       pause_display              00421fc8   display3.obj
 0001:00020fc9       pause_display2             00421fc9   display3.obj
 0001:00020fcc       pause_delete               00421fcc   display3.obj
 0001:00020fd0       pause_cursor               00421fd0   display3.obj
 0001:0002108c       adv_vdp2_display           0042208c   display3.obj
 0001:0002170c       init_adv_map               0042270c   display3.obj
 0001:00021710       ending_vdp2_display        00422710   display3.obj
 0001:000217a0       count_down_start_ending    004227a0   display3.obj
 0001:00021c3c       count_down_start_replay    00422c3c   display3.obj
 0001:0002255c       resreplay_display          0042355c   display3.obj
 0001:000225d4       rep_res_init               004235d4   display3.obj
 0001:00022a44       tinyOther                  00423a44   OTHERSUB.obj
 0001:00023655       simpleOther                00424655   OTHERSUB.obj
 0001:00024ad4       OtherCarCtrl               00425ad4   OTHERSUB.obj
 0001:00024f00       set_target_pos             00425f00   OTHERSUB.obj
 0001:000252fc       set_target_spd             004262fc   OTHERSUB.obj
 0001:00025878       getAngle                   00426878   OTHERSUB.obj
 0001:00025cd5       setVelocity                00426cd5   OTHERSUB.obj
 0001:0002649c       outer_product_p            0042749c   CAR.obj
 0001:000266e0       regvect_inner              004276e0   CAR.obj
 0001:000268f0       vecval                     004278f0   CAR.obj
 0001:000269c8       vecval_2                   004279c8   CAR.obj
 0001:00026a64       regvect                    00427a64   CAR.obj
 0001:00026c64       calc_xyzpoint              00427c64   CAR.obj
 0001:00026ed8       calc_rad                   00427ed8   CAR.obj
 0001:000272d4       calc_reverse               004282d4   CAR.obj
 0001:000273dc       calc_dispang               004283dc   CAR.obj
 0001:000273e6       calc_dispang2p             004283e6   CAR.obj
 0001:00027514       calc_dispang2              00428514   CAR.obj
 0001:0002762c       spline                     0042862c   CAR.obj
 0001:00027af8       get_block                  00428af8   CAR.obj
 0001:00027db4       inspect_polygon_b          00428db4   CAR.obj
 0001:00028200       get_coli_area              00429200   CAR.obj
 0001:000282b4       get_y                      004292b4   CAR.obj
 0001:00028408       get_d                      00429408   CAR.obj
 0001:000285a4       inspect_polygon            004295a4   CAR.obj
 0001:000285b1       inspect_polygon2           004295b1   CAR.obj
 0001:00028b8c       get_poly_map               00429b8c   CAR.obj
 0001:00028eb8       get_other_map              00429eb8   CAR.obj
 0001:00028f88       get_poly_map1p             00429f88   CAR.obj
 0001:00028fe0       get_poly_map2p             00429fe0   CAR.obj
 0001:000292d8       get_poly_map1p_net         0042a2d8   CAR.obj
 0001:00029330       get_poly_map2p_net         0042a330   CAR.obj
 0001:0002960c       get_block2                 0042a60c   CAR.obj
 0001:000297d4       get_coli2                  0042a7d4   CAR.obj
 0001:000298c0       get_coli3                  0042a8c0   CAR.obj
 0001:00029bcc       vs_rank_calc               0042abcc   CAR.obj
 0001:00029e58       valtobit_w                 0042ae58   CAR.obj
 0001:00029e8e       w_valtobit_tbl             0042ae8e   CAR.obj
 0001:00029eb0       make_gswdata               0042aeb0   CAR.obj
 0001:0002a170       pl1p_or_switch             0042b170   CAR.obj
 0001:0002a18c       pl2p_or_switch             0042b18c   CAR.obj
 0001:0002a1a8       view_changer2p             0042b1a8   CAR.obj
 0001:0002a1b4       view_changer1p             0042b1b4   CAR.obj
 0001:0002a1ef       view_changer               0042b1ef   CAR.obj
 0001:0002a264       config_keyset              0042b264   CAR.obj
 0001:0002a520       bpeset                     0042b520   EXTDATA.obj
 0001:0002af18       set_pict_2p_battle         0042bf18   CS_BATTLE_2P_PSET.obj
 0001:0002b1f6       bt_move_picture            0042c1f6   CS_BATTLE_2P_PSET.obj
 0001:0002b367       bt_pict_bright_1p          0042c367   CS_BATTLE_2P_PSET.obj
 0001:0002b6bc       bt_pict_bright_2p          0042c6bc   CS_BATTLE_2P_PSET.obj
 0001:0002b910       pict_bright_btlay1_2       0042c910   CS_BATTLE_2P_PSET.obj
 0001:0002b936       pict_bright_btlay2_2       0042c936   CS_BATTLE_2P_PSET.obj
 0001:0002ba40       bt_chg_c_name_1p           0042ca40   CS_BATTLE_2P_PSET.obj
 0001:0002bb98       bt_chg_c_name_2p           0042cb98   CS_BATTLE_2P_PSET.obj
 0001:0002bcf0       delete_all_btlay1          0042ccf0   CS_BATTLE_2P_PSET.obj
 0001:0002bd2c       delete_all_btlay2          0042cd2c   CS_BATTLE_2P_PSET.obj
 0001:0002bd68       re_draw_btlay1             0042cd68   CS_BATTLE_2P_PSET.obj
 0001:0002be1c       re_draw_btlay2             0042ce1c   CS_BATTLE_2P_PSET.obj
 0001:0002bed0       bt_chg_crs_name            0042ced0   CS_BATTLE_2P_PSET.obj
 0001:0002c221       bt_chg_lap_name            0042d221   CS_BATTLE_2P_PSET.obj
 0001:0002c342       bt_chg_delay               0042d342   CS_BATTLE_2P_PSET.obj
 0001:0002c44e       bt_chg_on_off              0042d44e   CS_BATTLE_2P_PSET.obj
 0001:0002c55a       bt_chg_lag                 0042d55a   CS_BATTLE_2P_PSET.obj
 0001:0002c596       bt_draw_number_6           0042d596   CS_BATTLE_2P_PSET.obj
 0001:0002c789       bt_draw_others             0042d789   CS_BATTLE_2P_PSET.obj
 0001:0002ca66       bt_draw_number_8           0042da66   CS_BATTLE_2P_PSET.obj
 0001:0002cc24       delete_btlay1_0            0042dc24   CS_BATTLE_2P_PSET.obj
 0001:0002ccdc       delete_btlay2_0            0042dcdc   CS_BATTLE_2P_PSET.obj
 0001:0002cd94       delete_btlay1_1            0042dd94   CS_BATTLE_2P_PSET.obj
 0001:0002ce54       delete_btlay2_1            0042de54   CS_BATTLE_2P_PSET.obj
 0001:0002cf14       delete_btlay3              0042df14   CS_BATTLE_2P_PSET.obj
 0001:0002cf83       bt_set_pict_result         0042df83   CS_BATTLE_2P_PSET.obj
 0001:0002d124       bt_ret_bt_2p               0042e124   CS_BATTLE_2P_PSET.obj
 0001:0002d153       bt_set_bt_2p               0042e153   CS_BATTLE_2P_PSET.obj
 0001:0002d153       __bt_set_bt_2p             0042e153   CS_BATTLE_2P_PSET.obj
 0001:0002d9d4       record_csort               0042e9d4   REC_TSORT.obj
 0001:0002dd4b       record_2sort               0042ed4b   REC_TSORT.obj
 0001:0002df0f       record_c2sort              0042ef0f   REC_TSORT.obj
 0001:0002df83       record_tmsort              0042ef83   REC_TSORT.obj
 0001:0002e015       record_ctmsort             0042f015   REC_TSORT.obj
 0001:0002e1c0       _bt_move_sprite            0042f1c0 f BATTLE_2P.obj
 0001:0002e330       _bt_sprite_bright_1p       0042f330 f BATTLE_2P.obj
 0001:0002e460       _bt_sprite_bright_2p       0042f460 f BATTLE_2P.obj
 0001:0002e590       _bt_disp_sprite2           0042f590 f BATTLE_2P.obj
 0001:0002e5a0       _re_draw_btlay1            0042f5a0 f BATTLE_2P.obj
 0001:0002e620       _re_draw_btlay2            0042f620 f BATTLE_2P.obj
 0001:0002e6b0       _bt_course_bright_1p       0042f6b0 f BATTLE_2P.obj
 0001:0002e740       _bt_laps_bright_1p         0042f740 f BATTLE_2P.obj
 0001:0002e7b0       _disp_tune_car_1p          0042f7b0 f BATTLE_2P.obj
 0001:0002e850       _disp_tune_car_2p          0042f850 f BATTLE_2P.obj
 0001:0002e8f0       _bt_tune_bright_1p         0042f8f0 f BATTLE_2P.obj
 0001:0002e960       _bt_tune_bright_2p         0042f960 f BATTLE_2P.obj
 0001:0002e9d0       _set_crs_sprite            0042f9d0 f BATTLE_2P.obj
 0001:0002eb30       _set_laps_sprite           0042fb30 f BATTLE_2P.obj
 0001:0002ec80       record_request             0042fc80   REC_REQUEST.obj
 0001:0002f6b0       _WaveOpen                  004306b0 f DS.obj
 0001:0002f720       _WaveLoad                  00430720 f DS.obj
 0001:0002fa90       _SetDSBuffer               00430a90 f DS.obj
 0001:0002ff80       _WaveRequest               00430f80 f DS.obj
 0001:00030100       _WavePlay                  00431100 f DS.obj
 0001:000301b0       _WaveStop                  004311b0 f DS.obj
 0001:00030260       _ALLStop                   00431260 f DS.obj
 0001:00030360       _EnginePause               00431360 f DS.obj
 0001:000303e0       _ENGStop                   004313e0 f DS.obj
 0001:00030450       _WavePause                 00431450 f DS.obj
 0001:00030580       _WaveResume                00431580 f DS.obj
 0001:00030680       _WaveFree                  00431680 f DS.obj
 0001:000306f0       _WaveCloseEngine           004316f0 f DS.obj
 0001:00030740       _WaveCloseGame             00431740 f DS.obj
 0001:000307b0       _WaveClose                 004317b0 f DS.obj
 0001:00030880       _GetWaveStatus             00431880 f DS.obj
 0001:000308d0       _GetWaveInfo               004318d0 f DS.obj
 0001:00030920       _EngineSet                 00431920 f DS.obj
 0001:00030970       _Engine2pSet               00431970 f DS.obj
 0001:000309c0       _EngineSound               004319c0 f DS.obj
 0001:00030c30       _Engine2pSound             00431c30 f DS.obj
 0001:00030ef0       _ReadTable                 00431ef0 f DS.obj
 0001:00030fc0       _WaveCtrl                  00431fc0 f DS.obj
 0001:000310f0       _SlipSound                 004320f0 f DS.obj
 0001:00031240       _Henkan                    00432240 f DS.obj
 0001:00031760       _bankchg                   00432760 f DS.obj
 0001:00031770       _EngineInit                00432770 f DS.obj
 0001:00031860       _ENGSound                  00432860 f DS.obj
 0001:00031880       _ENG2pSound                00432880 f DS.obj
 0001:000318a0       _roadNoise                 004328a0 f DS.obj
 0001:000318c0       _WaveWater                 004328c0 f DS.obj
 0001:000318f0       _Navi                      004328f0 f DS.obj
 0001:00031a80       _SetVol                    00432a80 f DS.obj
 0001:00031a90       _SeqVol                    00432a90 f DS.obj
 0001:00031aa0       _SetVol0                   00432aa0 f DS.obj
 0001:00031ab0       _ChkWater                  00432ab0 f DS.obj
 0001:00031b70       _WaterStop                 00432b70 f DS.obj
 0001:00031c00       _SEStop                    00432c00 f DS.obj
 0001:00031cb0       _pcmplay                   00432cb0 f DS.obj
 0001:00031cd0       _SDMPlay                   00432cd0 f DS.obj
 0001:00032150       _DJ_play                   00433150 f DS.obj
 0001:00032180       _wave_end_chk              00433180 f DS.obj
 0001:00032200       _WevBank_Load              00433200 f DS.obj
 0001:00032210       _ErrorMessage              00433210 f gameproc.obj
 0001:00032260       _InitBuffer                00433260 f gameproc.obj
 0001:000322d0       _DestroyBuffer             004332d0 f gameproc.obj
 0001:00032330       _PreInitializeGame         00433330 f gameproc.obj
 0001:000323a0       _InitializeGame            004333a0 f gameproc.obj
 0001:000323b0       _error_print               004333b0 f gameproc.obj
 0001:00032440       _ClipFrameDisp             00433440 f gameproc.obj
 0001:00032490       _PitchCheck                00433490 f gameproc.obj
 0001:000324a0       _draw_takeya               004334a0 f gameproc.obj
 0001:00032fe0       _NewGameFrame              00433fe0 f gameproc.obj
 0001:000334f0       _DestroyGame               004344f0 f gameproc.obj
 0001:00033560       _DispModeSelectDisp        00434560 f gameproc.obj
 0001:00033630       __ClearFrame               00434630 f gameproc.obj
 0001:00033700       judgement_scrl             00434700   SCRLMOVE.obj
 0001:00033955       judge_scrl                 00434955   SCRLMOVE.obj
 0001:00033a6d       judge_a_scrl               00434a6d   SCRLMOVE.obj
 0001:00033de0       _ChangeSelectDisplayMode   00434de0 f SaturnMain.obj
 0001:00033e50       _ChangeGameDisplayMode     00434e50 f SaturnMain.obj
 0001:00033ec0       _SaturnMain                00434ec0 f SaturnMain.obj
 0001:000349a0       _result_sub2               004359a0 f SaturnMain.obj
 0001:00034c30       _result_sub                00435c30 f SaturnMain.obj
 0001:000355c0       _AdrChange                 004365c0 f SaturnSim.obj
 0001:00035630       _DIV_FIXED_C               00436630 f SaturnSim.obj
 0001:00035690       _MyDiv64                   00436690 f SaturnSim.obj
 0001:00035760       _Div64R0R1_R2              00436760 f SaturnSim.obj
 0001:00035830       _Div64R0R1_R3              00436830 f SaturnSim.obj
 0001:00035900       _Div64R0R4_R1              00436900 f SaturnSim.obj
 0001:000359d0       _Div64R1R2_R3              004369d0 f SaturnSim.obj
 0001:00035aa0       _Div64R1R2_R5              00436aa0 f SaturnSim.obj
 0001:00035b70       _Div64R1R2_R6              00436b70 f SaturnSim.obj
 0001:00035c40       _Div64R1R10_R2             00436c40 f SaturnSim.obj
 0001:00035d10       _Div64R2R1_R3              00436d10 f SaturnSim.obj
 0001:00035de0       _Div64R2R3_R1              00436de0 f SaturnSim.obj
 0001:00035eb0       _Div64R3R1_R2              00436eb0 f SaturnSim.obj
 0001:00035f80       _Div64R3R2_R1              00436f80 f SaturnSim.obj
 0001:00036050       _Div64R3R4_R1              00437050 f SaturnSim.obj
 0001:00036120       _Div64R3R4_R6              00437120 f SaturnSim.obj
 0001:000361f0       _Div64R3R5_R7              004371f0 f SaturnSim.obj
 0001:000362c0       _Div64R4R3_R2              004372c0 f SaturnSim.obj
 0001:00036390       _Div64R5R6_R7              00437390 f SaturnSim.obj
 0001:00036460       _Div64R6R7_R0              00437460 f SaturnSim.obj
 0001:00036530       _Div64R8R9_R1              00437530 f SaturnSim.obj
 0001:00036600       _Div64R10R1_R2             00437600 f SaturnSim.obj
 0001:000366d0       _Div64R0_R3                004376d0 f SaturnSim.obj
 0001:000367d0       _Div64R0_R1                004377d0 f SaturnSim.obj
 0001:000368d0       _Div64R0_R4                004378d0 f SaturnSim.obj
 0001:000369d0       _Div64R0_R2                004379d0 f SaturnSim.obj
 0001:00036ad0       _Div64R1_R0                00437ad0 f SaturnSim.obj
 0001:00036bd0       _Div64R1_R4                00437bd0 f SaturnSim.obj
 0001:00036cd0       _Div64R2_R3                00437cd0 f SaturnSim.obj
 0001:00036dd0       _Div64R4_R5                00437dd0 f SaturnSim.obj
 0001:00036ed0       _Div64R5_R4                00437ed0 f SaturnSim.obj
 0001:00036fd0       _Div32R1_R0                00437fd0 f SaturnSim.obj
 0001:000370a0       _gfc_cdplay                004380a0 f SaturnSim.obj
 0001:000370b0       _SlaveSHOn                 004380b0 f SaturnSim.obj
 0001:000370c0       _PER_Init                  004380c0 f SaturnSim.obj
 0001:000370d0       _PER_GetPer                004380d0 f SaturnSim.obj
 0001:000370e0       _PER_LInit                 004380e0 f SaturnSim.obj
 0001:000370f0       _PER_LGetPer               004380f0 f SaturnSim.obj
 0001:00037100       _PER_GetSys                00438100 f SaturnSim.obj
 0001:00037110       _per_getsys                00438110 f SaturnSim.obj
 0001:00037120       _PER_IntFunc               00438120 f SaturnSim.obj
 0001:00037130       _res_ei                    00438130 f SaturnSim.obj
 0001:00037140       _res_di                    00438140 f SaturnSim.obj
 0001:00037150       _SYS_CheckTrack            00438150 f SaturnSim.obj
 0001:00037160       _SYS_Exit                  00438160 f SaturnSim.obj
 0001:00037170       _gfc_cdpause               00438170 f SaturnSim.obj
 0001:00037180       _SlaveSHOff                00438180 f SaturnSim.obj
 0001:00037190       _gfc_cdseek                00438190 f SaturnSim.obj
 0001:000371a0       _gfc_cdstat                004381a0 f SaturnSim.obj
 0001:000371b0       _per_get_time_adr          004381b0 f SaturnSim.obj
 0001:000371c0       _CDC_GetPeriStat           004381c0 f SaturnSim.obj
 0001:000371d0       _SoundOff                  004381d0 f SaturnSim.obj
 0001:000371e0       _SoundOn                   004381e0 f SaturnSim.obj
 0001:000371f0       _gfc_cdrestart             004381f0 f SaturnSim.obj
 0001:00037200       _per_get_sys               00438200 f SaturnSim.obj
 0001:00037210       _GetPaletteIndex           00438210 f SaturnSim.obj
 0001:00037220       _ChgSaturnColor            00438220 f SaturnSim.obj
 0001:00037350       _set_polygon_scale         00438350 f SaturnSim.obj
 0001:00037770       _Poly_DC                   00438770 f SaturnSim.obj
 0001:00037980       _SuturnPolygon             00438980 f SaturnSim.obj
 0001:00037c40       _SuturnTransformSprite     00438c40 f SaturnSim.obj
 0001:00037f60       _CnvTexture                00438f60 f SaturnSim.obj
 0001:00038230       _SpriteCmdClr              00439230 f SaturnSim.obj
 0001:00038240       _SpriteCmdOut              00439240 f SaturnSim.obj
 0001:000383f0       _SpriteCmdOut2p            004393f0 f SaturnSim.obj
 0001:00038700       _SpriteCmdOutNet           00439700 f SaturnSim.obj
 0001:00038a10       _SpriteCmdOut_DC           00439a10 f SaturnSim.obj
 0001:00038bc0       _Convert4bit               00439bc0 f SaturnSim.obj
 0001:00038c00       _Convert4bitLookup         00439c00 f SaturnSim.obj
 0001:00038ea0       _PalHistInit               00439ea0 f SaturnSim.obj
 0001:00038ec0       _PalHistDump               00439ec0 f SaturnSim.obj
 0001:00038f50       _HistCheck                 00439f50 f SaturnSim.obj
 0001:00039060       _PaletteCacheClr           0043a060 f SaturnSim.obj
 0001:00039090       _RGB16ToPaletteNo          0043a090 f SaturnSim.obj
 0001:00039270       _RGB16ToPaletteNoOld       0043a270 f SaturnSim.obj
 0001:000392e0       _Convert4bitLookupPal      0043a2e0 f SaturnSim.obj
 0001:000395a0       _Convert6bit               0043a5a0 f SaturnSim.obj
 0001:000395e0       _Convert7bit               0043a5e0 f SaturnSim.obj
 0001:00039620       _Convert8bit               0043a620 f SaturnSim.obj
 0001:00039660       _Convert16bit              0043a660 f SaturnSim.obj
 0001:000396a0       _set_alpha_color           0043a6a0 f SaturnSim.obj
 0001:00039770       record_rec_disp            0043a770   REC_DISP.obj
 0001:00039fc2       record_name_disp           0043afc2   REC_DISP.obj
 0001:0003a1bd       record_2x2_disp            0043b1bd   REC_DISP.obj
 0001:0003a274       record_spc_disp            0043b274   REC_DISP.obj
 0001:0003a2bf       record_spc_disp_l          0043b2bf   REC_DISP.obj
 0001:0003a309       boxdisp                    0043b309   REC_DISP.obj
 0001:0003a395       boxdisp2                   0043b395   REC_DISP.obj
 0001:0003a420       clip2d_4                   0043b420   CLIP2D.obj
 0001:0003a750       clip2d_3                   0043b750   CLIP2D.obj
 0001:0003a966       beta_clip2d_4              0043b966   CLIP2D.obj
 0001:0003aaf8       beta_clip2d_3              0043baf8   CLIP2D.obj
 0001:0003ac9c       get_clip2d_flag            0043bc9c   CLIP2D.obj
 0001:0003ad88       get_hvminmax3              0043bd88   CLIP2D.obj
 0001:0003aee0       get_hvminmax_sub           0043bee0   CLIP2D.obj
 0001:0003b0a4       chk_poly_out_screen        0043c0a4   CLIP2D.obj
 0001:0003b140       chk_poly_in_screen         0043c140   CLIP2D.obj
 0001:0003b1dc       chk_in_frame               0043c1dc   CLIP2D.obj
 0001:0003b260       sort_cmd_vert              0043c260   CLIP2D.obj
 0001:0003b624       sort_vert_b                0043c624   CLIP2D.obj
 0001:0003b784       sort_vert_c                0043c784   CLIP2D.obj
 0001:0003b8e4       sort_vert_d                0043c8e4   CLIP2D.obj
 0001:0003ba44       exchg_cmdvert              0043ca44   CLIP2D.obj
 0001:0003bc54       get_most_near_vert         0043cc54   CLIP2D.obj
 0001:0003bf0b       clip2d_main                0043cf0b   CLIP2D.obj
 0001:0003c032       beta_clip2d                0043d032   CLIP2D.obj
 0001:0003c170       sort_clip2d_vert           0043d170   CLIP2D.obj
 0001:0003c7a0       set_clip2dbuf              0043d7a0   CLIP2D.obj
 0001:0003c9ab       v_clip                     0043d9ab   CLIP2D.obj
 0001:0003ce88       set_cp_v                   0043de88   CLIP2D.obj
 0001:0003cf84       get_cp_v                   0043df84   CLIP2D.obj
 0001:0003d114       h_clip                     0043e114   CLIP2D.obj
 0001:0003d582       set_cp_h                   0043e582   CLIP2D.obj
 0001:0003d5f7       get_cp_h                   0043e5f7   CLIP2D.obj
 0001:0003d760       set_clip2d_poly            0043e760   CLIP2D.obj
 0001:0003eb2c       get_vertice_data           0043fb2c   CLIP2D.obj
 0001:0003ecf4       sort_cmd_vert2             0043fcf4   CLIP2D.obj
 0001:0003f398       guide_corse                00440398   ndcorse.obj
 0001:00040690       _WhiteFadeSet              00441690 f fade.obj
 0001:000408b0       _WhiteFadeSetPal           004418b0 f fade.obj
 0001:00040990       _FadeCtrl8                 00441990 f fade.obj
 0001:000409b0       _FadeCtrl16                004419b0 f fade.obj
 0001:000409d0       _FadeOff                   004419d0 f fade.obj
 0001:00040a00       result2p_main              00441a00   RES2_MAIN.obj
 0001:00040a00       __result2p_main            00441a00   RES2_MAIN.obj
 0001:00040fef       result2p_main_loop         00441fef   RES2_MAIN.obj
 0001:00040fef       __result2p_main_loop       00441fef   RES2_MAIN.obj
 0001:000416fc       hitCheck2                  004426fc   CARCOLI.obj
 0001:00041874       get_coli_ball              00442874   CARCOLI.obj
 0001:00042118       hitCheck                   00443118   CARCOLI.obj
 0001:00042a0c       carColiGP                  00443a0c   CARCOLI.obj
 0001:00042b11       carColiOtr                 00443b11   CARCOLI.obj
 0001:00043017       carColiVS                  00444017   CARCOLI.obj
 0001:00043134       balldemo_init              00444134   BALLDEMO.obj
 0001:00043325       sl_balldemo_init           00444325   BALLDEMO.obj
 0001:0004334d       balldemo_main              0044434d   BALLDEMO.obj
 0001:000437cc       sl_balldemo_main           004447cc   BALLDEMO.obj
 0001:0004385c       ball_act                   0044485c   BALLDEMO.obj
 0001:000438c0       ball_init                  004448c0   BALLDEMO.obj
 0001:00043b4f       draw_ball                  00444b4f   BALLDEMO.obj
 0001:00043c39       floor_act                  00444c39   BALLDEMO.obj
 0001:00043c9c       floor_init                 00444c9c   BALLDEMO.obj
 0001:00043d96       draw_floor                 00444d96   BALLDEMO.obj
 0001:00043fc6       checkdemo_init             00444fc6   BALLDEMO.obj
 0001:0004416d       checkdemo_main             0044516d   BALLDEMO.obj
 0001:00044418       car_act                    00445418   BALLDEMO.obj
 0001:00044481       car_act_main               00445481   BALLDEMO.obj
 0001:000444e4       light_act                  004454e4   BALLDEMO.obj
 0001:0004464c       InitKickback               0044564c   STEER.obj
 0001:0004464d       getIO                      0044564d   STEER.obj
 0001:000446a8       KickbackOff                004456a8   STEER.obj
 0001:000446ca       KickbackSetCenter          004456ca   STEER.obj
 0001:000446cb       KickbackCentering          004456cb   STEER.obj
 0001:000446cc       getSteer                   004456cc   STEER.obj
 0001:0004476f       KickbackCtrl               0044576f   STEER.obj
 0001:00044770       _PauseInit                 00445770 f winapi.obj
 0001:00044950       _PauseEnd                  00445950 f winapi.obj
 0001:00044990       _PauseDraw                 00445990 f winapi.obj
 0001:00044bd0       _MyConfigWrite             00445bd0 f winapi.obj
 0001:00044d80       _Load16BMP                 00445d80 f winapi.obj
 0001:00045020       _MyConfigRead              00446020 f winapi.obj
 0001:000453a0       _CDInsertCheck_sub         004463a0 f winapi.obj
 0001:00045430       _CDInsertCheck             00446430 f winapi.obj
 0001:00045500       _EnumWindowsProc@8         00446500 f winapi.obj
 0001:00045570       _SetCheckMark              00446570 f winapi.obj
 0001:000455b0       _SetMenuEnable             004465b0 f winapi.obj
 0001:000455f0       _MenuEnable                004465f0 f winapi.obj
 0001:00045670       _SetMenuNo                 00446670 f winapi.obj
 0001:00045690       PowerInit                  00446690   POWER.obj
 0001:0004585f       PowerGet                   0044685f   POWER.obj
 0001:000466bc       PowerUse                   004476bc   POWER.obj
 0001:0004684f       TorqueGet                  0044784f   POWER.obj
 0001:00046b01       engineSoundInit            00447b01   POWER.obj
 0001:00046b29       engineSound                00447b29   POWER.obj
 0001:00046b2a       wasteGateInit              00447b2a   POWER.obj
 0001:00046b68       wasteGateCtrl              00447b68   POWER.obj
 0001:00046f70       SoundEnableFlagTbl         00447f70   POWER.obj
 0001:00046f78       getGear                    00447f78   POWER.obj
 0001:000470e6       getGearAT                  004480e6   POWER.obj
 0001:00047350       getBrake                   00448350   POWER.obj
 0001:000477f8       load_dsp_program           004487f8   DSP.obj
 0001:000478a0       dsp_init                   004488a0   DSP.obj
 0001:000478bc       dsp_program_data           004488bc   DSP.obj
 0001:000478c0       dsp_calc_vertices          004488c0   DSP.obj
 0001:000479b5       dsp_wait                   004489b5   DSP.obj
 0001:000479f4       guide_europe               004489f4   ndeurope.obj
 0001:00048ce4       start_init                 00449ce4   STARThattori.obj
 0001:00048ce4       __start_init               00449ce4   STARThattori.obj
 0001:0004965c       __ceremony_init            0044a65c   CEREMONY.obj
 0001:0004965c       ceremony_init              0044a65c   CEREMONY.obj
 0001:00049a33       ceremony_main              0044aa33   CEREMONY.obj
 0001:00049e94       ceremony_camera_act        0044ae94   CEREMONY.obj
 0001:0004a694       get_camera_angle           0044b694   CEREMONY.obj
 0001:0004a7e8       ceremony_car_act           0044b7e8   CEREMONY.obj
 0001:0004a873       ceremony_car_main          0044b873   CEREMONY.obj
 0001:0004a9f8       DrawStage                  0044b9f8   CEREMONY.obj
 0001:0004aabf       InitCeremonyCar            0044babf   CEREMONY.obj
 0001:0004ac24       InitKamifubuki             0044bc24   CEREMONY.obj
 0001:0004acec       rndKami                    0044bcec   CEREMONY.obj
 0001:0004b040       Kamifubuki                 0044c040   CEREMONY.obj
 0001:0004b0ae       kami_act                   0044c0ae   CEREMONY.obj
 0001:0004b463       driver_act                 0044c463   CEREMONY.obj
 0001:0004b8a0       _cd_GetFileSize            0044c8a0 f Cdload.obj
 0001:0004b970       _PNT_Offset                0044c970 f Cdload.obj
 0001:0004b9b0       _tire_poly_color_patch     0044c9b0 f Cdload.obj
 0001:0004b9e0       _cd_load_patch             0044c9e0 f Cdload.obj
 0001:0004c320       _cd_load                   0044d320 f Cdload.obj
 0001:0004c470       _cd_load2                  0044d470 f Cdload.obj
 0001:0004c580       _cd_load_course_expand     0044d580 f Cdload.obj
 0001:0004c700       _LoadEventData_C           0044d700 f Cdload.obj
 0001:0004c730       _mad_patch                 0044d730 f Cdload.obj
 0001:0004c9b0       _gfc_madload               0044d9b0 f Cdload.obj
 0001:0004cb90       _PHOTOTBL_Load             0044db90 f Cdload.obj
 0001:0004cdc0       poweron_start              0044ddc0   BOOT.obj
 0001:0004d0f4       watanabe_init              0044e0f4   AC_G_SELECT.obj
 0001:0004d4dc       __g_select_init            0044e4dc   AC_G_SELECT.obj
 0001:0004d4dc       g_select_init              0044e4dc   AC_G_SELECT.obj
 0001:0004d979       g_select_main              0044e979   AC_G_SELECT.obj
 0001:0004dbda       g_white_in                 0044ebda   AC_G_SELECT.obj
 0001:0004dc9a       g_check_pad                0044ec9a   AC_G_SELECT.obj
 0001:0004e049       draw_champ                 0044f049   AC_G_SELECT.obj
 0001:0004e259       draw_prac                  0044f259   AC_G_SELECT.obj
 0001:0004f8c0       _InitJoystick              004508c0 f joyctrl.obj
 0001:0004f9f0       _ReadJoystick              004509f0 f joyctrl.obj
 0001:0004fae0       init_action                00450ae0   ACTION.obj
 0001:0004fb1a       act_loop                   00450b1a   ACTION.obj
 0001:0004fbb1       draw_loop                  00450bb1   ACTION.obj
 0001:0004fc49       clear_all_action_status    00450c49   ACTION.obj
 0001:0004fc5d       clear_action_status        00450c5d   ACTION.obj
 0001:0004fce8       set_action                 00450ce8   ACTION.obj
 0001:0004fdd8       check_control              00450dd8   ACTION.obj
 0001:0004ff0c       time_pict_set              00450f0c   AC_PICT_SET.obj
 0001:00050037       set_pict_ac_g_select       00451037   AC_PICT_SET.obj
 0001:000505d8       set_pict_ac_c_select       004515d8   AC_PICT_SET.obj
 0001:00050da4       set_pict_ac_crs_select     00451da4   AC_PICT_SET.obj
 0001:0005143c       record_menu                0045243c   REC_MENU2.obj
 0001:000519e4       record_dataset             004529e4   REC_DATASET.obj
 0001:00051a3c       recordtime_setup           00452a3c   REC_DATASET.obj
 0001:000525a0       set_default_ghost          004535a0   REC_DATASET.obj
 0001:0005260a       cmptime_setup              0045360a   REC_DATASET.obj
 0001:00052870       init_system                00453870   VDP.obj
 0001:00052874       init_vect_slave            00453874   VDP.obj
 0001:00052890       int_mask_set               00453890   VDP.obj
 0001:00052894       init_smpcif                00453894   VDP.obj
 0001:00052898       pad_kind_init              00453898   VDP.obj
 0001:0005289c       pad_kind                   0045389c   VDP.obj
 0001:000528b8       init_vram                  004538b8   VDP.obj
 0001:000528f8       vram_allclr                004538f8   VDP.obj
 0001:00052970       vram_scrmap_clr            00453970   VDP.obj
 0001:000529a0       vram_scrmap_clr2           004539a0   VDP.obj
 0001:00052aa4       vram_scrmap_a_clr          00453aa4   VDP.obj
 0001:00052ad4       vram_scrmap_b_clr          00453ad4   VDP.obj
 0001:00052b04       vram_scrmap_c_clr          00453b04   VDP.obj
 0001:00052b34       vram_scrmap_d_clr          00453b34   VDP.obj
 0001:00052b64       vram_scrmap_r_clr          00453b64   VDP.obj
 0001:00052b94       vram_cgall_clr             00453b94   VDP.obj
 0001:00052bc4       vram_cga_clr               00453bc4   VDP.obj
 0001:00052bf4       vram_cgb_clr               00453bf4   VDP.obj
 0001:00052c24       vram_cgc_clr               00453c24   VDP.obj
 0001:00052c54       vram_cgd_clr               00453c54   VDP.obj
 0001:00052c84       init_vdp1sys               00453c84   VDP.obj
 0001:00052c85       init_vdp1sys2              00453c85   VDP.obj
 0001:00052c88       init_vdp2sys               00453c88   VDP.obj
 0001:00052c8c       tv_on                      00453c8c   VDP.obj
 0001:00052c90       tv_off                     00453c90   VDP.obj
 0001:00052c94       tv_off_boot                00453c94   VDP.obj
 0001:00052ca0       cdsec_chk                  00453ca0   VDP.obj
 0001:00052ca4       init_event                 00453ca4   EVENT.obj
 0001:00052cd4       exec_event                 00453cd4   EVENT.obj
 0001:00052d66       get_event_work             00453d66   EVENT.obj
 0001:00052dbb       set_event                  00453dbb   EVENT.obj
 0001:00052eb0       del_event                  00453eb0   EVENT.obj
 0001:00052fd5       set_object                 00453fd5   EVENT.obj
 0001:00052fd8       set_car_c_select           00453fd8   POLY_SET.obj
 0001:00053321       csl_disp_poly_mc           00454321   POLY_SET.obj
 0001:0005344f       csl_disp_poly_ac           0045444f   POLY_SET.obj
 0001:0005356f       csl_disp_poly_ad           0045456f   POLY_SET.obj
 0001:0005368f       csl_disp_poly_md           0045468f   POLY_SET.obj
 0001:000537c0       _load_default_ghost        004547c0 f bup_file.obj
 0001:000538f0       _backup_init               004548f0 f bup_file.obj
 0001:00053a80       _bup_data_init             00454a80 f bup_file.obj
 0001:00053ad0       _backup_setup              00454ad0 f bup_file.obj
 0001:00053be0       _backup_save               00454be0 f bup_file.obj
 0001:00053ca0       _backup_g_save             00454ca0 f bup_file.obj
 0001:00053e30       _BUP_Read                  00454e30 f bup_file.obj
 0001:00053ec0       _BUP_Write                 00454ec0 f bup_file.obj
 0001:00053f30       _BUP_INIT_C                00454f30 f bup_file.obj
 0001:00053fe0       _BUP_T_SAVE_C              00454fe0 f bup_file.obj
 0001:00054090       _BUP_G_SAVE_C              00455090 f bup_file.obj
 0001:00054130       sysid_hard_id              00455130   VECTOR.obj
 0001:00054140       sysid_co_id                00455140   VECTOR.obj
 0001:00054150       sysid_no                   00455150   VECTOR.obj
 0001:0005415a       sysid_ver                  0045515a   VECTOR.obj
 0001:00054160       sysid_rel                  00455160   VECTOR.obj
 0001:00054168       sysid_dev                  00455168   VECTOR.obj
 0001:00054170       sysid_area                 00455170   VECTOR.obj
 0001:0005417a       sysid_backup               0045517a   VECTOR.obj
 0001:00054180       sysid_per                  00455180   VECTOR.obj
 0001:00054190       sysid_name                 00455190   VECTOR.obj
 0001:00054210       sysid_ip_size              00455210   VECTOR.obj
 0001:00054218       sysid_mstktop              00455218   VECTOR.obj
 0001:0005421c       sysid_sstktop              0045521c   VECTOR.obj
 0001:00054220       sysid_1staddr              00455220   VECTOR.obj
 0001:00054224       sysid_1stsize              00455224   VECTOR.obj
 0001:00054230       timecmp_display            00455230   display2.obj
 0001:00054300       timecmp_display_f          00455300   display2.obj
 0001:00054693       ctime_write_sub            00455693   display2.obj
 0001:00054694       ctime_write_subs           00455694   display2.obj
 0001:00054695       ctime_write_subss          00455695   display2.obj
 0001:00054698       ctime_write_sub2           00455698   display2.obj
 0001:0005469c       tcmp_disp_on               0045569c   display2.obj
 0001:000546a6       tcmp_disp_com              004556a6   display2.obj
 0001:0005472c       tcmp_disp_off              0045572c   display2.obj
 0001:0005473c       tcmp_disp_end              0045573c   display2.obj
 0001:00054790       ftcmp_disp_on              00455790   display2.obj
 0001:00054844       ftcmp_disp_endi            00455844   display2.obj
 0001:000548c8       ftcmp_disp_end             004558c8   display2.obj
 0001:00054934       nftcmp_disp_init           00455934   display2.obj
 0001:000549c0       retime_etc_display         004559c0   display2.obj
 0001:00054e88       retime_etc_display2p       00455e88   display2.obj
 0001:00055108       rfrank_display             00456108   display2.obj
 0001:0005518c       rlap_race_rcalc            0045618c   display2.obj
 0001:00055568       rlap_prac_rcalc            00456568   display2.obj
 0001:0005579c       rlap_prac_fcalc            0045679c   display2.obj
 0001:0005593c       rlap_calc                  0045693c   display2.obj
 0001:00055b80       result_display             00456b80   display2.obj
 0001:00055bf4       rpresult_tbl               00456bf4   display2.obj
 0001:000565ac       tresult_tbl                004575ac   display2.obj
 0001:00056a40       _InitialDirectPlay         00457a40 f dpctrl.obj
 0001:00056ca0       _DestroyDirectPlay         00457ca0 f dpctrl.obj
 0001:00056d70       _SWDataSend                00457d70 f dpctrl.obj
 0001:00056e30       _SWDataSendReceive         00457e30 f dpctrl.obj
 0001:00057160       _WaitTimeCalc              00458160 f dpctrl.obj
 0001:000573b0       _CloseProvider@0           004583b0 f dpctrl.obj
 0001:00057410       _SendDirectPlayWaitMessage 00458410 f dpctrl.obj
 0001:00057430       _SendDirectPlay            00458430 f dpctrl.obj
 0001:00057490       _SendDirectPlayMessage     00458490 f dpctrl.obj
 0001:00057640       _ReceiveDirectPlay         00458640 f dpctrl.obj
 0001:00057710       _ReceiveDirectPlayMessage  00458710 f dpctrl.obj
 0001:000577a0       _ManageDirectPlayMessage   004587a0 f dpctrl.obj
 0001:00057ad0       _WaitRival_Master          00458ad0 f dpctrl.obj
 0001:00057b00       _WaitRival_Slave           00458b00 f dpctrl.obj
 0001:00057b30       _DlgProcWaitRival_Master@16 00458b30 f dpctrl.obj
 0001:00057e50       _DlgProcWaitRival_Slave@16 00458e50 f dpctrl.obj
 0001:00058050       _EnumSession@16            00459050 f dpctrl.obj
 0001:000580e0       _EnumSP@20                 004590e0 f dpctrl.obj
 0001:000581e0       _SelectProvider            004591e0 f dpctrl.obj
 0001:000583c0       _DlgProcLinkGame@16        004593c0 f dpctrl.obj
 0001:00058940       _RemoteCreate              00459940 f dpctrl.obj
 0001:000589f0       _LinkEndMessage_sub        004599f0 f dpctrl.obj
 0001:00058a60       _LinkEndMessage            00459a60 f dpctrl.obj
 0001:00058ac0       _LinkStopMessage_sub       00459ac0 f dpctrl.obj
 0001:00058b30       _LinkStopMessage           00459b30 f dpctrl.obj
 0001:00058b90       _DPERR_MBOX                00459b90 f dpctrl.obj
 0001:00058bd0       _DPERR_MBOX_J              00459bd0 f dpctrl.obj
 0001:00059140       _DPERR_MBOX_E              0045a140 f dpctrl.obj
 0001:000596b0       _get_machine_name          0045a6b0 f dpctrl.obj
 0001:00059710       _get_logon_name            0045a710 f dpctrl.obj
 0001:000597a0       _CloseVsGame               0045a7a0 f dpctrl.obj
 0001:000597c0       _InitVsGame                0045a7c0 f dpctrl.obj
 0001:000598c4       name_main                  0045a8c4   NAME_MAIN.obj
 0001:000598c4       __name_main                0045a8c4   NAME_MAIN.obj
 0001:00059b48       name_main2                 0045ab48   NAME_MAIN.obj
 0001:00059b48       __name_main2               0045ab48   NAME_MAIN.obj
 0001:0005a8a6       name_main_loop             0045b8a6   NAME_MAIN.obj
 0001:0005d2f8       rec_scr_act                0045e2f8   REC_SCRACT.obj
 0001:0005d978       _poweron_start             0045e978   CINTF.obj
 0001:0005d995       _title_init_adv            0045e995   CINTF.obj
 0001:0005d9ad       _adv_main                  0045e9ad   CINTF.obj
 0001:0005d9c5       _bpe_expand                0045e9c5   CINTF.obj
 0001:0005d9f8       _game_init                 0045e9f8   CINTF.obj
 0001:0005da10       _game_main                 0045ea10   CINTF.obj
 0001:0005da28       _ginit_vs                  0045ea28   CINTF.obj
 0001:0005da40       _game_main2p               0045ea40   CINTF.obj
 0001:0005da58       _init_game_work_start      0045ea58   CINTF.obj
 0001:0005da70       _set_grpara_int            0045ea70   CINTF.obj
 0001:0005da88       _set_grpara_int2p          0045ea88   CINTF.obj
 0001:0005daa0       _pre_fade_inout            0045eaa0   CINTF.obj
 0001:0005dab8       _fade_inout_work           0045eab8   CINTF.obj
 0001:0005dad0       _backup_freeze             0045ead0   CINTF.obj
 0001:0005dae8       __backup_check             0045eae8   CINTF.obj
 0001:0005db00       __backup_g_check           0045eb00   CINTF.obj
 0001:0005db18       _backup_melt               0045eb18   CINTF.obj
 0001:0005db30       _record_connect            0045eb30   CINTF.obj
 0001:0005db48       _record_connect2           0045eb48   CINTF.obj
 0001:0005db60       _name_main                 0045eb60   CINTF.obj
 0001:0005db78       _name_main2                0045eb78   CINTF.obj
 0001:0005db90       _name_main_loop            0045eb90   CINTF.obj
 0001:0005dba8       _name_exit                 0045eba8   CINTF.obj
 0001:0005dbc0       _name_exit_loop            0045ebc0   CINTF.obj
 0001:0005dbd8       _game_over                 0045ebd8   CINTF.obj
 0001:0005dbf0       _game_over_loop            0045ebf0   CINTF.obj
 0001:0005dc08       _ceremony_init             0045ec08   CINTF.obj
 0001:0005dc20       _ceremony_main             0045ec20   CINTF.obj
 0001:0005dc38       _result_main               0045ec38   CINTF.obj
 0001:0005dc50       _result_main_loop          0045ec50   CINTF.obj
 0001:0005dc68       _result2p_main             0045ec68   CINTF.obj
 0001:0005dc80       _result2p_main_loop        0045ec80   CINTF.obj
 0001:0005dc98       _photo_init                0045ec98   CINTF.obj
 0001:0005dcb0       _photo_main                0045ecb0   CINTF.obj
 0001:0005dcc8       _ending_init               0045ecc8   CINTF.obj
 0001:0005dce0       _ending_main               0045ece0   CINTF.obj
 0001:0005dcf8       _x_result_init             0045ecf8   CINTF.obj
 0001:0005dd10       _x_result_main             0045ed10   CINTF.obj
 0001:0005dd28       _mkpoly_init               0045ed28   CINTF.obj
 0001:0005dd40       _REPLAY_INIT2              0045ed40   CINTF.obj
 0001:0005dd58       _title_init                0045ed58   CINTF.obj
 0001:0005dd70       _g_select_init             0045ed70   CINTF.obj
 0001:0005dd88       _g_select_main             0045ed88   CINTF.obj
 0001:0005dda0       _c_select_init             0045eda0   CINTF.obj
 0001:0005ddb8       _c_select_main             0045edb8   CINTF.obj
 0001:0005ddd0       _crs_select_init           0045edd0   CINTF.obj
 0001:0005dde8       _crs_select_main           0045ede8   CINTF.obj
 0001:0005de00       _slt_mode_init             0045ee00   CINTF.obj
 0001:0005de18       _slt_mode_main             0045ee18   CINTF.obj
 0001:0005de30       _color_change_init         0045ee30   CINTF.obj
 0001:0005de48       _color_change_main         0045ee48   CINTF.obj
 0001:0005de60       _disp_car_main_battle2p    0045ee60   CINTF.obj
 0001:0005de78       _disp_course_main_battle2p 0045ee78   CINTF.obj
 0001:0005de90       _disp_car_main_timeattack  0045ee90   CINTF.obj
 0001:0005dea8       _disp_course_main_timeattack 0045eea8   CINTF.obj
 0001:0005dec0       _disp_car_main_setting1    0045eec0   CINTF.obj
 0001:0005ded8       _disp_car_main_setting2    0045eed8   CINTF.obj
 0001:0005def0       _disp_obj_main_setting     0045eef0   CINTF.obj
 0001:0005df08       _put_modeltype             0045ef08   CINTF.obj
 0001:0005df20       _put_modeltype2            0045ef20   CINTF.obj
 0001:0005df38       _cs_set_crs                0045ef38   CINTF.obj
 0001:0005df50       _bt_set_crs                0045ef50   CINTF.obj
 0001:0005df68       _md_set_crs                0045ef68   CINTF.obj
 0001:0005df80       _key_repeat_init           0045ef80   CINTF.obj
 0001:0005df98       _check_cursor_posi         0045ef98   CINTF.obj
 0001:0005dfb0       _check_cursor_posi2        0045efb0   CINTF.obj
 0001:0005dfc8       _bt_disp_spr               0045efc8   CINTF.obj
 0001:0005dfe0       _pad_check                 0045efe0   CINTF.obj
 0001:0005dff8       _check_stratos_flg         0045eff8   CINTF.obj
 0001:0005e010       _check_tune_flg            0045f010   CINTF.obj
 0001:0005e028       _check_lake_flg            0045f028   CINTF.obj
 0001:0005e040       _save_set_data             0045f040   CINTF.obj
 0001:0005e058       _set_car                   0045f058   CINTF.obj
 0001:0005e070       backup_init                0045f070   CINTF.obj
 0001:0005e075       bup_data_init              0045f075   CINTF.obj
 0001:0005e07a       backup_setup               0045f07a   CINTF.obj
 0001:0005e07f       backup_save                0045f07f   CINTF.obj
 0001:0005e084       backup_g_save              0045f084   CINTF.obj
 0001:0005e089       _shreg_init                0045f089   CINTF.obj
 0001:0005f120       _GetCDTrackInf             00460120 f CDSND.obj
 0001:0005f290       _CDsndInit                 00460290 f CDSND.obj
 0001:0005f420       _CDsndExit                 00460420 f CDSND.obj
 0001:0005f4d0       _CDsndGetMode              004604d0 f CDSND.obj
 0001:0005f520       _CDsndSetPlayTrack         00460520 f CDSND.obj
 0001:0005f590       _CDsndPlay                 00460590 f CDSND.obj
 0001:0005f720       _CDsndRePlay               00460720 f CDSND.obj
 0001:0005f750       _CDsndResume               00460750 f CDSND.obj
 0001:0005f7a0       _CDsndPause                004607a0 f CDSND.obj
 0001:0005f830       _CDsndStop                 00460830 f CDSND.obj
 0001:0005f8d0       _CDsndNotify               004608d0 f CDSND.obj
 0001:0005fad0       _snd_CDPlay                00460ad0 f CDSND.obj
 0001:0005fef0       _snd_CDPause               00460ef0 f CDSND.obj
 0001:0005ff70       _snd_CDResume              00460f70 f CDSND.obj
 0001:0005ffc0       _snd_CDStop                00460fc0 f CDSND.obj
 0001:00060050       title2_init                00461050   ADV.obj
 0001:00060078       title_init_adv             00461078   ADV.obj
 0001:00060078       adv_init                   00461078   ADV.obj
 0001:000600f8       adv_start                  004610f8   ADV.obj
 0001:0006033f       init_adv_stage             0046133f   ADV.obj
 0001:0006053c       init_adv_work_start        0046153c   ADV.obj
 0001:000606b8       init_adv_work              004616b8   ADV.obj
 0001:00060a18       init_adv_vram              00461a18   ADV.obj
 0001:00060afc       adv_plmt                   00461afc   ADV.obj
 0001:00060b64       adv_plmt2p                 00461b64   ADV.obj
 0001:00060bcc       adv_plmove                 00461bcc   ADV.obj
 0001:00060c28       adv_pinit                  00461c28   ADV.obj
 0001:00060d44       adv_pwait                  00461d44   ADV.obj
 0001:00060e34       adv_pgo                    00461e34   ADV.obj
 0001:00060e70       adv_pmove                  00461e70   ADV.obj
 0001:00060e80       copy_disp_para             00461e80   ADV.obj
 0001:00061044       adv_main                   00462044   ADV.obj
 0001:00061238       adv_main_sub               00462238   ADV.obj
 0001:0006146c       a_pause_init               0046246c   ADV.obj
 0001:000614d0       a_pause                    004624d0   ADV.obj
 0001:00061604       a_restart_init             00462604   ADV.obj
 0001:000616d0       adv_ctrl                   004626d0   ADV.obj
 0001:000618e4       replay2_ca                 004628e4   ADV.obj
 0001:00061a18       camera_vr1                 00462a18   ADV.obj
 0001:00061f8c       calc_camera_pmap2          00462f8c   ADV.obj
 0001:000620c1       memcpy_l                   004630c1   ADV.obj
 0001:000620c1       memcpy                     004630c1   ADV.obj
 0001:000621c4       x_result_init              004631c4   x_result.obj
 0001:0006225b       x_result_main              0046325b   x_result.obj
 0001:00065ea0       record_RTxxx               00466ea0   REC_RTXXX.obj
 0001:00066190       _ScrlObj_Game_Off          00467190 f Scrlobj.obj
 0001:00066210       _ScrlObj_Result_Off        00467210 f Scrlobj.obj
 0001:00066240       _ScrlObj_Adv_Off           00467240 f Scrlobj.obj
 0001:00066250       _ScrlObj_Name_Off          00467250 f Scrlobj.obj
 0001:00066260       _ScrlObj_Over_Off          00467260 f Scrlobj.obj
 0001:00066270       _ScrlObj_Over_On           00467270 f Scrlobj.obj
 0001:00066280       _ScrlObj_Staff_Off         00467280 f Scrlobj.obj
 0001:00066290       _ScrlObj_Staff2_Off        00467290 f Scrlobj.obj
 0001:000662a0       _ScrlObj_Off               004672a0 f Scrlobj.obj
 0001:00066360       _GetCenter                 00467360 f Scrlobj.obj
 0001:000663b0       _ChangeSaturnPosi          004673b0 f Scrlobj.obj
 0001:00066420       _ChangeVGAPosi             00467420 f Scrlobj.obj
 0001:00066470       _fn16bitPacth              00467470 f Scrlobj.obj
 0001:00066580       _NaviBMP_Flip              00467580 f Scrlobj.obj
 0001:00066680       _ScrlObj_Init              00467680 f Scrlobj.obj
 0001:00066b50       _ScrlObj_Free              00467b50 f Scrlobj.obj
 0001:00066ba0       _BoxWrite                  00467ba0 f Scrlobj.obj
 0001:00066c60       _BoxWriteYOverCheck        00467c60 f Scrlobj.obj
 0001:00066d80       _BoxWriteXOverCheck        00467d80 f Scrlobj.obj
 0001:00066eb0       _put_gyakusou              00467eb0 f Scrlobj.obj
 0001:00067100       _put_tacho                 00468100 f Scrlobj.obj
 0001:00067230       _put_navi                  00468230 f Scrlobj.obj
 0001:000672d0       _put_shift                 004682d0 f Scrlobj.obj
 0001:000674b0       _put_font                  004684b0 f Scrlobj.obj
 0001:00067520       _put_speed2                00468520 f Scrlobj.obj
 0001:00067680       _put_decimal2              00468680 f Scrlobj.obj
 0001:00067740       _put_decimal2XOverCheck    00468740 f Scrlobj.obj
 0001:000677f0       _put_decimal2YOverCheck    004687f0 f Scrlobj.obj
 0001:000678c0       _put_speed                 004688c0 f Scrlobj.obj
 0001:00067a30       _put_rank                  00468a30 f Scrlobj.obj
 0001:00067c90       _put_extend_time           00468c90 f Scrlobj.obj
 0001:00067ee0       _put_laptime               00468ee0 f Scrlobj.obj
 0001:00068640       _put_laptime_freerun       00469640 f Scrlobj.obj
 0001:000688c0       _put_timecmp               004698c0 f Scrlobj.obj
 0001:00068a10       _put_besttime              00469a10 f Scrlobj.obj
 0001:00068b00       _put_result_pactice_lap    00469b00 f Scrlobj.obj
 0001:00068c90       _put_result_rp             00469c90 f Scrlobj.obj
 0001:00069a30       _put_result_t              0046aa30 f Scrlobj.obj
 0001:00069ca0       _put_carmark               0046aca0 f Scrlobj.obj
 0001:00069d60       _put_free_etc              0046ad60 f Scrlobj.obj
 0001:00069df0       _put_attack_etc            0046adf0 f Scrlobj.obj
 0001:00069f90       _Put_ScrlObj_race          0046af90 f Scrlobj.obj
 0001:0006a240       _Put_ScrlObj_freerun       0046b240 f Scrlobj.obj
 0001:0006a450       _Put_ScrlObj_attack        0046b450 f Scrlobj.obj
 0001:0006a5e0       _put_vs_bestlap            0046b5e0 f Scrlobj.obj
 0001:0006a750       _put_rank_vs_laps_sub      0046b750 f Scrlobj.obj
 0001:0006a880       _put_rank_vs_laps          0046b880 f Scrlobj.obj
 0001:0006ab80       _put_rank_vs_lag           0046bb80 f Scrlobj.obj
 0001:0006af90       _put_etc_laps_net          0046bf90 f Scrlobj.obj
 0001:0006b170       _put_etc_lag_net           0046c170 f Scrlobj.obj
 0001:0006b390       _put_flag1st_sub           0046c390 f Scrlobj.obj
 0001:0006b420       _put_flag1st               0046c420 f Scrlobj.obj
 0001:0006b510       _put_flag1st_net           0046c510 f Scrlobj.obj
 0001:0006b590       _put_timecmp_vs_lag        0046c590 f Scrlobj.obj
 0001:0006b680       _put_timecmp_vs_laps       0046c680 f Scrlobj.obj
 0001:0006b870       _put_timecmp_lag_net       0046c870 f Scrlobj.obj
 0001:0006b9f0       _put_timecmp_laps_net      0046c9f0 f Scrlobj.obj
 0001:0006bba0       _Put_ScrlObj_vs            0046cba0 f Scrlobj.obj
 0001:0006be70       _Put_ScrlObj_net           0046ce70 f Scrlobj.obj
 0001:0006c000       _put_adv_press_start       0046d000 f Scrlobj.obj
 0001:0006c060       _put_adv_toyota            0046d060 f Scrlobj.obj
 0001:0006c2c0       _put_adv_ranking_sub       0046d2c0 f Scrlobj.obj
 0001:0006c660       _put_adv_ranking           0046d660 f Scrlobj.obj
 0001:0006c9a0       _Put_ScrlObj_adv           0046d9a0 f Scrlobj.obj
 0001:0006ca30       _put_result_yn             0046da30 f Scrlobj.obj
 0001:0006ccb0       _put_DebugInfo_sub         0046dcb0 f Scrlobj.obj
 0001:0006ccf0       _put_DebugInfo             0046dcf0 f Scrlobj.obj
 0001:0006cfc0       _put_result_ta_title       0046dfc0 f Scrlobj.obj
 0001:0006d010       _LapCountupTimeInit        0046e010 f Scrlobj.obj
 0001:0006d030       _MakeCountupTime           0046e030 f Scrlobj.obj
 0001:0006d090       _put_ta_result             0046e090 f Scrlobj.obj
 0001:0006d6e0       _put_result_ranking_sub    0046e6e0 f Scrlobj.obj
 0001:0006dbc0       _put_ranking               0046ebc0 f Scrlobj.obj
 0001:0006dcb0       _put_ranking_result        0046ecb0 f Scrlobj.obj
 0001:0006ddf0       _put_vs_net_result         0046edf0 f Scrlobj.obj
 0001:0006e290       _put_continue              0046f290 f Scrlobj.obj
 0001:0006e400       _put_vs_result             0046f400 f Scrlobj.obj
 0001:0006e510       _put_net_result            0046f510 f Scrlobj.obj
 0001:0006e610       _put_staff                 0046f610 f Scrlobj.obj
 0001:0006e750       _put_staff2_sub            0046f750 f Scrlobj.obj
 0001:0006e7c0       _Put_ScrlObj_name          0046f7c0 f Scrlobj.obj
 0001:0006e950       _Put_ScrlObj               0046f950 f Scrlobj.obj
 0001:0006eff0       mkpoly_init                0046fff0   MKPOLY.obj
 0001:0006f04a       s_mkpoly_init              0047004a   MKPOLY.obj
 0001:0006f060       m_mkpoly_init              00470060   MKPOLY.obj
 0001:0006f074       mkpoly_init_sub            00470074   MKPOLY.obj
 0001:0006f2a4       mkpoly_init_2p             004702a4   MKPOLY.obj
 0001:0006f38c       mkpoly_init_net            0047038c   MKPOLY.obj
 0001:0006f43a       mkpoly_frame_init          0047043a   MKPOLY.obj
 0001:0006f451       m_mkpoly_frame_init        00470451   MKPOLY.obj
 0001:0006f4ca       s_mkpoly_frame_init        004704ca   MKPOLY.obj
 0001:0006f543       get_mkpolywk               00470543   MKPOLY.obj
 0001:0006f595       set_vertice_type           00470595   MKPOLY.obj
 0001:0006f618       perspective                00470618   MKPOLY.obj
 0001:0006f66f       set_pers_scale             0047066f   MKPOLY.obj
 0001:0006f68d       set_clip3d_f               0047068d   MKPOLY.obj
 0001:0006f6a4       set_scaledivz              004706a4   MKPOLY.obj
 0001:0006f726       polyline_on                00470726   MKPOLY.obj
 0001:0006f743       polyline_off               00470743   MKPOLY.obj
 0001:0006f760       set_poly_offset            00470760   MKPOLY.obj
 0001:0006f7cf       DRAW_POLYGON               004707cf   MKPOLY.obj
 0001:0006f9ac       draw_course_2p             004709ac   MKPOLY.obj
 0001:0006fc96       draw_course_net            00470c96   MKPOLY.obj
 0001:0006ff7c       draw_course_polygon        00470f7c   MKPOLY.obj
 0001:0006ff7c       draw_course                00470f7c   MKPOLY.obj
 0001:000703b4       count_course_polygon       004713b4   MKPOLY.obj
 0001:00070581       draw_polygon               00471581   MKPOLY.obj
 0001:00070819       draw_polygon2              00471819   MKPOLY.obj
 0001:00070aad       draw_offset_polygon        00471aad   MKPOLY.obj
 0001:00070d3f       draw_clip_polygon          00471d3f   MKPOLY.obj
 0001:00071028       draw_polygon_init          00472028   MKPOLY.obj
 0001:00071170       set_object_matrix          00472170   MKPOLY.obj
 0001:00071274       set_course_matrix          00472274   MKPOLY.obj
 0001:000713a2       entry_polygon4             004723a2   MKPOLY.obj
 0001:00071590       entry_polygon3             00472590   MKPOLY.obj
 0001:000716dc       get_vertbuf_addr4          004726dc   MKPOLY.obj
 0001:0007183a       set_surface_normal         0047283a   MKPOLY.obj
 0001:000718cd       set_clipflg4               004728cd   MKPOLY.obj
 0001:00071a17       set_clipflg3               00472a17   MKPOLY.obj
 0001:00071b0b       zclip4                     00472b0b   MKPOLY.obj
 0001:00071b9e       zclip3                     00472b9e   MKPOLY.obj
 0001:00071c12       set_polydata4              00472c12   MKPOLY.obj
 0001:00071d6f       set_polydata3              00472d6f   MKPOLY.obj
 0001:00071ecc       set_vertice_data           00472ecc   MKPOLY.obj
 0001:000721b5       chk_revpoly                004731b5   MKPOLY.obj
 0001:0007235b       rewrt_chk_revpoly          0047335b   MKPOLY.obj
 0001:0007235c       chkrev_norm_prg            0047335c   MKPOLY.obj
 0001:00072385       chkrev_mirror_prg          00473385   MKPOLY.obj
 0001:000723b0       get_sortpnt4               004733b0   MKPOLY.obj
 0001:00072434       spnt4_middle               00473434   MKPOLY.obj
 0001:00072460       spnt4_near                 00473460   MKPOLY.obj
 0001:000724d3       get_sortpnt_ret            004734d3   MKPOLY.obj
 0001:000724d4       spnt4_far                  004734d4   MKPOLY.obj
 0001:00072548       spnt4_road                 00473548   MKPOLY.obj
 0001:000725d7       spnt4_iwayama              004735d7   MKPOLY.obj
 0001:00072619       get_sortpnt3               00473619   MKPOLY.obj
 0001:0007268f       spnt3_middle               0047368f   MKPOLY.obj
 0001:00072721       spnt3_far                  00473721   MKPOLY.obj
 0001:00072772       spnt3_road                 00473772   MKPOLY.obj
 0001:000727db       spnt3_iwayama              004737db   MKPOLY.obj
 0001:00072845       entry_zbuf                 00473845   MKPOLY.obj
 0001:00072983       entry_zbuf2                00473983   MKPOLY.obj
 0001:00072ab1       set_poly_command           00473ab1   MKPOLY.obj
 0001:00072bdd       set_normal_polygon         00473bdd   MKPOLY.obj
 0001:00072c38       set_mesh_polygon           00473c38   MKPOLY.obj
 0001:00072c93       set_flatgour_polygon       00473c93   MKPOLY.obj
 0001:00072d31       set_texture_polygon        00473d31   MKPOLY.obj
 0001:00072e20       set_textshad_polygon       00473e20   MKPOLY.obj
 0001:00072ec7       set_textgour_polygon       00473ec7   MKPOLY.obj
 0001:00072ee1       chk_sortpnt                00473ee1   MKPOLY.obj
 0001:00072f68       set_gourshad_tbl           00473f68   MKPOLY.obj
 0001:00073234       flat_shading               00474234   MKPOLY.obj
 0001:00074568       get_crosszh                00475568   MKPOLY.obj
 0001:0007487a       calc_vertices              0047587a   MKPOLY.obj
 0001:00074cec       calc_offset_vertices       00475cec   MKPOLY.obj
 0001:000751ac       calc_clip_vertices         004761ac   MKPOLY.obj
 0001:00075836       calc_vertbright            00476836   MKPOLY.obj
 0001:0007595c       draw_color_polygon         0047695c   MKPOLY.obj
 0001:00075c5a       entry_color_polygon4       00476c5a   MKPOLY.obj
 0001:00075dd0       entry_color_polygon3       00476dd0   MKPOLY.obj
 0001:00075f30       draw_people_polygon        00476f30   MKPOLY.obj
 0001:0007621c       calc_people_vertices       0047721c   MKPOLY.obj
 0001:00076502       draw_splash_polygon        00477502   MKPOLY.obj
 0001:000767ec       calc_splash_vertices       004777ec   MKPOLY.obj
 0001:00076ab4       dispcar_init               00477ab4   DISPCAR.obj
 0001:00076b38       dispCar                    00477b38   DISPCAR.obj
 0001:00076bd6       dispGhost                  00477bd6   DISPCAR.obj
 0001:000779f9       dispSelectCar2             004789f9   DISPCAR.obj
 0001:00077a20       dispSelectCar              00478a20   DISPCAR.obj
 0001:0007809a       dispTachoMeter_2p          0047909a   DISPCAR.obj
 0001:000780d2       dispTachoMeter_net         004790d2   DISPCAR.obj
 0001:000780d2       dispTachoMeter             004790d2   DISPCAR.obj
 0001:000783b8       dispCountDown              004793b8   DISPCAR.obj
 0001:00078ccc       Title_Tbl                  00479ccc   OPT_DISP.obj
 0001:00078cfc       Sub_Tbl                    00479cfc   OPT_DISP.obj
 0001:00078e18       Snd_Tbl                    00479e18   OPT_DISP.obj
 0001:00079004       Tbl_1P                     0047a004   OPT_DISP.obj
 0001:0007905c       PAD_Tbl                    0047a05c   OPT_DISP.obj
 0001:0007906c       HANDLE_Tbl                 0047a06c   OPT_DISP.obj
 0001:0007907c       option_title_disp          0047a07c   OPT_DISP.obj
 0001:000791b4       option_subtitle_disp       0047a1b4   OPT_DISP.obj
 0001:00079428       option_sndtitle_disp       0047a428   OPT_DISP.obj
 0001:00079b45       option_keyconfig_disp2     0047ab45   OPT_DISP.obj
 0001:00079dc7       option_keyconfig_disp      0047adc7   OPT_DISP.obj
 0001:00079fd8       string_disp                0047afd8   OPT_DISP.obj
 0001:0007a384       backup_freeze              0047b384   BUP_FREEZE.obj
 0001:0007a718       guide_yosemite             0047b718   ndyosemi.obj
 0001:0007ba08       dma_load                   0047ca08   ETCSUB.obj
 0001:0007ba84       dmacopy                    0047ca84   ETCSUB.obj
 0001:0007baa0       copy_memory                0047caa0   ETCSUB.obj
 0001:0007baec       copy_memory2               0047caec   ETCSUB.obj
 0001:0007bb38       memcopy                    0047cb38   ETCSUB.obj
 0001:0007bb38       copy_memory4               0047cb38   ETCSUB.obj
 0001:0007bb84       fill_memory                0047cb84   ETCSUB.obj
 0001:0007bbbc       fill_memory2               0047cbbc   ETCSUB.obj
 0001:0007bbf4       fill_memory4               0047cbf4   ETCSUB.obj
 0001:0007bc2a       init_workarea              0047cc2a   ETCSUB.obj
 0001:0007bc2c       get_random                 0047cc2c   ETCSUB.obj
 0001:0007bc90       hex2bcd                    0047cc90   ETCSUB.obj
 0001:0007bc90       hex2dec                    0047cc90   ETCSUB.obj
 0001:0007bd6c       bcd2hex                    0047cd6c   ETCSUB.obj
 0001:0007bddd       count_polygon              0047cddd   ETCSUB.obj
 0001:0007bf2f       chk_pushstart              0047cf2f   ETCSUB.obj
 0001:0007bfb1       chg_mainvect               0047cfb1   ETCSUB.obj
 0001:0007bfe0       chk_cpu                    0047cfe0   ETCSUB.obj
 0001:0007c015       move_xyz_position          0047d015   ETCSUB.obj
 0001:0007c1a0       rotate_xyz_angle           0047d1a0   ETCSUB.obj
 0001:0007c2e8       check_screen               0047d2e8   ETCSUB.obj
 0001:0007c561       check_screen2              0047d561   ETCSUB.obj
 0001:0007c7ed       boxwrt                     0047d7ed   ETCSUB.obj
 0001:0007c8bc       boxwrt2                    0047d8bc   ETCSUB.obj
 0001:0007c989       boxfill                    0047d989   ETCSUB.obj
 0001:0007ca2f       boxfill2                   0047da2f   ETCSUB.obj
 0001:0007cad4       set_scrl_cgs               0047dad4   ETCSUB.obj
 0001:0007cb62       set_scrl_maps              0047db62   ETCSUB.obj
 0001:0007cbf8       disp_msg                   0047dbf8   ETCSUB.obj
 0001:0007cc70       init_fade                  0047dc70   ETCSUB.obj
 0001:0007cd44       init_whitefade             0047dd44   ETCSUB.obj
 0001:0007cdb6       fade                       0047ddb6   ETCSUB.obj
 0001:0007cf07       init_perform               0047df07   ETCSUB.obj
 0001:0007cf08       get_perform                0047df08   ETCSUB.obj
 0001:0007cf09       diso_hex_byte              0047df09   ETCSUB.obj
 0001:0007cf23       disp_hex_word              0047df23   ETCSUB.obj
 0001:0007cf36       disp_hex_long              0047df36   ETCSUB.obj
 0001:0007cf40       disp_hex                   0047df40   ETCSUB.obj
 0001:0007cfdc       DRAW_COLOR_POLYGON         0047dfdc   ETCSUB.obj
 0001:0007d046       colorfade                  0047e046   ETCSUB.obj
 0001:0007d0cc       colorfadesub               0047e0cc   ETCSUB.obj
 0001:0007d264       submode_act                0047e264   ETCSUB.obj
 0001:0007d2a9       dec_modetimer              0047e2a9   ETCSUB.obj
 0001:0007d2f0       _staffroll_init            0047e2f0 f staffroll.obj
 0001:0007d360       _staffroll_main            0047e360 f staffroll.obj
 0001:0007d410       _put_staff2                0047e410 f staffroll.obj
 0001:0007d470       _staffroll_main_exit       0047e470 f staffroll.obj
 0001:0007d4a0       _option_scroll_act_1       0047e4a0 f option.obj
 0001:0007d510       _option_scroll_act_2       0047e510 f option.obj
 0001:0007d630       _option_init               0047e630 f option.obj
 0001:0007d780       _opt_move_sprite           0047e780 f option.obj
 0001:0007d810       _option_sprite_set         0047e810 f option.obj
 0001:0007da80       _option_exit               0047ea80 f option.obj
 0001:0007daa0       _option_main               0047eaa0 f option.obj
 0001:0007dcc0       _option_scroll_act_3       0047ecc0 f option.obj
 0001:0007e8d0       _sound_sprite_set          0047f8d0 f option.obj
 0001:0007eaf0       _option_sound              0047faf0 f option.obj
 0001:0007f880       _option_line_scroll        00480880 f option.obj
 0001:0007fd70       _option_scroll_init        00480d70 f option.obj
 0001:0007fde0       _option_scroll_set         00480de0 f option.obj
 0001:0007ff10       _sound_up                  00480f10 f option.obj
 0001:0007ff60       _sound_down                00480f60 f option.obj
 0001:0007ffb0       _option_scroll_change      00480fb0 f option.obj
 0001:00080200       _sound_in_set_sprite       00481200 f option.obj
 0001:00080280       _sound_out_set_sprite      00481280 f option.obj
 0001:000802f0       advExec                    004812f0   ADVCTRL.obj
 0001:00080db9       adv_break                  00481db9   ADVCTRL.obj
 0001:00080e41       zoomCam                    00481e41   ADVCTRL.obj
 0001:00081023       advctrlinit                00482023   ADVCTRL.obj
 0001:0008119f       advFrmCtrl                 0048219f   ADVCTRL.obj
 0001:000816a4       set_advdata                004826a4   ADVCTRL.obj
 0001:0008173c       mapset_l                   0048273c   ADVCTRL.obj
 0001:00081804       a_title_init               00482804   ADVCTRL.obj
 0001:00081962       a_title_wait               00482962   ADVCTRL.obj
 0001:00081c6e       a_startwait2               00482c6e   ADVCTRL.obj
 0001:00081d05       a_startwait                00482d05   ADVCTRL.obj
 0001:00081df4       a_title_fout               00482df4   ADVCTRL.obj
 0001:00081e49       a_segalogo_init            00482e49   ADVCTRL.obj
 0001:00081f49       a_segalogo_wait            00482f49   ADVCTRL.obj
 0001:00082024       a_segalogo_fout            00483024   ADVCTRL.obj
 0001:00082094       a_sportslogo_init          00483094   ADVCTRL.obj
 0001:000821ae       a_sportslogo_wait          004831ae   ADVCTRL.obj
 0001:00082349       a_sportslogo_fout          00483349   ADVCTRL.obj
 0001:000824bc       name_smoji_act             004834bc   NAME_SELMOJI.obj
 0001:00083464       name_check                 00484464   NAME_SELMOJI.obj
 0001:00083610       _PolyMesh8                 00484610 f Fpoly8.obj
 0001:000852b0       ??0LBitmapFile@@QAE@XZ     004862b0 f LBitmapF.obj
 0001:000852c0       ??0LBitmapFile@@QAE@PBD@Z  004862c0 f LBitmapF.obj
 0001:000852e0       ??1LBitmapFile@@QAE@XZ     004862e0 f LBitmapF.obj
 0001:00085310       ?Load@LBitmapFile@@QAEHPBD@Z 00486310 f LBitmapF.obj
 0001:000854e0       ?Save@LBitmapFile@@QAEHPBD@Z 004864e0 f LBitmapF.obj
 0001:000856c0       ?SetupPalette@LBitmapFile@@QAEHK@Z 004866c0 f LBitmapF.obj
 0001:000858b0       ?SetPalette@LBitmapFile@@QAEHPAGH@Z 004868b0 f LBitmapF.obj
 0001:00085980       ?SetupHeader@LBitmapFile@@QAEHJJK@Z 00486980 f LBitmapF.obj
 0001:000859f0       ?Create@LBitmapFile@@QAEHJJK@Z 004869f0 f LBitmapF.obj
 0001:00085a50       ?StrechDIBtoDC@LBitmapFile@@QAEXPAUHDC__@@JJJJ@Z 00486a50 f LBitmapF.obj
 0001:00085b80       ?ReverseUD@LBitmapFile@@QAEXXZ 00486b80 f LBitmapF.obj
 0001:00085c70       _GetBGNo                   00486c70 f Bgctrl.obj
 0001:00085dc0       _BMPtoBETA                 00486dc0 f Bgctrl.obj
 0001:000862a0       _LoadBMPPalette_sub        004872a0 f Bgctrl.obj
 0001:000864d0       _LoadBMPPalette            004874d0 f Bgctrl.obj
 0001:00086550       _GamePaletteLoad           00487550 f Bgctrl.obj
 0001:00086580       _GameBG_Init_ADV           00487580 f Bgctrl.obj
 0001:000865a0       _GameBG_Init               004875a0 f Bgctrl.obj
 0001:00086810       _GameBG_Free               00487810 f Bgctrl.obj
 0001:00086870       _PutBG                     00487870 f Bgctrl.obj
 0001:00086d60       _start_init_watanabe       00487d60 f Bgctrl.obj
 0001:00086da0       _start_main_watanabe       00487da0 f Bgctrl.obj
 0001:00086e30       _game_over2                00487e30 f Bgctrl.obj
 0001:00086f2c       frmwrt                     00487f2c   VARIETY.obj
 0001:00087128       frmwrt2                    00488128   VARIETY.obj
 0001:00087321       frmdel                     00488321   VARIETY.obj
 0001:000874d9       frmdel2                    004884d9   VARIETY.obj
 0001:0008768f       cd_cg_set                  0048868f   VARIETY.obj
 0001:00087729       cd_map_set                 00488729   VARIETY.obj
 0001:000877c3       cd_map_set_s               004887c3   VARIETY.obj
 0001:00087832       cd_map_set2                00488832   VARIETY.obj
 0001:000878cc       cd_color_set               004888cc   VARIETY.obj
 0001:00087966       cd_frm_set                 00488966   VARIETY.obj
 0001:000879d5       cd_frm_set2                004889d5   VARIETY.obj
 0001:00087a50       _MabikiInit                00488a50 f mabiki.obj
 0001:00087a60       _Mabiki                    00488a60 f mabiki.obj
 0001:00087cd0       InitSplash                 00488cd0   SPLASH.obj
 0001:00087e03       set_splenable              00488e03   SPLASH.obj
 0001:00087e34       SetSplash                  00488e34   SPLASH.obj
 0001:00088d38       ExecSplash                 00489d38   SPLASH.obj
 0001:00088f30       sl_ExecSplash              00489f30   SPLASH.obj
 0001:00088f60       dispSplash                 00489f60   SPLASH.obj
 0001:00089036       splash_act                 0048a036   SPLASH.obj
 0001:00089065       water_act                  0048a065   SPLASH.obj
 0001:0008916b       sand_act                   0048a16b   SPLASH.obj
 0001:00089230       title_init_toya            0048a230   TITLEtoya.obj
 0001:00089298       normal_cainit              0048a298   CAMERA.obj
 0001:00089450       vs_cainit                  0048a450   CAMERA.obj
 0001:000895e0       normal_ca                  0048a5e0   CAMERA.obj
 0001:00089700       goal_eye                   0048a700   CAMERA.obj
 0001:00089718       start_eye                  0048a718   CAMERA.obj
 0001:000898c0       game_eye                   0048a8c0   CAMERA.obj
 0001:00089974       vs1p_ca                    0048a974   CAMERA.obj
 0001:00089c48       replay_ca                  0048ac48   CAMERA.obj
 0001:00089d10       replay_cactl               0048ad10   CAMERA.obj
 0001:0008a180       calc_camera_pmap           0048b180   CAMERA.obj
 0001:0008a264       cmove_vr1                  0048b264   CAMERA.obj
 0001:0008a5d0       cmove_vr3                  0048b5d0   CAMERA.obj
 0001:0008a890       cmove_goal                 0048b890   CAMERA.obj
 0001:0008ab4c       init_cmove_start           0048bb4c   CAMERA.obj
 0001:0008ad0c       cmove_start                0048bd0c   CAMERA.obj
 0001:0008af00       calc_vr2ang                0048bf00   CAMERA.obj
 0001:0008b058       camera_posi_game           0048c058   CAMERA.obj
 0001:0008b2bc       camera_matrix_car          0048c2bc   CAMERA.obj
 0001:0008b528       camera_matrix_goal         0048c528   CAMERA.obj
 0001:0008b640       camera_matrix_start        0048c640   CAMERA.obj
 0001:0008b790       _Texture16_Seethrough      0048c790 f Ftex5.obj
 0001:0008c2b0       start_init_watanabe        0048d2b0   STARTwatanabe.obj
 0001:0008cb54       timeact2p_init             0048db54   RES2_TIMEACT.obj
 0001:0008cd7c       timeact2p_act              0048dd7c   RES2_TIMEACT.obj
 0001:0008d02c       color_act2                 0048e02c   REC_CORACT.obj
 0001:0008d202       color_act                  0048e202   REC_CORACT.obj
 0001:0008d30b       Color_Tbl                  0048e30b   REC_CORACT.obj
 0001:0008d324       record_menu_init           0048e324   REC_MENU.obj
 0001:0008d6d0       _Texture8_Seethrough       0048e6d0 f ftex5_8.obj
 0001:0008e0e0       rec_cmark_act              0048f0e0   REC_CMARKACT.obj
 0001:0008e5c8       md_set_crs                 0048f5c8   CS_POLY_SET.obj
 0001:0008e687       cs_set_crs                 0048f687   CS_POLY_SET.obj
 0001:0008e746       bt_set_crs                 0048f746   CS_POLY_SET.obj
 0001:0008e805       disp_course                0048f805   CS_POLY_SET.obj
 0001:0008e925       disp_obj_cs                0048f925   CS_POLY_SET.obj
 0001:0008e9f0       set_light_obj              0048f9f0   CS_POLY_SET.obj
 0001:0008ea36       calc_obj_posi              0048fa36   CS_POLY_SET.obj
 0001:0008eb6b       disp_spr_tm                0048fb6b   CS_POLY_SET.obj
 0001:0008ec70       disp_spr                   0048fc70   CS_POLY_SET.obj
 0001:0008eeac       bt_disp_spr                0048feac   CS_POLY_SET.obj
 0001:0008f364       bt_disp_spr2               00490364   CS_POLY_SET.obj
 0001:0008f5a8       rec_moji_act               004905a8   REC_MOJIACT.obj
 0001:0008fc34       EvCheckPoint               00490c34   PUBLIC.obj
 0001:0008fc7a       CheckPointMain             00490c7a   PUBLIC.obj
 0001:000900b0       get_top_pl_work            004910b0   PUBLIC.obj
 0001:00090278       EvPole                     00491278   PUBLIC.obj
 0001:000902d1       PoleMain                   004912d1   PUBLIC.obj
 0001:000903dc       EvFlag                     004913dc   PUBLIC.obj
 0001:000904eb       FlagMain                   004914eb   PUBLIC.obj
 0001:0009069d       EvStart                    0049169d   PUBLIC.obj
 0001:00090787       StartMain                  00491787   PUBLIC.obj
 0001:00090c53       EvPilon                    00491c53   PUBLIC.obj
 0001:00090cdd       PilonMain                  00491cdd   PUBLIC.obj
 0001:00090e88       EvPeopleA                  00491e88   PUBLIC.obj
 0001:00090ed4       PeopleAMain                00491ed4   PUBLIC.obj
 0001:00091011       EvChampPeople              00492011   PUBLIC.obj
 0001:000910dc       ChampPeopleMain            004920dc   PUBLIC.obj
 0001:0009112f       EvPeopleB                  0049212f   PUBLIC.obj
 0001:000911c8       PeopleBMain                004921c8   PUBLIC.obj
 0001:000912c6       EvCameraManA               004922c6   PUBLIC.obj
 0001:000912c6       EvPeopleC                  004922c6   PUBLIC.obj
 0001:000912c7       TurnToCamera               004922c7   PUBLIC.obj
 0001:000913b4       SetPeopleModel             004923b4   PUBLIC.obj
 0001:000914e4       EvGake                     004924e4   PUBLIC.obj
 0001:0009153d       GakeMain                   0049253d   PUBLIC.obj
 0001:00091aa0       InitIwayama                00492aa0   PUBLIC.obj
 0001:00091ac2       EvIwayama                  00492ac2   PUBLIC.obj
 0001:00091d8c       vint_in                    00492d8c   INT.obj
 0001:00091ee8       int_normal                 00492ee8   INT.obj
 0001:00091ee8       int_no                     00492ee8   INT.obj
 0001:00091ef8       int_dmag                   00492ef8   INT.obj
 0001:00091ef9       int_dmag_com               00492ef9   INT.obj
 0001:00091f70       int_dma                    00492f70   INT.obj
 0001:00091fb4       int_color                  00492fb4   INT.obj
 0001:00092030       int_stop_dma               00493030   INT.obj
 0001:00092034       int_dma_wait               00493034   INT.obj
 0001:00092114       int_m1_other               00493114   INT.obj
 0001:00092130       int_m1_color               00493130   INT.obj
 0001:00092150       int_m1_colorm              00493150   INT.obj
 0001:000921cc       int_m1_nocolor             004931cc   INT.obj
 0001:00092200       int_m1_colorg              00493200   INT.obj
 0001:00092254       int_m1_colorg_com          00493254   INT.obj
 0001:00092298       int_m1_colorg2p            00493298   INT.obj
 0001:000924f0       vint_out                   004934f0   INT.obj
 0001:00092764       sync_vout                  00493764   INT.obj
 0001:00092765       sync_dsp                   00493765   INT.obj
 0001:00092766       sync_vin                   00493766   INT.obj
 0001:00092767       sync                       00493767   INT.obj
 0001:00092768       intm_sync                  00493768   INT.obj
 0001:00092769       ints_sync                  00493769   INT.obj
 0001:00093038       record_asort               00494038   REC_ASORT.obj
 0001:00093185       record_entry               00494185   REC_ASORT.obj
 0001:000933b0       _init_texture              004943b0 f Texture.obj
 0001:000933e0       _AddExTexture              004943e0 f Texture.obj
 0001:00093510       _ExTexture                 00494510 f Texture.obj
 0001:00093540       _ExTextureCourse           00494540 f Texture.obj
 0001:00093570       _setup_texture             00494570 f Texture.obj
 0001:00093690       _entry_texture             00494690 f Texture.obj
 0001:00093700       _set_texture_cg            00494700 f Texture.obj
 0001:00093760       _set_texture_cl            00494760 f Texture.obj
 0001:000937c0       _set_course_model_00       004947c0 f Texture.obj
 0001:00093860       _set_course_model          00494860 f Texture.obj
 0001:00093900       _set_course_texture        00494900 f Texture.obj
 0001:000939a0       _set_course_model_2p       004949a0 f Texture.obj
 0001:00093a40       _set_game2p_model          00494a40 f Texture.obj
 0001:00093c90       _set_game_texture          00494c90 f Texture.obj
 0001:00093fe0       _GameTextureReload         00494fe0 f Texture.obj
 0001:00094340       _set_car_texture           00495340 f Texture.obj
 0001:000944e0       _set_object_model          004954e0 f Texture.obj
 0001:00094680       _set_object2p_model        00495680 f Texture.obj
 0001:00094910       _set_animal2_model         00495910 f Texture.obj
 0001:00094a80       _set_alphabet_model        00495a80 f Texture.obj
 0001:00094aa0       _set_select_model          00495aa0 f Texture.obj
 0001:00094c10       _set_ceremony_model        00495c10 f Texture.obj
 0001:00094e90       _set_staff_model           00495e90 f Texture.obj
 0001:00095000       __result_main              00496000   RES_MAIN.obj
 0001:00095000       result_main                00496000   RES_MAIN.obj
 0001:00095811       result_main_loop           00496811   RES_MAIN.obj
 0001:00096174       InitGenerator              00497174   GENERATOR.obj
 0001:00096278       ExecGenerator              00497278   GENERATOR.obj
 0001:000965f1       sl_ExecGenerator           004975f1   GENERATOR.obj
 0001:00096822       InitGenerator_2p           00497822   GENERATOR.obj
 0001:000968f3       InitGenerator_net          004978f3   GENERATOR.obj
 0001:000969c4       ExecGenerator_2p           004979c4   GENERATOR.obj
 0001:00096bb6       sl_ExecGenerator_2p        00497bb6   GENERATOR.obj
 0001:00096d54       InitGeneratorSub           00497d54   GENERATOR.obj
 0001:00096fb2       ExecGenerator_net          00497fb2   GENERATOR.obj
 0001:00097424       LoadEventData              00498424   GENERATOR.obj
 0001:00097440       EventExecTbl               00498440   GENERATOR.obj
 0001:000974c0       title_init_hori            004984c0   TITLEhori.obj
 0001:00097da0       _IsJoyConnect              00498da0 f Keydlg.obj
 0001:00097dc0       _FindIndex                 00498dc0 f Keydlg.obj
 0001:00097e90       _FindKey                   00498e90 f Keydlg.obj
 0001:00097f50       _KeyListCopy_Key           00498f50 f Keydlg.obj
 0001:00097ff0       _KeyListCopy_Joy           00498ff0 f Keydlg.obj
 0001:00098070       _KeyListCopy               00499070 f Keydlg.obj
 0001:000980b0       _ComboIDtoKeyPtr           004990b0 f Keydlg.obj
 0001:000981a0       _SetKeyComboItem           004991a0 f Keydlg.obj
 0001:000981f0       _SetInputDeviceType        004991f0 f Keydlg.obj
 0001:00098380       _GetComboData              00499380 f Keydlg.obj
 0001:00098440       _ConfigKeyPage@16          00499440 f Keydlg.obj
 0001:00098710       _SetJoyPlayer_pad_cur      00499710 f Keydlg.obj
 0001:00098800       _ConfigJoyPage@16          00499800 f Keydlg.obj
 0001:00098ca0       _CreatePropertySheet       00499ca0 f Keydlg.obj
 0001:00098da0       _CreateKeyConfig           00499da0 f Keydlg.obj
 0001:00098e60       _KeycodeToKeyname          00499e60 f Keydlg.obj
 0001:00098fc0       _KeynameToKeycode          00499fc0 f Keydlg.obj
 0001:00099114       init_alwram                0049a114   INIT.obj
 0001:00099194       init_wram                  0049a194   INIT.obj
 0001:000991d0       init_colorwk               0049a1d0   INIT.obj
 0001:0009920c       init_game_work_start       0049a20c   INIT.obj
 0001:00099608       init_game_work_start2p     0049a608   INIT.obj
 0001:000996b0       cg_dataset                 0049a6b0   INIT.obj
 0001:000998a8       init_game_vram             0049a8a8   INIT.obj
 0001:00099a3c       game_scr_on                0049aa3c   INIT.obj
 0001:00099a40       result_mchg_cg             0049aa40   INIT.obj
 0001:00099ab0       c_race                     0049aab0   INIT.obj
 0001:00099bec       c_practice                 0049abec   INIT.obj
 0001:00099dd8       c_vs                       0049add8   INIT.obj
 0001:00099eb4       init_gspr2                 0049aeb4   INIT.obj
 0001:00099ee0       init_gspr                  0049aee0   INIT.obj
 0001:0009a034       init_nscr_vol              0049b034   INIT.obj
 0001:0009a112       colorset                   0049b112   INIT.obj
 0001:0009a1c8       crs_dataset                0049b1c8   INIT.obj
 0001:0009a1d8       crs_adv_dataset            0049b1d8   INIT.obj
 0001:0009a1fc       crs_cer_dataset            0049b1fc   INIT.obj
 0001:0009a1fc       crs_bgdataset              0049b1fc   INIT.obj
 0001:0009a358       init_game_work             0049b358   INIT.obj
 0001:0009a9e0       init_game_work2p           0049b9e0   INIT.obj
 0001:0009af00       myline_set                 0049bf00   INIT.obj
 0001:0009b149       copy_dram                  0049c149   INIT.obj
 0001:0009b729       copy_dram2                 0049c729   INIT.obj
 0001:0009bb41       data_copy                  0049cb41   INIT.obj
 0001:0009bb44       init_nclram                0049cb44   INIT.obj
 0001:0009bbf0       set_tasc_cg                0049cbf0   INIT.obj
 0001:0009bcb8       set_space_cg               0049ccb8   INIT.obj
 0001:0009bd8c       set_tasc_cl                0049cd8c   INIT.obj
 0001:0009bdcc       init_adv_vdp2              0049cdcc   INIT.obj
 0001:0009bf74       init_ending_vdp2           0049cf74   INIT.obj
 0001:0009c0d0       init_pcmdata               0049d0d0   INIT.obj
 0001:0009c0d4       record_disp                0049d0d4   REC_MODEDISP.obj
 0001:0009c438       game_ctrl                  0049d438   GCTRL.obj
 0001:0009d23c       camera_ctrl                0049e23c   GCTRL.obj
 0001:0009d270       camera1p_ctrl              0049e270   GCTRL.obj
 0001:0009d2b8       camera2p_ctrl              0049e2b8   GCTRL.obj
 0001:0009d3b0       camera_non                 0049e3b0   GCTRL.obj
 0001:0009d3b4       clr_camera_ctrl_work       0049e3b4   GCTRL.obj
 0001:0009d408       rscroll_ctrl               0049e408   GCTRL.obj
 0001:0009d43c       rscroll2p_ctrl             0049e43c   GCTRL.obj
 0001:0009d4ac       rscroll_non                0049e4ac   GCTRL.obj
 0001:0009d4b0       clr_rscroll_ctrl_work      0049e4b0   GCTRL.obj
 0001:0009d504       car_move_ctrl              0049e504   GCTRL.obj
 0001:0009d668       allclr_car_ctrl_work       0049e668   GCTRL.obj
 0001:0009d70c       car_move2p_ctrl            0049e70c   GCTRL.obj
 0001:0009d740       m_car_move2p_ctrl          0049e740   GCTRL.obj
 0001:0009d7e8       s_car_move2p_ctrl          0049e7e8   GCTRL.obj
 0001:0009da80       car_disp2p_ctrl            0049ea80   GCTRL.obj
 0001:0009dab4       m_car_disp2p_ctrl          0049eab4   GCTRL.obj
 0001:0009db5c       s_car_disp2p_ctrl          0049eb5c   GCTRL.obj
 0001:0009deb0       _battle_scroll_act_1       0049eeb0 f CS_BATTLE_2P.obj
 0001:0009df30       _battle_scroll_act_2       0049ef30 f CS_BATTLE_2P.obj
 0001:0009e000       _battle_2p_init            0049f000 f CS_BATTLE_2P.obj
 0001:0009e3c0       _battle_2p_main            0049f3c0 f CS_BATTLE_2P.obj
 0001:0009eee0       _btlay_1p_0                0049fee0 f CS_BATTLE_2P.obj
 0001:0009f150       _btlay_2p_0                004a0150 f CS_BATTLE_2P.obj
 0001:0009f430       _btlay_1p_1                004a0430 f CS_BATTLE_2P.obj
 0001:0009f5f0       _btlay_2p_1                004a05f0 f CS_BATTLE_2P.obj
 0001:0009f850       _btlay_1p_2                004a0850 f CS_BATTLE_2P.obj
 0001:0009faa0       _btlay_2p_2                004a0aa0 f CS_BATTLE_2P.obj
 0001:0009fcf0       _btlay_1p_3                004a0cf0 f CS_BATTLE_2P.obj
 0001:0009fd90       _btlay_2p_3                004a0d90 f CS_BATTLE_2P.obj
 0001:0009fe00       _btlay4                    004a0e00 f CS_BATTLE_2P.obj
 0001:0009ffa0       _btlay5                    004a0fa0 f CS_BATTLE_2P.obj
 0001:000a01a0       _btlay6                    004a11a0 f CS_BATTLE_2P.obj
 0001:000a06d0       _btlay7                    004a16d0 f CS_BATTLE_2P.obj
 0001:000a08b0       _btlay8                    004a18b0 f CS_BATTLE_2P.obj
 0001:000a0bc0       _bt_cancel                 004a1bc0 f CS_BATTLE_2P.obj
 0001:000a0c00       _calc_padmax0              004a1c00 f CS_BATTLE_2P.obj
 0001:000a0c40       _calc_padmax1              004a1c40 f CS_BATTLE_2P.obj
 0001:000a0c50       _calc_padmax3              004a1c50 f CS_BATTLE_2P.obj
 0001:000a0c70       _pass_setting_1p           004a1c70 f CS_BATTLE_2P.obj
 0001:000a0cd0       _pass_setting_2p           004a1cd0 f CS_BATTLE_2P.obj
 0001:000a0d30       _bt_dummy                  004a1d30 f CS_BATTLE_2P.obj
 0001:000a0d40       _bt_ret_battle_2p          004a1d40 f CS_BATTLE_2P.obj
 0001:000a0e00       _battle_scroll_change      004a1e00 f CS_BATTLE_2P.obj
 0001:000a1d40       _battle_line_scroll        004a2d40 f CS_BATTLE_2P.obj
 0001:000a1fa0       _battle_scroll_init        004a2fa0 f CS_BATTLE_2P.obj
 0001:000a2010       _battle_scroll_set         004a3010 f CS_BATTLE_2P.obj
 0001:000a2140       _battle_2pscroll_change    004a3140 f CS_BATTLE_2P.obj
 0001:000a23f0       _battle_line_2pscroll      004a33f0 f CS_BATTLE_2P.obj
 0001:000a2530       _battle_2pscroll_init      004a3530 f CS_BATTLE_2P.obj
 0001:000a2590       _battle_2pscroll_set       004a3590 f CS_BATTLE_2P.obj
 0001:000a26c0       _battle_scroll_set_poly    004a36c0 f CS_BATTLE_2P.obj
 0001:000a27b0       name_moji_act              004a37b0   NAME_MOJI.obj
 0001:000a2be1       _draw_polygon              004a3be1   NAME_MOJI.obj
 0001:000a3260       name_disp                  004a4260   NAME_DISP.obj
 0001:000a3260       adv_name_disp              004a4260   NAME_DISP.obj
 0001:000a3260       adv_rec_disp               004a4260   NAME_DISP.obj
 0001:000a3260       name_rec_disp              004a4260   NAME_DISP.obj
 0001:000a3260       adv_record_disp            004a4260   NAME_DISP.obj
 0001:000a3260       name_name_disp             004a4260   NAME_DISP.obj
 0001:000a3261       name_disp2                 004a4261   NAME_DISP.obj
 0001:000a3288       set_flatgour_tbl           004a4288   SHADING.obj
 0001:000a3300       zsort                      004a4300   ZSORT.obj
 0001:000a3859       zsort2                     004a4859   ZSORT.obj
 0001:000a3db5       clr_zsortcnt               004a4db5   ZSORT.obj
 0001:000a3e3b       normal_zsort               004a4e3b   ZSORT.obj
 0001:000a3f14       game_zsort                 004a4f14   ZSORT.obj
 0001:000a4171       game_zsort_2p              004a5171   ZSORT.obj
 0001:000a44fc       link_cmdtbl                004a54fc   ZSORT.obj
 0001:000a457f       get_top_cmdtbl             004a557f   ZSORT.obj
 0001:000a46f7       get_top_cmdtbl_2p          004a56f7   ZSORT.obj
 0001:000a494f       set_game_cmdtbl            004a594f   ZSORT.obj
 0001:000a49e8       set_vsgame_cmdtbl          004a59e8   ZSORT.obj
 0001:000a4b68       set_gamescrn_cmdtbl        004a5b68   ZSORT.obj
 0001:000a4d03       set_centerline_cmdtbl      004a5d03   ZSORT.obj
 0001:000a4fc0       CallQMotion                004a5fc0   MOTION.obj
 0001:000a533c       EndCallMotion              004a633c   MOTION.obj
 0001:000a5a40       _line_scroll_init          004a6a40 f record.obj
 0001:000a5ad0       _line_scroll_set           004a6ad0 f record.obj
 0001:000a5c00       _timeattack_pict_set       004a6c00 f record.obj
 0001:000a5d70       _a_p_t_pict_set            004a6d70 f record.obj
 0001:000a5fc0       _a_c_p_pict_set            004a6fc0 f record.obj
 0001:000a60b0       _a_p_c_pict_set            004a70b0 f record.obj
 0001:000a6180       _change_lap_pict_set       004a7180 f record.obj
 0001:000a61a0       _game_start_pict_set       004a71a0 f record.obj
 0001:000a61e0       _change_cource_pict_set    004a71e0 f record.obj
 0001:000a6210       _change_timeattack_cource_pict_set 004a7210 f record.obj
 0001:000a6240       _change_timeattack_car_pict_set 004a7240 f record.obj
 0001:000a6300       _line_scroll_change        004a7300 f record.obj
 0001:000a6940       _line_scroll_main          004a7940 f record.obj
 0001:000a6af0       _record_scroll_act_1       004a7af0 f record.obj
 0001:000a6b80       _record_scroll_act_2       004a7b80 f record.obj
 0001:000a6d70       _record_init               004a7d70 f record.obj
 0001:000a7770       _record_main               004a8770 f record.obj
 0001:000a7ab0       _record_scroll_lanking     004a8ab0 f record.obj
 0001:000a7d00       _record_main_championship  004a8d00 f record.obj
 0001:000a84e0       _record_main_practice      004a94e0 f record.obj
 0001:000a89c0       _record_main_timeattack    004a99c0 f record.obj
 0001:000a9aa0       _record_scroll_act_3       004aaaa0 f record.obj
 0001:000a9ae0       _record_time_get           004aaae0 f record.obj
 0001:000a9f50       _moji_reload               004aaf50 f record.obj
 0001:000aa010       _mirror_mode_off           004ab010 f record.obj
 0001:000aa020       _mirror_mode_check         004ab020 f record.obj
 0001:000aa040       _champion_game_flag_main   004ab040 f record.obj
 0001:000aa070       _champion_car_flag_main    004ab070 f record.obj
 0001:000aa0a0       _champion_cource_flag_main 004ab0a0 f record.obj
 0001:000aa0f0       _mode_select_flag_main     004ab0f0 f record.obj
 0001:000aa120       _stratos_check             004ab120 f record.obj
 0001:000aa1d0       initCarControl             004ab1d0   CARCTRL.obj
 0001:000aa259       carControl                 004ab259   CARCTRL.obj
 0001:000aa3eb       calc_kajyu                 004ab3eb   CARCTRL.obj
 0001:000aaad8       calc_front                 004abad8   CARCTRL.obj
 0001:000ab44b       calc_rear                  004ac44b   CARCTRL.obj
 0001:000abed5       vibration_y                004aced5   CARCTRL.obj
 0001:000ac5c8       pointvecsub                004ad5c8   CARCTRL.obj
 0001:000ac748       guidetbl                   004ad748   OTHERDAT.obj
 0001:000ac758       CarRankTable               004ad758   OTHERDAT.obj
 0001:000ac76c       octpr_inittbl              004ad76c   OTHERDAT.obj
 0001:000ac9f4       distStep_e                 004ad9f4   OTHERDAT.obj
 0001:000aca54       octgptbl                   004ada54   OTHERDAT.obj
 0001:000acb40       acc_gp                     004adb40   OTHERDAT.obj
 0001:000acb50       acc_pr                     004adb50   OTHERDAT.obj
 0001:000acb90       crvspdmin                  004adb90   OTHERDAT.obj
 0001:000acb94       setOtherCar                004adb94   OTHERSET.obj
 0001:000acf67       update_pos                 004adf67   OTHERSET.obj
 0001:000ad2f9       calc_tforce                004ae2f9   OTHERSET.obj
 0001:000ad5bd       calc_rear_force            004ae5bd   OTHERSET.obj
 0001:000adadb       turn_yaw_r                 004aeadb   OTHERSET.obj
 0001:000adec1       turn_yaw_f                 004aeec1   OTHERSET.obj
 0001:000ae1c0       calc_cousin                004af1c0   OTHERSET.obj
 0001:000ae5c5       calc_moment                004af5c5   OTHERSET.obj
 0001:000aebd1       outforce                   004afbd1   OTHERSET.obj
 0001:000aedcb       ctrl_roll                  004afdcb   OTHERSET.obj
 0001:000af41f       calc_resist                004b041f   OTHERSET.obj
 0001:000af8e8       tinyForce                  004b08e8   OTHERSET.obj
 0001:000b007d       otrCarColi                 004b107d   OTHERSET.obj
 0001:000b0e44       set_pict_tm_att            004b1e44   CS_TM_ATT_PSET.obj
 0001:000b11f4       tm_color_chg               004b21f4   CS_TM_ATT_PSET.obj
 0001:000b12aa       tm_pict_bright             004b22aa   CS_TM_ATT_PSET.obj
 0001:000b16b4       pict_bright_tmlay2         004b26b4   CS_TM_ATT_PSET.obj
 0001:000b17fc       chg_c_name                 004b27fc   CS_TM_ATT_PSET.obj
 0001:000b19dc       chg_crs_name               004b29dc   CS_TM_ATT_PSET.obj
 0001:000b1cfc       chg_lap_name               004b2cfc   CS_TM_ATT_PSET.obj
 0001:000b1e6c       delete_lap_seat            004b2e6c   CS_TM_ATT_PSET.obj
 0001:000b1ea8       draw_lap_time              004b2ea8   CS_TM_ATT_PSET.obj
 0001:000b209f       set_pict_result            004b309f   CS_TM_ATT_PSET.obj
 0001:000b2290       return_tm_att              004b3290   CS_TM_ATT_PSET.obj
 0001:000b22e0       __tm_set_tm_att            004b32e0   CS_TM_ATT_PSET.obj
 0001:000b22e0       tm_set_tm_att              004b32e0   CS_TM_ATT_PSET.obj
 0001:000b2a7c       record_RAC                 004b3a7c   REC_RAC.obj
 0001:000b2e40       _DeleteScrollBitmapTable   004b3e40 f LoadScrollBmp.obj
 0001:000b2ea0       _LoadInitScrollPalette     004b3ea0 f LoadScrollBmp.obj
 0001:000b2f20       _CreateScrollBitmapTable   004b3f20 f LoadScrollBmp.obj
 0001:000b3190       ?LoadScrollBitmap_All_Compress@@YAHXZ 004b4190 f LoadScrollBmp.obj
 0001:000b3330       _LoadScrollBitmap          004b4330 f LoadScrollBmp.obj
 0001:000b3350       record_RACx                004b4350   REC_RACX.obj
 0001:000b363c       t_cos                      004b463c   MATH.obj
 0001:000b3654       t_sin                      004b4654   MATH.obj
 0001:000b3a74       r_sin                      004b4a74   MATH.obj
 0001:000b3aa0       sin                        004b4aa0   MATH.obj
 0001:000b3af0       r_cos                      004b4af0   MATH.obj
 0001:000b3b1c       cos                        004b4b1c   MATH.obj
 0001:000b3b6c       r_atan                     004b4b6c   MATH.obj
 0001:000b3bc8       atan                       004b4bc8   MATH.obj
 0001:000b3e1c       distance_2d                004b4e1c   MATH.obj
 0001:000b3f30       distance_3d                004b4f30   MATH.obj
 0001:000b4050       sqrt                       004b5050   MATH.obj
 0001:000b4164       inner_product              004b5164   MATH.obj
 0001:000b4228       outer_product              004b5228   MATH.obj
 0001:000b44a8       calc_point                 004b54a8   MATH.obj
 0001:000b4764       calc_point2                004b5764   MATH.obj
 0001:000b49d8       bspline                    004b59d8   MATH.obj
 0001:000b4c45       get_lookat_angle           004b5c45   MATH.obj
 0001:000b4efc       record_RTx                 004b5efc   REC_RTX.obj
 0001:000b5478       c_outp2                    004b6478   COPRO.obj
 0001:000b550c       c_getr                     004b650c   COPRO.obj
 0001:000b5694       c_vecval                   004b6694   COPRO.obj
 0001:000b57d4       c_turnd                    004b67d4   COPRO.obj
 0001:000b57fc       c_turnv                    004b67fc   COPRO.obj
 0001:000b57fc       c_turnv2                   004b67fc   COPRO.obj
 0001:000b5824       c_turnsub                  004b6824   COPRO.obj
 0001:000b5c1c       c_turnsub2                 004b6c1c   COPRO.obj
 0001:000b6020       turn_alpha                 004b7020   COPRO.obj
 0001:000b62d0       turn_beta                  004b72d0   COPRO.obj
 0001:000b6584       regularAngle               004b7584   COPRO.obj
 0001:000b6610       asinf                      004b7610   COPRO.obj
 0001:000b67d8       c_point_rm                 004b77d8   COPRO.obj
 0001:000b6820       c_point_mm                 004b7820   COPRO.obj
 0001:000b6820       c_point                    004b7820   COPRO.obj
 0001:000b6820       c_vector                   004b7820   COPRO.obj
 0001:000b6adc       c_point_rr                 004b7adc   COPRO.obj
 0001:000b6b24       c_point_mr                 004b7b24   COPRO.obj
 0001:000b6db8       c_point_rr_xz              004b7db8   COPRO.obj
 0001:000b6e00       c_point_mr_xz              004b7e00   COPRO.obj
 0001:000b6fc1       c_point_rm_xz              004b7fc1   COPRO.obj
 0001:000b7008       c_point_mm_xz              004b8008   COPRO.obj
 0001:000b71e4       c_reg                      004b81e4   COPRO.obj
 0001:000b71e4       c_reg_xz                   004b81e4   COPRO.obj
 0001:000b749c       initOtherGP                004b849c   OTHERCTRL.obj
 0001:000b79d7       initgp_sub                 004b89d7   OTHERCTRL.obj
 0001:000b7ca3       initOtherPR                004b8ca3   OTHERCTRL.obj
 0001:000b81f8       initOtherCar               004b91f8   OTHERCTRL.obj
 0001:000b88ee       otherCtrl                  004b98ee   OTHERCTRL.obj
 0001:000b8a25       otherctrlGP                004b9a25   OTHERCTRL.obj
 0001:000b8f54       otherctrlPR                004b9f54   OTHERCTRL.obj
 0001:000b92a6       chkranksub                 004ba2a6   OTHERCTRL.obj
 0001:000b9384       getCarLink                 004ba384   OTHERCTRL.obj
 0001:000b96c0       initial_matrix             004ba6c0   MATRIX.obj
 0001:000b9708       unit_matrix                004ba708   MATRIX.obj
 0001:000b97cc       push_matrix                004ba7cc   MATRIX.obj
 0001:000b9934       pop_matrix                 004ba934   MATRIX.obj
 0001:000b993c       copy_matrix                004ba93c   MATRIX.obj
 0001:000b9adb       translate2                 004baadb   MATRIX.obj
 0001:000b9b08       translate                  004bab08   MATRIX.obj
 0001:000b9c30       translate_xy               004bac30   MATRIX.obj
 0001:000b9d34       translate_xz               004bad34   MATRIX.obj
 0001:000b9e40       translate_yz               004bae40   MATRIX.obj
 0001:000b9f4c       translate_x                004baf4c   MATRIX.obj
 0001:000ba000       translate_y                004bb000   MATRIX.obj
 0001:000ba0b4       translate_z                004bb0b4   MATRIX.obj
 0001:000ba168       scale                      004bb168   MATRIX.obj
 0001:000ba2b8       scale_x                    004bb2b8   MATRIX.obj
 0001:000ba350       scale_y                    004bb350   MATRIX.obj
 0001:000ba3ec       scale_z                    004bb3ec   MATRIX.obj
 0001:000ba488       reverse_x                  004bb488   MATRIX.obj
 0001:000ba4f0       reverse_y                  004bb4f0   MATRIX.obj
 0001:000ba558       reverse_z                  004bb558   MATRIX.obj
 0001:000ba5c0       r_rotate_x                 004bb5c0   MATRIX.obj
 0001:000ba5ea       rotate_x                   004bb5ea   MATRIX.obj
 0001:000ba7b4       r_rotate_y                 004bb7b4   MATRIX.obj
 0001:000ba7de       rotate_y                   004bb7de   MATRIX.obj
 0001:000ba9b0       r_rotate_z                 004bb9b0   MATRIX.obj
 0001:000ba9da       rotate_z                   004bb9da   MATRIX.obj
 0001:000bab9c       sincos                     004bbb9c   MATRIX.obj
 0001:000bac12       mul_matrix                 004bbc12   MATRIX.obj
 0001:000badb9       calc_camera_matrix         004bbdb9   MATRIX.obj
 0001:000bae7e       t_rotate_x                 004bbe7e   MATRIX.obj
 0001:000baf11       t_rotate_y                 004bbf11   MATRIX.obj
 0001:000bafa4       t_rotate_z                 004bbfa4   MATRIX.obj
 0001:000bb038       purge_matrix               004bc038   MATRIX.obj
 0001:000bb077       get_matrixbuf              004bc077   MATRIX.obj
 0001:000bb0bf       store_matrix_pointer       004bc0bf   MATRIX.obj
 0001:000bb114       restore_matrix_pointer     004bc114   MATRIX.obj
 0001:000bb170       _tm_scroll_act_1           004bc170 f tm_attck.obj
 0001:000bb1e0       _tm_scroll_act_2           004bc1e0 f tm_attck.obj
 0001:000bb290       _time_attck_init           004bc290 f tm_attck.obj
 0001:000bb4c0       _time_attck_main           004bc4c0 f tm_attck.obj
 0001:000bb870       _tm_lay0                   004bc870 f tm_attck.obj
 0001:000bbb60       _tm_lay1                   004bcb60 f tm_attck.obj
 0001:000bbda0       _tm_lay2                   004bcda0 f tm_attck.obj
 0001:000bbef0       _tm_lay3                   004bcef0 f tm_attck.obj
 0001:000bc110       _tm_lay4                   004bd110 f tm_attck.obj
 0001:000bc2a0       _tm_cancel                 004bd2a0 f tm_attck.obj
 0001:000bc2e0       _set_sprite_tm_att         004bd2e0 f tm_attck.obj
 0001:000bc3e0       _tm_sprite_bright          004bd3e0 f tm_attck.obj
 0001:000bc520       _at_mt_disp                004bd520 f tm_attck.obj
 0001:000bc680       _tm_course_bright          004bd680 f tm_attck.obj
 0001:000bc6f0       _tm_tune_bright            004bd6f0 f tm_attck.obj
 0001:000bc780       _pass_setting              004bd780 f tm_attck.obj
 0001:000bc7f0       _disp_tune_car             004bd7f0 f tm_attck.obj
 0001:000bc890       _disp_standard_car         004bd890 f tm_attck.obj
 0001:000bc900       _record_time_disp          004bd900 f tm_attck.obj
 0001:000bcbe0       _record_time_erace         004bdbe0 f tm_attck.obj
 0001:000bcd00       _set_tm_course             004bdd00 f tm_attck.obj
 0001:000bcdd0       _set_tm_lap                004bddd0 f tm_attck.obj
 0001:000bce00       _tm_scroll_change          004bde00 f tm_attck.obj
 0001:000bd3f0       _tm_line_scroll            004be3f0 f tm_attck.obj
 0001:000bd5e0       _tm_scroll_init            004be5e0 f tm_attck.obj
 0001:000bd660       _tm_scroll_set             004be660 f tm_attck.obj
 0001:000bd790       _tm_scroll_set_poly        004be790 f tm_attck.obj
 0001:000bd850       rec_mark_act               004be850   REC_MARKACT.obj
 0001:000bddb0       _PolyMesh16                004bedb0 f FPOLY16.obj
 0001:000c0280       crs_select_init            004c1280   AC_CRS_SELECT.obj
 0001:000c06ab       crs_select_main            004c16ab   AC_CRS_SELECT.obj
 0001:000c0927       crs_white_in               004c1927   AC_CRS_SELECT.obj
 0001:000c09e7       crs_check_pad              004c19e7   AC_CRS_SELECT.obj
 0001:000c0c54       crs_blink                  004c1c54   AC_CRS_SELECT.obj
 0001:000c2d10       _gfxBlt                    004c3d10 f gfx.obj
 0001:000c2ee0       _gfxCreateSolidColorBitmap 004c3ee0 f gfx.obj
 0001:000c2f30       _gfxCreateVramBitmap       004c3f30 f gfx.obj
 0001:000c2fe0       _gfxDestroyBitmap          004c3fe0 f gfx.obj
 0001:000c3030       _gfxStretchBackbuffer      004c4030 f gfx.obj
 0001:000c3090       _gfxFlip                   004c4090 f gfx.obj
 0001:000c30b0       _gfxUpdateWindow           004c40b0 f gfx.obj
 0001:000c30e0       _gfxSwapBuffers            004c40e0 f gfx.obj
 0001:000c31a0       _gfxBegin                  004c41a0 f gfx.obj
 0001:000c31d0       _gfxEnd                    004c41d0 f gfx.obj
 0001:000c3230       _gfxRestore                004c4230 f gfx.obj
 0001:000c3620       _gfxRestoreAll             004c4620 f gfx.obj
 0001:000c3690       _gfxFillBack               004c4690 f gfx.obj
 0001:000c36d0       _resultlink_init           004c46d0 f res_link.obj
 0001:000c3710       _resultlink_main           004c4710 f res_link.obj
 0001:000c3850       __name_exit                004c4850   NAME_EXIT.obj
 0001:000c3850       name_exit                  004c4850   NAME_EXIT.obj
 0001:000c3c72       name_exit_loop             004c4c72   NAME_EXIT.obj
 0001:000c4ec8       __game_over                004c5ec8   NAME_EXIT.obj
 0001:000c4ec8       game_over                  004c5ec8   NAME_EXIT.obj
 0001:000c5117       game_over_loop             004c6117   NAME_EXIT.obj
 0001:000c5550       init_pict_w                004c6550   CS_PICT_SET.obj
 0001:000c55cf       set_pict_md_slt            004c65cf   CS_PICT_SET.obj
 0001:000c57d4       md_color_chg               004c67d4   CS_PICT_SET.obj
 0001:000c588a       md_pict_set_bright         004c688a   CS_PICT_SET.obj
 0001:000c5b90       set_pict_next_md           004c6b90   CS_PICT_SET.obj
 0001:000c5d98       set_pict_record            004c6d98   CS_PICT_SET.obj
 0001:000c5f94       record_RAP                 004c6f94   REC_RAP.obj
 0001:000c6378       execOtherCar               004c7378   OTHERCAR.obj
 0001:000c64c2       sleepctrl                  004c74c2   OTHERCAR.obj
 0001:000c695f       speed_ctrl                 004c795f   OTHERCAR.obj
 0001:000c8120       nearCarProc                004c9120   OTHERCAR.obj
 0001:000c835c       setMark                    004c935c   OTHERCAR.obj
 0001:000c887d       b_spline                   004c987d   OTHERCAR.obj
 0001:000c8fec       set_2way_cache             004c9fec   CACHE.obj
 0001:000c8fed       purge_00                   004c9fed   CACHE.obj
 0001:000c8fee       cache_all_purge            004c9fee   CACHE.obj
 0001:000c8fef       clear_cache                004c9fef   CACHE.obj
 0001:000c8ff0       clear_cache_ram            004c9ff0   CACHE.obj
 0001:000c8ff4       lscrl_init                 004c9ff4   LINE_SCRL.obj
 0001:000c9012       lscrl_init2                004ca012   LINE_SCRL.obj
 0001:000c905b       lscrl_plus                 004ca05b   LINE_SCRL.obj
 0001:000c9083       lscrl_plus2                004ca083   LINE_SCRL.obj
 0001:000c9164       lscrl_minus                004ca164   LINE_SCRL.obj
 0001:000c918c       lscrl_minus2               004ca18c   LINE_SCRL.obj
 0001:000c926d       spr_plus                   004ca26d   LINE_SCRL.obj
 0001:000c9321       spr_minus                  004ca321   LINE_SCRL.obj
 0001:000c93e0       _DDEnable                  004ca3e0 f ddraw.obj
 0001:000c9840       _DDDisable                 004ca840 f ddraw.obj
 0001:000c98d0       _DDClear                   004ca8d0 f ddraw.obj
 0001:000c9990       _DDCreateFlippingSurface   004ca990 f ddraw.obj
 0001:000c9d30       _DDCreateSurface           004cad30 f ddraw.obj
 0001:000c9e00       _DDColorMatch              004cae00 f ddraw.obj
 0001:000c9ef0       _CreateDefaultPal          004caef0 f ddraw.obj
 0001:000c9fe0       _Splash                    004cafe0 f ddraw.obj
 0001:000ca020       _MemAlloc                  004cb020 f ddraw.obj
 0001:000ca030       _CMemAlloc                 004cb030 f ddraw.obj
 0001:000ca050       _MemFree                   004cb050 f ddraw.obj
 0001:000ca060       _EnumDisplayModesCallback@8 004cb060 f ddraw.obj
 0001:000ca0b0       tm_attck_init              004cb0b0   CS_TM_ATTCK.obj
 0001:000ca768       tm_attck_main              004cb768   CS_TM_ATTCK.obj
 0001:000cc2fb       check_mirror               004cd2fb   CS_TM_ATTCK.obj
 0001:000cc374       pad_check                  004cd374   CS_TM_ATTCK.obj
 0001:000cc3b5       pad_check2                 004cd3b5   CS_TM_ATTCK.obj
 0001:000cc638       check_stratos_flg          004cd638   CS_TM_ATTCK.obj
 0001:000cc68b       check_lake_flg             004cd68b   CS_TM_ATTCK.obj
 0001:000cc6de       check_tune_flg             004cd6de   CS_TM_ATTCK.obj
 0001:000cc781       tm_open_win                004cd781   CS_TM_ATTCK.obj
 0001:000cc938       tm_close_win               004cd938   CS_TM_ATTCK.obj
 0001:000ccad1       tm_get_times               004cdad1   CS_TM_ATTCK.obj
 0001:000ccbd9       tm_solute_times            004cdbd9   CS_TM_ATTCK.obj
 0001:000ce62e       check_ghost_md             004cf62e   CS_TM_ATTCK.obj
 0001:000ce854       set_car                    004cf854   CS_CAR_SET.obj
 0001:000ce9cf       disp_car                   004cf9cf   CS_CAR_SET.obj
 0001:000cec88       disp_car_tm_setting        004cfc88   CS_CAR_SET.obj
 0001:000cef1f       display_car_tm             004cff1f   CS_CAR_SET.obj
 0001:000cefc5       put_modeltype              004cffc5   CS_CAR_SET.obj
 0001:000cefd7       put_modeltype2             004cffd7   CS_CAR_SET.obj
 0001:000cf014       bt_disp_car                004d0014   CS_CAR_SET.obj
 0001:000cf0b0       record_RT                  004d00b0   REC_RT.obj
 0001:000cf578       backup_melt                004d0578   BUP_MELT.obj
 0001:000cf90e       _backup_check              004d090e   BUP_MELT.obj
 0001:000cf9b4       _backup_g_check            004d09b4   BUP_MELT.obj
 0001:000cfad4       init_count                 004d0ad4   timer.obj
 0001:000cfb29       count_down                 004d0b29   timer.obj
 0001:000cfc8a       disp_time                  004d0c8a   timer.obj
 0001:000cfe07       draw_number                004d0e07   timer.obj
 0001:000d01ec       __photo_init               004d11ec   PHOTO.obj
 0001:000d01ec       photo_init                 004d11ec   PHOTO.obj
 0001:000d05b4       init_photo_work_start      004d15b4   PHOTO.obj
 0001:000d0704       init_photo_work            004d1704   PHOTO.obj
 0001:000d0898       photo_main                 004d1898   PHOTO.obj
 0001:000d12f0       _SuzuTexInit8              004d22f0 f Fchatex8.obj
 0001:000d1430       _SetPolygonDDInit8         004d2430 f Fchatex8.obj
 0001:000d1460       _Texture8                  004d2460 f Fchatex8.obj
 0001:000d2ef0       blinkle_init               004d3ef0   blinkle.obj
 0001:000d31b5       blinkle                    004d41b5   blinkle.obj
 0001:000d3600       init_light                 004d4600   LIGHT.obj
 0001:000d3600       init_light_vector          004d4600   LIGHT.obj
 0001:000d36d5       calc_light                 004d46d5   LIGHT.obj
 0001:000d37a2       rotate_light_vector        004d47a2   LIGHT.obj
 0001:000d37a2       rotate_light               004d47a2   LIGHT.obj
 0001:000d3adc       BUP_Mes_Tbl                004d4adc   REC_STRING.obj
 0001:000d428c       getIO_pad                  004d528c   PAD.obj
 0001:000d42d2       getIO_analog               004d52d2   PAD.obj
 0001:000d442a       getIO_digital              004d542a   PAD.obj
 0001:000d4722       get_accel                  004d5722   PAD.obj
 0001:000d4a1a       calc_diff                  004d5a1a   PAD.obj
 0001:000d4b48       carconfig                  004d5b48   PAD.obj
 0001:000d521c       cfg_stratos                004d621c   PAD.obj
 0001:000d5568       cardyncfgtbl               004d6568   PAD.obj
 0001:000d5678       cardyntable                004d6678   cardata.obj
 0001:000d56b8       carDynTarmac               004d66b8   cardata.obj
 0001:000d56ec       carDynGravel               004d66ec   cardata.obj
 0001:000d5720       carDynWater                004d6720   cardata.obj
 0001:000d5754       carDynSpecial              004d6754   cardata.obj
 0001:000d5788       testdump_onoff             004d6788   DEBUG.obj
 0001:000d5788       int_time_disp              004d6788   DEBUG.obj
 0001:000d5788       testdump                   004d6788   DEBUG.obj
 0001:000d5790       _SuzuTexInit16             004d6790 f Fchatex.obj
 0001:000d5890       _SetPolygonDDInit16        004d6890 f Fchatex.obj
 0001:000d58c0       _Texture16                 004d68c0 f Fchatex.obj
 0001:000d7b70       record_change              004d8b70   REC_CHANGE.obj
 0001:000d8064       adv_recordact_init         004d9064   REC_CHANGE.obj
 0001:000d8139       adv_recordact              004d9139   REC_CHANGE.obj
 0001:000d85b0       title_init_watanabe        004d95b0   TITLEwatanabe.obj
 0001:000d8ea0       title_init_next            004d9ea0   NEXT.obj
 0001:000d9056       game_main_xxx              004da056   NEXT.obj
 0001:000d947c       record_RTxx                004da47c   REC_RTXX.obj
 0001:000d9898       c_select_init              004da898   AC_C_SELECT.obj
 0001:000d9c0e       c_select_main              004dac0e   AC_C_SELECT.obj
 0001:000da08f       c_white_in                 004db08f   AC_C_SELECT.obj
 0001:000da14f       set_car_ablity             004db14f   AC_C_SELECT.obj
 0001:000da251       c_check_pad                004db251   AC_C_SELECT.obj
 0001:000dcb00       set_scr_int                004ddb00   scroll.obj
 0001:000dcb1c       init_scr_int               004ddb1c   scroll.obj
 0001:000dcb38       set_mov_scr                004ddb38   scroll.obj
 0001:000dcb3c       set_mov_scri               004ddb3c   scroll.obj
 0001:000dcb40       init_mov_scri              004ddb40   scroll.obj
 0001:000dcb7c       set_window_scr             004ddb7c   scroll.obj
 0001:000dcb80       set_window_scri            004ddb80   scroll.obj
 0001:000dcb84       init_window_scri           004ddb84   scroll.obj
 0001:000dcb88       init_gscroll               004ddb88   scroll.obj
 0001:000dcb90       init_oscroll               004ddb90   scroll.obj
 0001:000dcb94       init_rscroll               004ddb94   scroll.obj
 0001:000dcb98       init_coef_tbl              004ddb98   scroll.obj
 0001:000dcb9c       set_grpara                 004ddb9c   scroll.obj
 0001:000dcba6       set_grpara2                004ddba6   scroll.obj
 0001:000dcc68       clr_hscr_rr                004ddc68   scroll.obj
 0001:000dccb4       set_tp_rr                  004ddcb4   scroll.obj
 0001:000dccf0       set_grpara3                004ddcf0   scroll.obj
 0001:000dcd54       set_grpara_int             004ddd54   scroll.obj
 0001:000dcd74       set_grpara_com             004ddd74   scroll.obj
 0001:000dce68       set_grpara_int2p           004dde68   scroll.obj
 0001:000dcea0       set_rpara_int              004ddea0   scroll.obj
 0001:000dd098       init_rpara_int             004de098   scroll.obj
 0001:000dd0f4       m_reserve                  004de0f4   ERROR.obj
 0001:000dd0f6       m_inst_err                 004de0f6   ERROR.obj
 0001:000dd0f8       m_slot_err                 004de0f8   ERROR.obj
 0001:000dd0fa       m_addr_err                 004de0fa   ERROR.obj
 0001:000dd0fc       m_dma_err                  004de0fc   ERROR.obj
 0001:000dd0fe       m_nmi_int                  004de0fe   ERROR.obj
 0001:000dd100       m_userbreak_int            004de100   ERROR.obj
 0001:000dd102       m_trap                     004de102   ERROR.obj
 0001:000dd104       m_irl                      004de104   ERROR.obj
 0001:000dd106       s_reserve                  004de106   ERROR.obj
 0001:000dd11a       s_inst_err                 004de11a   ERROR.obj
 0001:000dd12b       s_slot_err                 004de12b   ERROR.obj
 0001:000dd13c       s_addr_err                 004de13c   ERROR.obj
 0001:000dd14d       s_dma_err                  004de14d   ERROR.obj
 0001:000dd15e       s_nmi_int                  004de15e   ERROR.obj
 0001:000dd16f       s_userbreak_int            004de16f   ERROR.obj
 0001:000dd180       s_trap                     004de180   ERROR.obj
 0001:000dd191       s_irl                      004de191   ERROR.obj
 0001:000dd1a2       s_error                    004de1a2   ERROR.obj
 0001:000dd1ac       push_all_register          004de1ac   ERROR.obj
 0001:000dd207       set_error_vector           004de207   ERROR.obj
 0001:000dd26c       master_error_vector        004de26c   ERROR.obj
 0001:000dd290       slave_error_vector         004de290   ERROR.obj
 0001:000dd2b4       set_error_msg              004de2b4   ERROR.obj
 0001:000dd2fc       InitHeli                   004de2fc   HELI.obj
 0001:000dd4ab       EvHelicopter               004de4ab   HELI.obj
 0001:000dd7a6       HeliMain                   004de7a6   HELI.obj
 0001:000de424       HeliDrive                  004df424   HELI.obj
 0001:000deede       MakeSandStorm              004dfede   HELI.obj
 0001:000df14c       SandStorm                  004e014c   HELI.obj
 0001:000df382       HeliSE                     004e0382   HELI.obj
 0001:000df568       bpe_expand                 004e0568   EXTRACT.obj
 0001:000dfac0       _Set_PC_Pad_type           004e0ac0 f Keyctrl.obj
 0001:000dfaf0       _InitKeyboard              004e0af0 f Keyctrl.obj
 0001:000dfb70       _PageUpDown                004e0b70 f Keyctrl.obj
 0001:000dfbb0       _GetConfigKey_Joy          004e0bb0 f Keyctrl.obj
 0001:000dfd00       _GetConfigKey              004e0d00 f Keyctrl.obj
 0001:000dfd30       _IsSelectProc              004e0d30 f Keyctrl.obj
 0001:000dfd50       _SwKeyboard                004e0d50 f Keyctrl.obj
 0001:000e0400       _MakeRestartCommand        004e1400 f Keyctrl.obj
 0001:000e0460       _SwRead                    004e1460 f Keyctrl.obj
 0001:000e0720       lap_time_init              004e1720   LAPTIME.obj
 0001:000e17d0       extend_time_calc           004e27d0   LAPTIME.obj
 0001:000e18e4       lag_time_calc              004e28e4   LAPTIME.obj
 0001:000e1bf4       check_lap                  004e2bf4   LAPTIME.obj
 0001:000e3d1c       clrtime_startlag2p         004e4d1c   LAPTIME.obj
 0001:000e3e14       lap_myline                 004e4e14   LAPTIME.obj
 0001:000e41a4       time_cmp_save              004e51a4   LAPTIME.obj
 0001:000e4510       time_cmp_save2p            004e5510   LAPTIME.obj
 0001:000e46d8       time_cmpst_save            004e56d8   LAPTIME.obj
 0001:000e46f0       time_cmpgl_save            004e56f0   LAPTIME.obj
 0001:000e499c       time_cmp                   004e599c   LAPTIME.obj
 0001:000e4bc8       lap_time_calc2p            004e5bc8   LAPTIME.obj
 0001:000e4bd4       lap_time_calc              004e5bd4   LAPTIME.obj
 0001:000e4bde       lap_time_calcs             004e5bde   LAPTIME.obj
 0001:000e4dd8       total_time_calc            004e5dd8   LAPTIME.obj
 0001:000e538c       total_time_calc_all        004e638c   LAPTIME.obj
 0001:000e56d4       time_adjustst              004e66d4   LAPTIME.obj
 0001:000e5a58       time_adjust                004e6a58   LAPTIME.obj
 0001:000e5e18       time_adjustst2p            004e6e18   LAPTIME.obj
 0001:000e60ac       vstime_cmp                 004e70ac   LAPTIME.obj
 0001:000e687c       game_end_chk               004e787c   LAPTIME.obj
 0001:000e6988       swclear                    004e7988   SWITCH.obj
 0001:000e6a80       swclear1p                  004e7a80   SWITCH.obj
 0001:000e6b08       swclear2p                  004e7b08   SWITCH.obj
 0001:000e6bac       pad_read                   004e7bac   SWITCH.obj
 0001:000e7067       no_connect                 004e8067   SWITCH.obj
 0001:000e70d4       read_sub                   004e80d4   SWITCH.obj
 0001:000e718e       sw_reset                   004e818e   SWITCH.obj
 0001:000e7238       slave_start                004e8238   SLAVE.obj
 0001:000e7239       initial_slave              004e8239   SLAVE.obj
 0001:000e723c       set_slave_exec             004e823c   SLAVE.obj
 0001:000e7380       wait_slave_end             004e8380   SLAVE.obj
 0001:000e7384       set_pict_setting           004e8384   CS_SETTING_PSET.obj
 0001:000e7680       delete_cslay0              004e8680   CS_SETTING_PSET.obj
 0001:000e7794       cs_chg_color_bg            004e8794   CS_SETTING_PSET.obj
 0001:000e78bc       cs_map_set_lay0            004e88bc   CS_SETTING_PSET.obj
 0001:000e7a78       cs_map_chg                 004e8a78   CS_SETTING_PSET.obj
 0001:000e7c20       cs_plane_chg               004e8c20   CS_SETTING_PSET.obj
 0001:000e7cec       set_button_pict            004e8cec   CS_SETTING_PSET.obj
 0001:000e8134       cs_color_chg_init          004e9134   CS_SETTING_PSET.obj
 0001:000e81ea       cs_color_chg               004e91ea   CS_SETTING_PSET.obj
 0001:000e839c       cs_pict_bright             004e939c   CS_SETTING_PSET.obj
 0001:000e8758       cs_pict_stop               004e9758   CS_SETTING_PSET.obj
 0001:000e87b4       cs_pict_dark               004e97b4   CS_SETTING_PSET.obj
 0001:000e880b       cs_pict_bright_cslay3      004e980b   CS_SETTING_PSET.obj
 0001:000e8ae8       setcoloffset               004e9ae8   CLROFFSET.obj
 0001:000e8bdb       inccoloffset               004e9bdb   CLROFFSET.obj
 0001:000e8d19       white_in                   004e9d19   CLROFFSET.obj
 0001:000e8e9f       sl_white_out               004e9e9f   CLROFFSET.obj
 0001:000e8f4f       pre_fade_inout             004e9f4f   CLROFFSET.obj
 0001:000e8fdb       fade_inout_init            004e9fdb   CLROFFSET.obj
 0001:000e917c       fade_inout_work            004ea17c   CLROFFSET.obj
 0001:000e9684       game_se_set                004ea684   GAMESD.obj
 0001:000e9a8e       game_se_set2p_net          004eaa8e   GAMESD.obj
 0001:000e9ac0       game_se_set2p              004eaac0   GAMESD.obj
 0001:000e9f10       crash_sd                   004eaf10   GAMESD.obj
 0001:000ea6ac       slip_sd                    004eb6ac   GAMESD.obj
 0001:000ea8b0       slip_jump                  004eb8b0   GAMESD.obj
 0001:000eafac       stone_attack_sd            004ebfac   GAMESD.obj
 0001:000eb1cc       road_noise_sd              004ec1cc   GAMESD.obj
 0001:000eb390       set_road_noise             004ec390   GAMESD.obj
 0001:000eb594       road_noise_fpsd            004ec594   GAMESD.obj
 0001:000eb7f0       road_noise2p_sd            004ec7f0   GAMESD.obj
 0001:000eb9d4       kansei_se_set              004ec9d4   GAMESD.obj
 0001:000eba2c       init_game_se               004eca2c   GAMESD.obj
 0001:000ebc34       replay_sdctrl              004ecc34   GAMESD.obj
 0001:000ebf00       game_init                  004ecf00   GAME.obj
 0001:000ebf00       __game_init                004ecf00   GAME.obj
 0001:000ec1a4       poly_game_init             004ed1a4   GAME.obj
 0001:000ec224       s_poly_game_init           004ed224   GAME.obj
 0001:000ec228       poly_vs_init               004ed228   GAME.obj
 0001:000ec330       game_init_sub              004ed330   GAME.obj
 0001:000ec56c       ginit_vs                   004ed56c   GAME.obj
 0001:000ec6a4       game_main2p                004ed6a4   GAME.obj
 0001:000ec798       game_main                  004ed798   GAME.obj
 0001:000ec8a4       game_main_ecom             004ed8a4   GAME.obj
 0001:000ed16c       pause_init                 004ee16c   GAME.obj
 0001:000ed1d0       pause                      004ee1d0   GAME.obj
 0001:000ed648       pause_end                  004ee648   GAME.obj
 0001:000ed6ac       restart_init               004ee6ac   GAME.obj
 0001:000ed74c       restart_wait               004ee74c   GAME.obj
 0001:000ed7e4       record_main                004ee7e4   REC_MAIN.obj
 0001:000ed7e4       __record_main              004ee7e4   REC_MAIN.obj
 0001:000ee065       RECORD_CG_SET              004ef065   REC_MAIN.obj
 0001:000eefd8       _cg_set                    004effd8   REC_MAIN.obj
 0001:000ef09b       _map_set                   004f009b   REC_MAIN.obj
 0001:000ef15e       map_set                    004f015e   REC_MAIN.obj
 0001:000ef1f8       _pal_set                   004f01f8   REC_MAIN.obj
 0001:000ef2ad       vdp2_set_w                 004f02ad   REC_MAIN.obj
 0001:000ef322       record_pict_init2          004f0322   REC_MAIN.obj
 0001:000ef339       record_pict_init           004f0339   REC_MAIN.obj
 0001:000ef50c       record_sel_init            004f050c   REC_MAIN.obj
 0001:000ef5a9       key_repeat_init            004f05a9   REC_MAIN.obj
 0001:000ef62b       key_repeat                 004f062b   REC_MAIN.obj
 0001:000ef836       REPLAY_INIT2               004f0836   REC_MAIN.obj
 0001:000efd80       execCar                    004f0d80   PLAYER.obj
 0001:000f0424       speed_limit                004f1424   PLAYER.obj
 0001:000f05f0       regular_xyzang             004f15f0   PLAYER.obj
 0001:000f06e8       calc_run_R                 004f16e8   PLAYER.obj
 0001:000f0b18       calc_new_vang              004f1b18   PLAYER.obj
 0001:000f0f10       hit_course_dir             004f1f10   PLAYER.obj
 0001:000f10ac       over_xyzang_limit          004f20ac   PLAYER.obj
 0001:000f1634       calc_tire_spd              004f2634   PLAYER.obj
 0001:000f193c       calc_xyzang_froad          004f293c   PLAYER.obj
 0001:000f2138       calc_tire_move             004f3138   PLAYER.obj
 0001:000f2574       wheelproc                  004f3574   PLAYER.obj
 0001:000f2f54       tire_fr_vect               004f3f54   PLAYER.obj
 0001:000f33c4       calc_tire_posi             004f43c4   PLAYER.obj
 0001:000f365c       coli_body                  004f465c   PLAYER.obj
 0001:000f3c2c       calc_hit_body              004f4c2c   PLAYER.obj
 0001:000f3fc8       coli_force                 004f4fc8   PLAYER.obj
 0001:000f46a4       vs_g_ctrl                  004f56a4   PLAYER.obj
 0001:000f48e8       goal_car_move              004f58e8   PLAYER.obj
 0001:000f48f2       goal_car_move2p            004f58f2   PLAYER.obj
 0001:000f4b24       init_sound                 004f5b24   SOUND.obj
 0001:000f4b28       sd_chg_driver              004f5b28   SOUND.obj
 0001:000f4b2c       sd_map_chg                 004f5b2c   SOUND.obj
 0001:000f4b58       sd_cmd_wait                004f5b58   SOUND.obj
 0001:000f4b5c       sd_map_chg_g               004f5b5c   SOUND.obj
 0001:000f4b84       sd_seq_end_chk             004f5b84   SOUND.obj
 0001:000f4b88       sd_se_end_chk              004f5b88   SOUND.obj
 0001:000f4b94       sd_cmd_set                 004f5b94   SOUND.obj
 0001:000f4b98       sd_seq_stop_set            004f5b98   SOUND.obj
 0001:000f4bc0       sd_seq_stop2_set           004f5bc0   SOUND.obj
 0001:000f4be8       sd_seq_vol_set             004f5be8   SOUND.obj
 0001:000f4c10       sd_midi_direct_set         004f5c10   SOUND.obj
 0001:000f4c14       sd_midi_direct_setv        004f5c14   SOUND.obj
 0001:000f4c19       sd_cmd_host_sets           004f5c19   SOUND.obj
 0001:000f4c1c       sd_da_vol_set              004f5c1c   SOUND.obj
 0001:000f4c20       sd_tol_vol_set             004f5c20   SOUND.obj
 0001:000f4c48       sd_se_set                  004f5c48   SOUND.obj
 0001:000f4cd0       sd_se_host_set             004f5cd0   SOUND.obj
 0001:000f4cd1       sd_se_host_sets            004f5cd1   SOUND.obj
 0001:000f4cd4       sd_qs_set                  004f5cd4   SOUND.obj
 0001:000f4cd8       init_pcm_player            004f5cd8   SOUND.obj
 0001:000f4cdc       set_pcm_player             004f5cdc   SOUND.obj
 0001:000f4ce0       pcm_player                 004f5ce0   SOUND.obj
 0001:000f4ce8       pcmp_init                  004f5ce8   SOUND.obj
 0001:000f4cec       pcmp_copy                  004f5cec   SOUND.obj
 0001:000f4d74       da_fade_init               004f5d74   SOUND.obj
 0001:000f4d78       da_fade_init2              004f5d78   SOUND.obj
 0001:000f4d7c       tol_fade_init              004f5d7c   SOUND.obj
 0001:000f4d80       da_fade_out                004f5d80   SOUND.obj
 0001:000f4d84       tol_fade_out               004f5d84   SOUND.obj
 0001:000f4d88       set_seq_sound              004f5d88   SOUND.obj
 0001:000f4db0       init_game_sound            004f5db0   SOUND.obj
 0001:000f4dbc       set_seq_pause_stop         004f5dbc   SOUND.obj
 0001:000f4e70       set_seq_pause_cont         004f5e70   SOUND.obj
 0001:000f4efc       sd_soft_res                004f5efc   SOUND.obj
 0001:000f4f0c       engine_off                 004f5f0c   SOUND.obj
 0001:000f4f58       engine_wait                004f5f58   SOUND.obj
 0001:000f4fac       set_sound                  004f5fac   SOUND.obj
 0001:000f4fb0       set_game_sound             004f5fb0   SOUND.obj
 0001:000f4fb0       seq_player                 004f5fb0   SOUND.obj
 0001:000f4fb4       set_game_sound_wait        004f5fb4   SOUND.obj
 0001:000f4fb4       seq_player_wait            004f5fb4   SOUND.obj
 0001:000f4fb8       init_replay_sound          004f5fb8   SOUND.obj
 0001:000f4fd4       replay_hyouka              004f5fd4   SOUND.obj
 0001:000f4fd8       disp_car_main_setting1     004f5fd8   CS_MD_SELECT.obj
 0001:000f506f       disp_car_main_setting2     004f606f   CS_MD_SELECT.obj
 0001:000f521e       disp_obj_main_setting      004f621e   CS_MD_SELECT.obj
 0001:000f5386       disp_car_main_battle2p     004f6386   CS_MD_SELECT.obj
 0001:000f55a9       disp_course_main_battle2p  004f65a9   CS_MD_SELECT.obj
 0001:000f570d       disp_car_main_timeattack   004f670d   CS_MD_SELECT.obj
 0001:000f58b8       disp_course_main_timeattack 004f68b8   CS_MD_SELECT.obj
 0001:000f5a20       color_change_init          004f6a20   CS_MD_SELECT.obj
 0001:000f5a6a       color_change_main          004f6a6a   CS_MD_SELECT.obj
 0001:000f5c06       slt_mode_init              004f6c06   CS_MD_SELECT.obj
 0001:000f64e0       slt_mode_main              004f74e0   CS_MD_SELECT.obj
 0001:000f6a7c       set_strlake                004f7a7c   CS_MD_SELECT.obj
 0001:000f6ae7       set_stratos                004f7ae7   CS_MD_SELECT.obj
 0001:000f6c3e       white_in_md                004f7c3e   CS_MD_SELECT.obj
 0001:000f6cfe       md_cansel                  004f7cfe   CS_MD_SELECT.obj
 0001:000f6d65       pad_check_md               004f7d65   CS_MD_SELECT.obj
 0001:000f7404       check_cursor_posi          004f8404   CS_MD_SELECT.obj
 0001:000f7460       check_cursor_posi2         004f8460   CS_MD_SELECT.obj
 0001:000f754c       win_set                    004f854c   CS_MD_SELECT.obj
 0001:000f791c       pict_set_next_md           004f891c   CS_MD_SELECT.obj
 0001:000f7a88       scrl_v_move_init           004f8a88   CS_MD_SELECT.obj
 0001:000f7b3f       diff_vect_move             004f8b3f   CS_MD_SELECT.obj
 0001:000f7e61       diff_vect_move1            004f8e61   CS_MD_SELECT.obj
 0001:000f80f4       diff_vect_move2            004f90f4   CS_MD_SELECT.obj
 0001:000f83e4       scrl_v_move                004f93e4   CS_MD_SELECT.obj
 0001:000f86f3       move_nbg0                  004f96f3   CS_MD_SELECT.obj
 0001:000f886d       time_cnt                   004f986d   CS_MD_SELECT.obj
 0001:000f88d9       delete_nbg0                004f98d9   CS_MD_SELECT.obj
 0001:000f8936       judge_disp_car             004f9936   CS_MD_SELECT.obj
 0001:000f8a35       judge_disp_car_bt          004f9a35   CS_MD_SELECT.obj
 0001:000f97a0       EvZebra                    004fa7a0   ANIMAL.obj
 0001:000f9874       ZebraMain                  004fa874   ANIMAL.obj
 0001:000f9c07       ZebraCrazy                 004fac07   ANIMAL.obj
 0001:000f9c14       EvOstrich                  004fac14   ANIMAL.obj
 0001:000f9c43       OstrichMain                004fac43   ANIMAL.obj
 0001:000f9d2a       EvBird1                    004fad2a   ANIMAL.obj
 0001:000f9e57       Bird1Main                  004fae57   ANIMAL.obj
 0001:000f9faf       bird1_walk                 004fafaf   ANIMAL.obj
 0001:000fa0ce       bird1_sae                  004fb0ce   ANIMAL.obj
 0001:000fa19a       bird1_fly                  004fb19a   ANIMAL.obj
 0001:000fa2e1       NearCar                    004fb2e1   ANIMAL.obj
 0001:000fa47c       EvBird2                    004fb47c   ANIMAL.obj
 0001:000fa5c1       Bird2Main                  004fb5c1   ANIMAL.obj
 0001:000fa7f6       EvElephant                 004fb7f6   ANIMAL.obj
 0001:000fa894       ElephantMain               004fb894   ANIMAL.obj
 0001:000fa9e3       EvSwan                     004fb9e3   ANIMAL.obj
 0001:000faa84       SwanMain                   004fba84   ANIMAL.obj
 0001:000fabfc       move_animal                004fbbfc   ANIMAL.obj
 0001:000faf90       record_R                   004fbf90   REC_R.obj
 0001:000fb347       CHANGE_SUB                 004fc347   REC_R.obj
 0001:000fb515       R_SCR_SUB                  004fc515   REC_R.obj
 0001:000fb617       rec_menu_scrR              004fc617   REC_R.obj
 0001:000fb6b8       rec_menu_scrL              004fc6b8   REC_R.obj
 0001:000fb6c7       rec_menu_scrRd             004fc6c7   REC_R.obj
 0001:000fb6f9       rec_menu_scrLd             004fc6f9   REC_R.obj
 0001:000fb728       rec_pad_sound              004fc728   REC_R.obj
 0001:000fb798       photoctrlinit              004fc798   PHOTOCTRL.obj
 0001:000fb7f2       photoExec                  004fc7f2   PHOTOCTRL.obj
 0001:000fb883       photo_move                 004fc883   PHOTOCTRL.obj
 0001:000fbaf2       photo_stop                 004fcaf2   PHOTOCTRL.obj
 0001:000fbbec       photo_break                004fcbec   PHOTOCTRL.obj
 0001:000fbcde       photoFrmCtrl               004fccde   PHOTOCTRL.obj
 0001:000fbdd1       calc_tblptr                004fcdd1   PHOTOCTRL.obj
 0001:000fbe99       photo_end                  004fce99   PHOTOCTRL.obj
 0001:000fbec6       _LZClose@4                 004fcec6 f lz32:LZ32.dll
 0001:000fbecc       _LZRead@12                 004fcecc f lz32:LZ32.dll
 0001:000fbed2       _LZSeek@12                 004fced2 f lz32:LZ32.dll
 0001:000fbed8       _LZOpenFileA@12            004fced8 f lz32:LZ32.dll
 0001:000fbede       _DirectDrawCreate@12       004fcede f ddraw:DDRAW.dll
 0001:000fbee4       _DirectSoundCreate@12      004fcee4 f dsound:DSOUND.dll
 0001:000fbeea       _DirectPlayCreate@12       004fceea f dplayx:DPLAYX.dll
 0001:000fbef0       _DirectPlayEnumerateA@8    004fcef0 f dplayx:DPLAYX.dll
 0001:000fbef8       __ftol                     004fcef8 f LIBC:ftol.obj
 0001:000fbf20       _fdiv_main_routine         004fcf20 f LIBC:adj_fdiv.obj
 0001:000fc037       __adj_fdiv_r               004fd037 f LIBC:adj_fdiv.obj
 0001:000fc4d6       __fdivp_sti_st             004fd4d6 f LIBC:adj_fdiv.obj
 0001:000fc4e9       __fdivrp_sti_st            004fd4e9 f LIBC:adj_fdiv.obj
 0001:000fc4fc       __adj_fdiv_m32             004fd4fc f LIBC:adj_fdiv.obj
 0001:000fc548       __adj_fdiv_m64             004fd548 f LIBC:adj_fdiv.obj
 0001:000fc594       __adj_fdiv_m16i            004fd594 f LIBC:adj_fdiv.obj
 0001:000fc5c8       __adj_fdiv_m32i            004fd5c8 f LIBC:adj_fdiv.obj
 0001:000fc5fc       __adj_fdivr_m32            004fd5fc f LIBC:adj_fdiv.obj
 0001:000fc648       __adj_fdivr_m64            004fd648 f LIBC:adj_fdiv.obj
 0001:000fc694       __adj_fdivr_m16i           004fd694 f LIBC:adj_fdiv.obj
 0001:000fc6c8       __adj_fdivr_m32i           004fd6c8 f LIBC:adj_fdiv.obj
 0001:000fc6fc       __safe_fdiv                004fd6fc f LIBC:adj_fdiv.obj
 0001:000fc711       __safe_fdivr               004fd711 f LIBC:adj_fdiv.obj
 0001:000fc726       __fprem_common             004fd726 f LIBC:adj_fdiv.obj
 0001:000fc92c       __adj_fprem                004fd92c f LIBC:adj_fdiv.obj
 0001:000fc9de       __fprem1_common            004fd9de f LIBC:adj_fdiv.obj
 0001:000fcbe4       __adj_fprem1               004fdbe4 f LIBC:adj_fdiv.obj
 0001:000fcc99       __safe_fprem               004fdc99 f LIBC:adj_fdiv.obj
 0001:000fcc9f       __safe_fprem1              004fdc9f f LIBC:adj_fdiv.obj
 0001:000fcca5       __adj_fpatan               004fdca5 f LIBC:adj_fdiv.obj
 0001:000fcca8       __adj_fptan                004fdca8 f LIBC:adj_fdiv.obj
 0001:000fccb0       __fpmath                   004fdcb0 f LIBC:fpinit.obj
 0001:000fccd0       __fpclear                  004fdcd0 f LIBC:fpinit.obj
 0001:000fcce0       __cfltcvt_init             004fdce0 f LIBC:fpinit.obj
 0001:000fcd20       _fclose                    004fdd20 f LIBC:fclose.obj
 0001:000fcd90       _fread                     004fdd90 f LIBC:fread.obj
 0001:000fcee0       __fsopen                   004fdee0 f LIBC:fopen.obj
 0001:000fcf10       _fopen                     004fdf10 f LIBC:fopen.obj
 0001:000fcf30       __cinit                    004fdf30 f LIBC:crt0dat.obj
 0001:000fcf60       _exit                      004fdf60 f LIBC:crt0dat.obj
 0001:000fcf80       __exit                     004fdf80 f LIBC:crt0dat.obj
 0001:000fd040       _fprintf                   004fe040 f LIBC:fprintf.obj
 0001:000fd080       _sin                       004fe080 f LIBC:87ctrig.obj
 0001:000fd08a       _cos                       004fe08a f LIBC:87ctrig.obj
 0001:000fd091       _tan                       004fe091 f LIBC:87ctrig.obj
 0001:000fd098       __CIsin                    004fe098 f LIBC:87ctrig.obj
 0001:000fd0a2       __CIcos                    004fe0a2 f LIBC:87ctrig.obj
 0001:000fd0a9       __CItan                    004fe0a9 f LIBC:87ctrig.obj
 0001:000fd0b0       _strncpy                   004fe0b0 f LIBC:strncpy.obj
 0001:000fd0e0       ??3@YAXPAX@Z               004fe0e0 f LIBC:delete.obj
 0001:000fd0f0       ??2@YAPAXI@Z               004fe0f0 f LIBC:new.obj
 0001:000fd100       _toupper                   004fe100 f LIBC:toupper.obj
 0001:000fd1e8       __global_unwind2           004fe1e8 f LIBC:exsup.obj
 0001:000fd22a       __local_unwind2            004fe22a f LIBC:exsup.obj
 0001:000fd282       __NLG_Return2              004fe282   LIBC:exsup.obj
 0001:000fd292       __abnormal_termination     004fe292 f LIBC:exsup.obj
 0001:000fd2b5       __NLG_Notify1              004fe2b5 f LIBC:exsup.obj
 0001:000fd2be       __NLG_Notify               004fe2be f LIBC:exsup.obj
 0001:000fd2d1       __NLG_Dispatch             004fe2d1   LIBC:exsup.obj
 0001:000fd2e0       ?_JumpToContinuation@@YGXPAXPAUEHRegistrationNode@@@Z 004fe2e0 f LIBC:trnsctrl.obj
 0001:000fd320       ?_CallMemberFunction0@@YGXPAX0@Z 004fe320 f LIBC:trnsctrl.obj
 0001:000fd330       ?_CallMemberFunction1@@YGXPAX00@Z 004fe330 f LIBC:trnsctrl.obj
 0001:000fd340       ?_CallMemberFunction2@@YGXPAX00H@Z 004fe340 f LIBC:trnsctrl.obj
 0001:000fd350       ?_UnwindNestedFrames@@YGXPAUEHRegistrationNode@@PAUEHExceptionRecord@@@Z 004fe350 f LIBC:trnsctrl.obj
 0001:000fd3b0       ___CxxFrameHandler         004fe3b0 f LIBC:trnsctrl.obj
 0001:000fd3f0       ?_CallCatchBlock2@@YAPAXPAUEHRegistrationNode@@PBU_s_FuncInfo@@PAXHK@Z 004fe3f0 f LIBC:trnsctrl.obj
 0001:000fd490       ?_CallSETranslator@@YAHPAUEHExceptionRecord@@PAUEHRegistrationNode@@PAX2PBU_s_FuncInfo@@H1@Z 004fe490 f LIBC:trnsctrl.obj
 0001:000fd5e0       _WinMainCRTStartup         004fe5e0 f LIBC:wincrt0.obj
 0001:000fd770       __amsg_exit                004fe770 f LIBC:wincrt0.obj
 0001:000fd7a0       __setdefaultprecision      004fe7a0 f LIBC:fp8.obj
 0001:000fd7c0       __ms_p5_test_fdiv          004fe7c0 f LIBC:testfdiv.obj
 0001:000fd810       __ms_p5_mp_test_fdiv       004fe810 f LIBC:testfdiv.obj
 0001:000fd930       __forcdecpt                004fe930 f LIBC:cvt.obj
 0001:000fd9a0       __cropzeros                004fe9a0 f LIBC:cvt.obj
 0001:000fda00       __positive                 004fea00 f LIBC:cvt.obj
 0001:000fda20       __fassign                  004fea20 f LIBC:cvt.obj
 0001:000fda70       __cftoe                    004fea70 f LIBC:cvt.obj
 0001:000fdbb0       __cftof                    004febb0 f LIBC:cvt.obj
 0001:000fdcb0       __cftog                    004fecb0 f LIBC:cvt.obj
 0001:000fddc0       __cfltcvt                  004fedc0 f LIBC:cvt.obj
 0001:000fde60       _free                      004fee60 f LIBC:free.obj
 0001:000fde80       __close                    004fee80 f LIBC:close.obj
 0001:000fdf50       __freebuf                  004fef50 f LIBC:_freebuf.obj
 0001:000fdf90       _fflush                    004fef90 f LIBC:fflush.obj
 0001:000fdfe0       __flush                    004fefe0 f LIBC:fflush.obj
 0001:000fe050       __flushall                 004ff050 f LIBC:fflush.obj
 0001:000fe0d0       __filbuf                   004ff0d0 f LIBC:_filbuf.obj
 0001:000fe1c0       __read                     004ff1c0 f LIBC:read.obj
 0001:000fe430       __openfile                 004ff430 f LIBC:_open.obj
 0001:000fe640       __getstream                004ff640 f LIBC:stream.obj
 0001:000fe6c0       __stbuf                    004ff6c0 f LIBC:_sftbuf.obj
 0001:000fe760       __ftbuf                    004ff760 f LIBC:_sftbuf.obj
 0001:000fe7b0       __output                   004ff7b0 f LIBC:output.obj
 0001:000ff2a0       __fFCOS                    005002a0   LIBC:87trig.obj
 0001:000ff2aa       __fFSIN                    005002aa   LIBC:87trig.obj
 0001:000ff2d0       __cintrindisp2             005002d0 f LIBC:87cdisp.obj
 0001:000ff30e       __cintrindisp1             0050030e f LIBC:87cdisp.obj
 0001:000ff344       __ctrandisp2               00500344 f LIBC:87cdisp.obj
 0001:000ff4b5       __ctrandisp1               005004b5 f LIBC:87cdisp.obj
 0001:000ff4e1       __fload                    005004e1 f LIBC:87cdisp.obj
 0001:000ff520       _malloc                    00500520 f LIBC:malloc.obj
 0001:000ff540       __nh_malloc                00500540 f LIBC:malloc.obj
 0001:000ff580       __heap_alloc               00500580 f LIBC:malloc.obj
 0001:000ff5a0       ___crtLCMapStringA         005005a0 f LIBC:aw_map.obj
 0001:000ff800       __isctype                  00500800 f LIBC:isctype.obj
 0001:000ff8a0       ___InternalCxxFrameHandler 005008a0 f LIBC:frame.obj
 0001:000ffd80       ___FrameUnwindToState      00500d80 f LIBC:frame.obj
 0001:00100300       __CallSettingFrame@12      00501300 f LIBC:lowhelpr.obj
 0001:00100325       __NLG_Return               00501325   LIBC:lowhelpr.obj
 0001:00100350       ?terminate@@YAXXZ          00501350 f LIBC:hooks.obj
 0001:001003d0       ?_inconsistency@@YAXXZ     005013d0 f LIBC:hooks.obj
 0001:00100450       __XcptFilter               00501450 f LIBC:winxfltr.obj
 0001:001005e0       __ismbblead                005015e0 f LIBC:ismbbyte.obj
 0001:00100640       __setenvp                  00501640 f LIBC:stdenvp.obj
 0001:00100720       __setargv                  00501720 f LIBC:stdargv.obj
 0001:001009a0       ___crtGetEnvironmentStringsA 005019a0 f LIBC:aw_env.obj
 0001:00100b40       __setmbcp                  00501b40 f LIBC:mbctype.obj
 0001:00100e00       ___initmbctable            00501e00 f LIBC:mbctype.obj
 0001:00100e10       __ioinit                   00501e10 f LIBC:ioinit.obj
 0001:00100ff0       __heap_init                00501ff0 f LIBC:heapinit.obj
 0001:00101010       __except_handler3          00502010 f LIBC:exsup3.obj
 0001:001010cd       __seh_longjmp_unwind@4     005020cd f LIBC:exsup3.obj
 0001:001010f0       __FF_MSGBANNER             005020f0 f LIBC:crt0msg.obj
 0001:00101130       __NMSG_WRITE               00502130 f LIBC:crt0msg.obj
 0001:00101320       __control87                00502320 f LIBC:ieee87.obj
 0001:00101360       __controlfp                00502360 f LIBC:ieee87.obj
 0001:001014c0       __fptrap                   005024c0 f LIBC:crt0fp.obj
 0001:001014d0       _tolower                   005024d0 f LIBC:tolower.obj
 0001:001015c0       __ZeroTail                 005025c0 f LIBC:intrncvt.obj
 0001:00101630       __IncMan                   00502630 f LIBC:intrncvt.obj
 0001:001016a0       __RoundMan                 005026a0 f LIBC:intrncvt.obj
 0001:00101750       __CopyMan                  00502750 f LIBC:intrncvt.obj
 0001:00101770       __FillZeroMan              00502770 f LIBC:intrncvt.obj
 0001:00101780       __IsZeroMan                00502780 f LIBC:intrncvt.obj
 0001:001017a0       __ShrMan                   005027a0 f LIBC:intrncvt.obj
 0001:00101850       __ld12cvt                  00502850 f LIBC:intrncvt.obj
 0001:00101a20       __ld12tod                  00502a20 f LIBC:intrncvt.obj
 0001:00101a40       __ld12tof                  00502a40 f LIBC:intrncvt.obj
 0001:00101a60       __atodbl                   00502a60 f LIBC:intrncvt.obj
 0001:00101aa0       __atoflt                   00502aa0 f LIBC:intrncvt.obj
 0001:00101ae0       __fptostr                  00502ae0 f LIBC:_fptostr.obj
 0001:00101b70       __fltout                   00502b70 f LIBC:cfout.obj
 0001:00101be0       ___dtold                   00502be0 f LIBC:cfout.obj
 0001:00101ca0       _memmove                   00502ca0 f LIBC:memmove.obj
 0001:00101df0       __dosmaperr                00502df0 f LIBC:dosmap.obj
 0001:00101e60       __alloc_osfhnd             00502e60 f LIBC:osfinfo.obj
 0001:00101f20       __set_osfhnd               00502f20 f LIBC:osfinfo.obj
 0001:00101fd0       __free_osfhnd              00502fd0 f LIBC:osfinfo.obj
 0001:00102060       __get_osfhandle            00503060 f LIBC:osfinfo.obj
 0001:001020b0       __commit                   005030b0 f LIBC:commit.obj
 0001:00102120       __write                    00503120 f LIBC:write.obj
 0001:00102350       ___initstdio               00503350 f LIBC:_file.obj
 0001:00102420       ___endstdio                00503420 f LIBC:_file.obj
 0001:00102440       __getbuf                   00503440 f LIBC:_getbuf.obj
 0001:00102490       __lseek                    00503490 f LIBC:lseek.obj
 0001:00102550       __sopen                    00503550 f LIBC:open.obj
 0001:00102970       __isatty                   00503970 f LIBC:isatty.obj
 0001:001029a0       _wctomb                    005039a0 f LIBC:wctomb.obj
 0001:00102a40       __aulldiv                  00503a40 f LIBC:ulldiv.obj
 0001:00102ab0       __aullrem                  00503ab0 f LIBC:ullrem.obj
 0001:00102b30       __flsbuf                   00503b30 f LIBC:_flsbuf.obj
 0001:00102c80       __trandisp1                00503c80 f LIBC:87disp.obj
 0001:00102ce7       __trandisp2                00503ce7 f LIBC:87disp.obj
 0001:00102d73       __rttospopde               00503d73   LIBC:87disp.obj
 0001:00102d78       __rttospop                 00503d78   LIBC:87disp.obj
 0001:00102d7a       __rtnospop                 00503d7a   LIBC:87disp.obj
 0001:00102d7c       __rttosnpop                00503d7c   LIBC:87disp.obj
 0001:00102d7d       __rtnospopde               00503d7d   LIBC:87disp.obj
 0001:00102d84       __rtzeropop                00503d84   LIBC:87disp.obj
 0001:00102d86       __rtzeronpop               00503d86   LIBC:87disp.obj
 0001:00102d8b       __rtonepop                 00503d8b   LIBC:87disp.obj
 0001:00102d8d       __rtonenpop                00503d8d   LIBC:87disp.obj
 0001:00102d92       __tosnan1                  00503d92   LIBC:87disp.obj
 0001:00102dbd       __nosnan2                  00503dbd   LIBC:87disp.obj
 0001:00102dbf       __tosnan2                  00503dbf   LIBC:87disp.obj
 0001:00102de7       __nan2                     00503de7   LIBC:87disp.obj
 0001:00102e26       __rtindfpop                00503e26   LIBC:87disp.obj
 0001:00102e28       __rtindfnpop               00503e28   LIBC:87disp.obj
 0001:00102e39       __rttosnpopde              00503e39   LIBC:87disp.obj
 0001:00102e43       __rtchsifneg               00503e43   LIBC:87disp.obj
 0001:00102e61       __fFEXP                    00503e61   LIBC:87tran.obj
 0001:00102ec8       __rtinfpopse               00503ec8   LIBC:87tran.obj
 0001:00102eca       __rtinfnpopse              00503eca   LIBC:87tran.obj
 0001:00102eda       __fFLN                     00503eda   LIBC:87tran.obj
 0001:00102f8f       __rtinfpop                 00503f8f   LIBC:87tran.obj
 0001:00102f91       __rtinfnpop                00503f91   LIBC:87tran.obj
 0001:00102fae       __ffexpm1                  00503fae   LIBC:87tran.obj
 0001:00103060       __87except                 00504060 f LIBC:87except.obj
 0001:00103180       __callnewh                 00504180 f LIBC:handler.obj
 0001:001031b0       ___crtGetStringTypeA       005041b0 f LIBC:aw_str.obj
 0001:00103310       ?__CxxUnhandledExceptionFilter@@YGJPAU_EXCEPTION_POINTERS@@@Z 00504310 f LIBC:unhandld.obj
 0001:00103370       ?__CxxRestoreUnhandledExceptionFilter@@YAXXZ 00504370 f LIBC:unhandld.obj
 0001:00103380       ?_ValidateRead@@YAHPBXI@Z  00504380 f LIBC:validate.obj
 0001:001033a0       ?_ValidateWrite@@YAHPAXI@Z 005043a0 f LIBC:validate.obj
 0001:001033c0       ?_ValidateExecute@@YAHP6GHXZ@Z 005043c0 f LIBC:validate.obj
 0001:001033e0       _abort                     005043e0 f LIBC:abort.obj
 0001:00103400       ___crtMessageBoxA          00504400 f LIBC:crtmbox.obj
 0001:001034a0       ___addl                    005044a0 f LIBC:mantold.obj
 0001:001034d0       ___add_12                  005044d0 f LIBC:mantold.obj
 0001:00103540       ___shl_12                  00504540 f LIBC:mantold.obj
 0001:00103580       ___shr_12                  00504580 f LIBC:mantold.obj
 0001:001035c0       ___mtold12                 005045c0 f LIBC:mantold.obj
 0001:001036b0       ___strgtold12              005046b0 f LIBC:strgtold.obj
 0001:00103e00       _$I10_OUTPUT               00504e00 f LIBC:x10fout.obj
 0001:001041a0       _calloc                    005051a0 f LIBC:calloc.obj
 0001:00104200       __fcloseall                00505200 f LIBC:closeall.obj
 0001:00104280       __chsize                   00505280 f LIBC:chsize.obj
 0001:001043f0       __powhlp                   005053f0 f LIBC:powhlp.obj
 0001:00104640       __d_inttype                00505640 f LIBC:powhlp.obj
 0001:001046c0       __raise_exc                005056c0 f LIBC:fpexcept.obj
 0001:00104a30       __handle_exc               00505a30 f LIBC:fpexcept.obj
 0001:00104cf0       __set_errno                00505cf0 f LIBC:fpexcept.obj
 0001:00104d20       __matherr                  00505d20 f LIBC:matherr.obj
 0001:00104d30       __statfp                   00505d30 f LIBC:fpctrl.obj
 0001:00104d50       __clrfp                    00505d50 f LIBC:fpctrl.obj
 0001:00104d70       __ctrlfp                   00505d70 f LIBC:fpctrl.obj
 0001:00104db0       __set_statfp               00505db0 f LIBC:fpctrl.obj
 0001:00104e10       __onexit                   00505e10 f LIBC:onexit.obj
 0001:00104e90       _atexit                    00505e90 f LIBC:onexit.obj
 0001:00104eb0       ___onexitinit              00505eb0 f LIBC:onexit.obj
 0001:00104ef0       _raise                     00505ef0 f LIBC:winsig.obj
 0001:001050c0       ___ld12mul                 005060c0 f LIBC:tenpow.obj
 0001:00105370       ___multtenpow12            00506370 f LIBC:tenpow.obj
 0001:001053f0       __setmode                  005063f0 f LIBC:setmode.obj
 0001:00105470       __chkstk                   00506470   LIBC:chkstk.obj
 0001:00105470       __alloca_probe             00506470   LIBC:chkstk.obj
 0001:001054a0       __set_exp                  005064a0 f LIBC:util.obj
 0001:001054e0       __sptype                   005064e0 f LIBC:util.obj
 0001:00105550       __decomp                   00506550 f LIBC:util.obj
 0001:00105640       __frnd                     00506640 f LIBC:frnd.obj
 0001:00105660       __fpclass                  00506660 f LIBC:ieeemisc.obj
 0001:00105710       _strncat                   00506710 f LIBC:strncat.obj
 0001:00105750       _realloc                   00506750 f LIBC:realloc.obj
 0001:001057c0       __msize                    005067c0 f LIBC:msize.obj
 0001:001057d6       _RtlUnwind@16              005067d6 f kernel32:KERNEL32.dll
 0002:000000b8       _INI_DEVICE_NAME           005070b8   winapi.obj
 0002:000000c8       _INI_KEY_NAMES             005070c8   winapi.obj
 0002:00000114       _szInifile                 00507114   winapi.obj
 0002:00000130       _IID_IDirectPlay2          00507130   dpctrl.obj
 0002:00000140       _IID_IDirectPlay2A         00507140   dpctrl.obj
 0002:00000150       _IID_IDirectPlay           00507150   dpctrl.obj
 0002:00000160       _CLSID_DirectDraw          00507160   dpctrl.obj
 0002:00000170       _CLSID_DirectDrawClipper   00507170   dpctrl.obj
 0002:00000180       _IID_IDirectDraw           00507180   dpctrl.obj
 0002:00000190       _IID_IDirectDraw2          00507190   dpctrl.obj
 0002:000001a0       _IID_IDirectDrawSurface    005071a0   dpctrl.obj
 0002:000001b0       _IID_IDirectDrawSurface2   005071b0   dpctrl.obj
 0002:000001c0       _IID_IDirectDrawPalette    005071c0   dpctrl.obj
 0002:000001d0       _IID_IDirectDrawClipper    005071d0   dpctrl.obj
 0002:000001e0       _CLSID_DirectSound         005071e0   dpctrl.obj
 0002:000001f0       _IID_IDirectSound          005071f0   dpctrl.obj
 0002:00000200       _IID_IDirectSoundBuffer    00507200   dpctrl.obj
 0002:00000210       _IID_IDirectSound3DListener 00507210   dpctrl.obj
 0002:00000220       _IID_IDirectSound3DBuffer  00507220   dpctrl.obj
 0002:00000588       _inttbl                    00507588   mabiki.obj
 0002:00000598       _mabiki_tbl                00507598   mabiki.obj
 0002:000005b8       _mabiki_tbl_max            005075b8   mabiki.obj
 0002:00000640       ___lookuptable             00507640   LIBC:output.obj
 0003:00000000       ___xc_a                    00508000   LIBC:crt0init.obj
 0003:00000008       ___xc_z                    00508008   LIBC:crt0init.obj
 0003:0000000c       ___xi_a                    0050800c   LIBC:crt0init.obj
 0003:00000018       ___xi_z                    00508018   LIBC:crt0init.obj
 0003:0000001c       ___xp_a                    0050801c   LIBC:crt0init.obj
 0003:00000024       ___xp_z                    00508024   LIBC:crt0init.obj
 0003:00000028       ___xt_a                    00508028   LIBC:crt0init.obj
 0003:0000002c       ___xt_z                    0050802c   LIBC:crt0init.obj
 0003:00000030       _B_cli_desert              00508030   Mcdesert.obj
 0003:0002a698       _mcdesert                  00532698   Mcdesert.obj
 0003:0002e698       _scroll_list               00536698   NScroll.obj
 0003:0002e6d8       _select_mode               005366d8   NScroll.obj
 0003:0002e7e8       _select_game               005367e8   NScroll.obj
 0003:0002e950       _select_car                00536950   NScroll.obj
 0003:0002eb38       _select_cource             00536b38   NScroll.obj
 0003:0002ed30       _select_2p_battle          00536d30   NScroll.obj
 0003:0002f0b8       _cource_select_2P          005370b8   NScroll.obj
 0003:0002f310       _select_laps_2P            00537310   NScroll.obj
 0003:0002f728       _select_tm_attck           00537728   NScroll.obj
 0003:0002f900       _select_course_tm          00537900   NScroll.obj
 0003:000302d8       _select_laps_tm            005382d8   NScroll.obj
 0003:00030310       _select_option             00538310   NScroll.obj
 0003:00030838       _select_option_sound       00538838   NScroll.obj
 0003:00030e80       _select_setting            00538e80   NScroll.obj
 0003:00031020       _car_setting               00539020   NScroll.obj
 0003:00031380       _select_record             00539380   NScroll.obj
 0003:00031ed0       _md_org_cl                 00539ed0   NScroll.obj
 0003:000320d0       _md_yel_cl                 0053a0d0   NScroll.obj
 0003:000322d0       _md_slt_cl                 0053a2d0   NScroll.obj
 0003:000324d0       _md_slt0_cl                0053a4d0   NScroll.obj
 0003:000326d0       _md_slt1_cl                0053a6d0   NScroll.obj
 0003:0004b8d0       _md_pal                    005538d0   NScroll.obj
 0003:0004bba8       _cchange_sur_num           00553ba8   NScroll.obj
 0003:0004bbb8       _reload                    00553bb8   NScroll.obj
 0003:0004bc80       _map_desertbg              00553c80   Mpdesert.obj
 0003:0004d390       _cs10_flg                  00555390   setting.obj
 0003:0004d394       _cs20_flg                  00555394   setting.obj
 0003:0004d398       _set_flg                   00555398   setting.obj
 0003:0004d39c       _new_set_car               0055539c   setting.obj
 0003:0004d3a0       _setting_scroll_flag       005553a0   setting.obj
 0003:0004d3a4       _setting_scroll_mode       005553a4   setting.obj
 0003:0004d3a8       _setting_scroll_delay      005553a8   setting.obj
 0003:0004d3b0       _set_carselect_out         005553b0   setting.obj
 0003:0004d510       _setting_in                00555510   setting.obj
 0003:0004d5f0       _atmt_out                  005555f0   setting.obj
 0003:0004d640       _atmt_in                   00555640   setting.obj
 0003:0004d690       _handling_out              00555690   setting.obj
 0003:0004d770       _handling_in               00555770   setting.obj
 0003:0004d850       _tire_in                   00555850   setting.obj
 0003:0004d930       _tire_out                  00555930   setting.obj
 0003:0004da10       _sus_in                    00555a10   setting.obj
 0003:0004daf0       _sus_out                   00555af0   setting.obj
 0003:0004dbd0       _save_in                   00555bd0   setting.obj
 0003:0004dc70       _save_out                  00555c70   setting.obj
 0003:0004dd10       _set_carselect_in          00555d10   setting.obj
 0003:0004de60       _setting_out               00555e60   setting.obj
 0003:0004e150       _dammy_in                  00556150   setting.obj
 0003:0004e170       _dammy_out                 00556170   setting.obj
 0003:0004e190       _setting_scroll_list       00556190   setting.obj
 0003:0004e1d8       _cl_desertbg               005561d8   Cldesert.obj
 0003:0004e3d8       _ghWnd                     005563d8   WinMain.obj
 0003:0004e3dc       _ghInstance                005563dc   WinMain.obj
 0003:0004e3e0       _bShowInfomation           005563e0   WinMain.obj
 0003:0004e3e4       _bFullscreen               005563e4   WinMain.obj
 0003:0004e3e8       _bSystemPause              005563e8   WinMain.obj
 0003:0004e3ec       _szAppClass                005563ec   WinMain.obj
 0003:0004e3f0       _szAppTitle                005563f0   WinMain.obj
 0003:0004e3f4       _bDA_LOOP                  005563f4   WinMain.obj
 0003:0004e3f8       _bDASound                  005563f8   WinMain.obj
 0003:0004e3fc       _bRealDraw                 005563fc   WinMain.obj
 0003:0004e400       _bDispModeSelect           00556400   WinMain.obj
 0003:0004e404       _DispModeCur               00556404   WinMain.obj
 0003:0004e408       _ghMenu                    00556408   WinMain.obj
 0003:0004e40c       _bBGDisp                   0055640c   WinMain.obj
 0003:0004e410       _gLanguage                 00556410   WinMain.obj
 0003:0004e414       _bAlways1st                00556414   WinMain.obj
 0003:0004e418       _gCDDrive                  00556418   WinMain.obj
 0003:0004e41c       _bSystemPause_SoundPass    0055641c   WinMain.obj
 0003:0004e420       _bChangeControlReq         00556420   WinMain.obj
 0003:0004e424       _bChangeControlWait        00556424   WinMain.obj
 0003:0004e428       _UserCode                  00556428   WinMain.obj
 0003:0004e42c       _RestartRaceReq            0055642c   WinMain.obj
 0003:0004e460       _szFPS                     00556460   WinMain.obj
 0003:0004e470       _szINFO                    00556470   WinMain.obj
 0003:0004e4a0       _szINFOW                   005564a0   WinMain.obj
 0003:0004e4d4       _InfoColor                 005564d4   WinMain.obj
 0003:0004e4d8       _FrameRateColor            005564d8   WinMain.obj
 0003:0004e4dc       _BackColor                 005564dc   WinMain.obj
 0003:0004e908       _B_btl_desert              00556908   Mldesert.obj
 0003:000517c0       _mldesert                  005597c0   Mldesert.obj
 0003:000519c0       _B_blk_desert              005599c0   Mbdesert.obj
 0003:000537b0       _mbdesert                  0055b7b0   Mbdesert.obj
 0003:000577b0       _lpDirectSound             0055f7b0   DS.obj
 0003:000577b4       _pWAVEBUF                  0055f7b4   DS.obj
 0003:000577b8       _gWAVENO                   0055f7b8   DS.obj
 0003:000577bc       _gENGNO                    0055f7bc   DS.obj
 0003:000577c0       _sound_flag                0055f7c0   DS.obj
 0003:000577c4       _start_flg                 0055f7c4   DS.obj
 0003:000577c8       _bWAVEPAUSE                0055f7c8   DS.obj
 0003:000577cc       _bEngPauseFlag             0055f7cc   DS.obj
 0003:000577d0       _bSlipFlag                 0055f7d0   DS.obj
 0003:000577d4       _WaveOpenFlag              0055f7d4   DS.obj
 0003:000577d8       _WaveCloseFlag             0055f7d8   DS.obj
 0003:000577dc       _bENGFLAG                  0055f7dc   DS.obj
 0003:000577e0       _bWater                    0055f7e0   DS.obj
 0003:000577e4       _Load0Flag                 0055f7e4   DS.obj
 0003:000577e8       _wave_check_flg            0055f7e8   DS.obj
 0003:000577ec       _race_end_flag             0055f7ec   DS.obj
 0003:000577f0       _g_check                   0055f7f0   DS.obj
 0003:000577f4       _ghost_check               0055f7f4   DS.obj
 0003:000577f8       _wavepause                 0055f7f8   DS.obj
 0003:000577fc       _Engine_2pflag             0055f7fc   DS.obj
 0003:00057800       _net_2pengine              0055f800   DS.obj
 0003:00057804       _CarNo                     0055f804   DS.obj
 0003:00057808       _coli_sound_flag           0055f808   DS.obj
 0003:0005780c       _gSLIPCNT                  0055f80c   DS.obj
 0003:00057810       _wavebank1                 0055f810   DS.obj
 0003:00057b58       _wavebank2                 0055fb58   DS.obj
 0003:00057b80       _wavebank3                 0055fb80   DS.obj
 0003:00057bd8       _wavebank4                 0055fbd8   DS.obj
 0003:00057c30       _wavebank5                 0055fc30   DS.obj
 0003:00057cb8       _wavebank6                 0055fcb8   DS.obj
 0003:00057ce0       _wavebank7                 0055fce0   DS.obj
 0003:00057d68       _enginebank1               0055fd68   DS.obj
 0003:00057d98       _enginebank2               0055fd98   DS.obj
 0003:00057dc8       _enginebank3               0055fdc8   DS.obj
 0003:00057df8       _optionbank                0055fdf8   DS.obj
 0003:00057f70       _WaveBankTable             0055ff70   DS.obj
 0003:00057fa0       _OCT1                      0055ffa0   DS.obj
 0003:00057fe0       _OCT2                      0055ffe0   DS.obj
 0003:00058c20       _error_list                00560c20   gameproc.obj
 0003:0005ad88       _DispScale                 00562d88   gameproc.obj
 0003:0005ad8c       _DispPolyType              00562d8c   gameproc.obj
 0003:0005adc0       _gGameMode                 00562dc0   SaturnMain.obj
 0003:0005adc4       _bSelectMode               00562dc4   SaturnMain.obj
 0003:0005add0       _master_flag               00562dd0   SaturnSim.obj
 0003:0005add4       _revchk_flg                00562dd4   SaturnSim.obj
 0003:0005add8       _ptsStart                  00562dd8   SaturnSim.obj
 0003:0005ae08       _PaletteCache              00562e08   SaturnSim.obj
 0003:0005ae48       _CasheCnt                  00562e48   SaturnSim.obj
 0003:0005ae4c       _pPauseBitmap              00562e4c   winapi.obj
 0003:0005b0e0       _GameScrObj                005630e0   scrdat.obj
 0003:0005b7d8       _AdvScrObj                 005637d8   scrdat.obj
 0003:0005b930       _NameScrObj                00563930   scrdat.obj
 0003:0005c100       _StaffScrObj               00564100   scrdat.obj
 0003:0005c420       _Staff2ScrObj              00564420   scrdat.obj
 0003:0005cc90       _ScrObjTbl                 00564c90   scrdat.obj
 0003:0005ede8       _fn_gmdl_tbl_00            00566de8   Cdload.obj
 0003:0005ee00       _fn_tex_tbl_00             00566e00   Cdload.obj
 0003:0005ee18       _fn_cl_tbl_00              00566e18   Cdload.obj
 0003:0005ee30       _fn_model_tbl              00566e30   Cdload.obj
 0003:0005ee40       _fn_gmdl_tbl_2p            00566e40   Cdload.obj
 0003:0005ee58       _fn_tex_tbl_2p             00566e58   Cdload.obj
 0003:0005ee70       _fn_cl_tbl_2p              00566e70   Cdload.obj
 0003:0005ee88       _fn_ending_tbl             00566e88   Cdload.obj
 0003:0005ee98       _fn_select_tbl             00566e98   Cdload.obj
 0003:0005eea8       _fn_staff_tbl              00566ea8   Cdload.obj
 0003:0005eeb8       _fn_model_2p_tbl           00566eb8   Cdload.obj
 0003:0005eed0       _fn_model_animal_tbl       00566ed0   Cdload.obj
 0003:0005eee0       _fn_eventtbl_tbl           00566ee0   Cdload.obj
 0003:0005eeec       _fn_model_alphabet_tbl     00566eec   Cdload.obj
 0003:0005eef0       _fn_camera_dat             00566ef0   Cdload.obj
 0003:0005eef4       _fn_phototbl_tbl           00566ef4   Cdload.obj
 0003:0005ef08       _model_base_tbl            00566f08   Cdload.obj
 0003:0005ef28       _model_base_tbl2p          00566f28   Cdload.obj
 0003:0005f268       _animal2_poly_tbl          00567268   Cdload.obj
 0003:0005f2f8       _object2p_poly_tbl         005672f8   Cdload.obj
 0003:0005f390       _alpha_poly_tbl            00567390   Cdload.obj
 0003:0005f480       _ending_poly_tbl           00567480   Cdload.obj
 0003:0005f550       _select_poly_tbl           00567550   Cdload.obj
 0003:0005f6b0       _staff_poly_tbl            005676b0   Cdload.obj
 0003:0005fa9c       _JoyNum                    00567a9c   joyctrl.obj
 0003:0005faa0       _opt_init_tbl              00567aa0   bup_file.obj
 0003:0005fb68       _rec_data_init             00567b68   bup_file.obj
 0003:00060768       _rec_table_init            00568768   bup_file.obj
 0003:00060878       _cmp_table_init            00568878   bup_file.obj
 0003:00060998       _DPTEST_GUID               00568998   dpctrl.obj
 0003:000609a8       _network                   005689a8   dpctrl.obj
 0003:000609ac       _lpIDC                     005689ac   dpctrl.obj
 0003:000609b0       _IsHost                    005689b0   dpctrl.obj
 0003:000609b4       _InitSWSendFlag            005689b4   dpctrl.obj
 0003:000609b8       _ReceiveBuffWtCount        005689b8   dpctrl.obj
 0003:000609bc       _ReceiveBuffRdCount        005689bc   dpctrl.obj
 0003:000609c0       _swdatawritecnt            005689c0   dpctrl.obj
 0003:000609c4       _swdatacnt                 005689c4   dpctrl.obj
 0003:000609c8       _InitLinkFlag              005689c8   dpctrl.obj
 0003:000609cc       _Index                     005689cc   dpctrl.obj
 0003:00061bd8       _B_cli_lake                00569bd8   Mclake.obj
 0003:0008b970       _mclake                    00593970   Mclake.obj
 0003:0008f970       R0                         00597970   sh2reg.obj
 0003:0008f970       _SH_R0                     00597970   sh2reg.obj
 0003:0008f970       _R0                        00597970   sh2reg.obj
 0003:0008f974       _SH_R1                     00597974   sh2reg.obj
 0003:0008f974       _R1                        00597974   sh2reg.obj
 0003:0008f974       R1                         00597974   sh2reg.obj
 0003:0008f978       R2                         00597978   sh2reg.obj
 0003:0008f978       _R2                        00597978   sh2reg.obj
 0003:0008f978       _SH_R2                     00597978   sh2reg.obj
 0003:0008f97c       _R3                        0059797c   sh2reg.obj
 0003:0008f97c       R3                         0059797c   sh2reg.obj
 0003:0008f97c       _SH_R3                     0059797c   sh2reg.obj
 0003:0008f980       _SH_R4                     00597980   sh2reg.obj
 0003:0008f980       R4                         00597980   sh2reg.obj
 0003:0008f980       _R4                        00597980   sh2reg.obj
 0003:0008f984       R5                         00597984   sh2reg.obj
 0003:0008f984       _R5                        00597984   sh2reg.obj
 0003:0008f984       _SH_R5                     00597984   sh2reg.obj
 0003:0008f988       _R6                        00597988   sh2reg.obj
 0003:0008f988       R6                         00597988   sh2reg.obj
 0003:0008f988       _SH_R6                     00597988   sh2reg.obj
 0003:0008f98c       _SH_R7                     0059798c   sh2reg.obj
 0003:0008f98c       R7                         0059798c   sh2reg.obj
 0003:0008f98c       _R7                        0059798c   sh2reg.obj
 0003:0008f990       _SH_R8                     00597990   sh2reg.obj
 0003:0008f990       R8                         00597990   sh2reg.obj
 0003:0008f990       _R8                        00597990   sh2reg.obj
 0003:0008f994       _R9                        00597994   sh2reg.obj
 0003:0008f994       _SH_R9                     00597994   sh2reg.obj
 0003:0008f994       R9                         00597994   sh2reg.obj
 0003:0008f998       R10                        00597998   sh2reg.obj
 0003:0008f998       _R10                       00597998   sh2reg.obj
 0003:0008f998       _SH_R10                    00597998   sh2reg.obj
 0003:0008f99c       _SH_R11                    0059799c   sh2reg.obj
 0003:0008f99c       _R11                       0059799c   sh2reg.obj
 0003:0008f99c       R11                        0059799c   sh2reg.obj
 0003:0008f9a0       _SH_R12                    005979a0   sh2reg.obj
 0003:0008f9a0       R12                        005979a0   sh2reg.obj
 0003:0008f9a0       _R12                       005979a0   sh2reg.obj
 0003:0008f9a4       R13                        005979a4   sh2reg.obj
 0003:0008f9a4       _SH_R13                    005979a4   sh2reg.obj
 0003:0008f9a4       _R13                       005979a4   sh2reg.obj
 0003:0008f9a8       _SH_R14                    005979a8   sh2reg.obj
 0003:0008f9a8       _R14                       005979a8   sh2reg.obj
 0003:0008f9a8       R14                        005979a8   sh2reg.obj
 0003:0008f9ac       MACL                       005979ac   sh2reg.obj
 0003:0008f9ac       _MACL                      005979ac   sh2reg.obj
 0003:0008f9ac       _SH_MACL                   005979ac   sh2reg.obj
 0003:0008f9b0       _MACH                      005979b0   sh2reg.obj
 0003:0008f9b0       _SH_MACH                   005979b0   sh2reg.obj
 0003:0008f9b0       MACH                       005979b0   sh2reg.obj
 0003:0008f9b4       PR                         005979b4   sh2reg.obj
 0003:0008f9b4       _PR                        005979b4   sh2reg.obj
 0003:0008f9b4       _SH_PR                     005979b4   sh2reg.obj
 0003:0008f9b8       _SR                        005979b8   sh2reg.obj
 0003:0008f9b8       SR                         005979b8   sh2reg.obj
 0003:0008f9b8       _SH_SR                     005979b8   sh2reg.obj
 0003:0008f9bc       _SH_VBR                    005979bc   sh2reg.obj
 0003:0008f9bc       _VBR                       005979bc   sh2reg.obj
 0003:0008f9bc       VBR                        005979bc   sh2reg.obj
 0003:0008f9c0       _SH_GBR                    005979c0   sh2reg.obj
 0003:0008f9c0       _GBR                       005979c0   sh2reg.obj
 0003:0008f9c0       GBR                        005979c0   sh2reg.obj
 0003:0008f9c4       _SH2I386_TEMP              005979c4   sh2reg.obj
 0003:0008f9c4       SH2I386_TEMP               005979c4   sh2reg.obj
 0003:0008f9c8       _NotifyWait                005979c8   CDSND.obj
 0003:0008f9cc       _bRePlay                   005979cc   CDSND.obj
 0003:0008f9d0       _gTrackNo                  005979d0   CDSND.obj
 0003:0008f9d4       _gCDInit                   005979d4   CDSND.obj
 0003:0008f9d8       _bPause                    005979d8   CDSND.obj
 0003:0008f9dc       _AMSELECT_STOP             005979dc   CDSND.obj
 0003:0008f9f4       _scrobj_tacho              005979f4   Scrlobj.obj
 0003:0008f9f8       _scrobj_tacho2             005979f8   Scrlobj.obj
 0003:0008f9fc       _scrobj_gyakusou           005979fc   Scrlobj.obj
 0003:0008fa00       _scrobj_navi               00597a00   Scrlobj.obj
 0003:0008fa04       _scrobj_shift              00597a04   Scrlobj.obj
 0003:0008fa08       _scrobj_speed              00597a08   Scrlobj.obj
 0003:0008fa0c       _scrobj_rank               00597a0c   Scrlobj.obj
 0003:0008fa10       _scrobj_extend             00597a10   Scrlobj.obj
 0003:0008fa14       _scrobj_laptime            00597a14   Scrlobj.obj
 0003:0008fa18       _scrobj_timecmp            00597a18   Scrlobj.obj
 0003:0008fa1c       _scrobj_besttime           00597a1c   Scrlobj.obj
 0003:0008fa20       _scrobj_result             00597a20   Scrlobj.obj
 0003:0008fa24       _scrobj_vswin              00597a24   Scrlobj.obj
 0003:0008fa28       _scrobj_over               00597a28   Scrlobj.obj
 0003:0008fa2c       _scrobj_adv                00597a2c   Scrlobj.obj
 0003:0008fa30       _scrobj_name               00597a30   Scrlobj.obj
 0003:0008fa34       _scrobj_replay             00597a34   Scrlobj.obj
 0003:0008fa38       _scrobj_staff              00597a38   Scrlobj.obj
 0003:0008fa3c       _scrobj_staff2             00597a3c   Scrlobj.obj
 0003:0008ff68       _B_btl_forest              00597f68   Mlforest.obj
 0003:00092d98       _mlforest                  0059ad98   Mlforest.obj
 0003:00092f98       _staff2_vpos_tbl           0059af98   staffroll.obj
 0003:00093070       _pad_position              0059b070   option.obj
 0003:00093074       _pre_pad                   0059b074   option.obj
 0003:00093078       _pre_posi                  0059b078   option.obj
 0003:0009307c       _sound_posi                0059b07c   option.obj
 0003:00093080       _sound_opt_flg             0059b080   option.obj
 0003:00093084       _sound_scroll_flag         0059b084   option.obj
 0003:00093088       _option_scroll_flag        0059b088   option.obj
 0003:0009308c       _option_scroll_mode        0059b08c   option.obj
 0003:00093090       _option_scroll_delay       0059b090   option.obj
 0003:00093098       _option_start_out          0059b098   option.obj
 0003:000930b8       _option_in                 0059b0b8   option.obj
 0003:00093428       _option_out                0059b428   option.obj
 0003:00093778       _sound_in                  0059b778   option.obj
 0003:00093c48       _sound_out                 0059bc48   option.obj
 0003:00094128       _option_scroll_list        0059c128   option.obj
 0003:00094178       _gBGColor                  0059c178   Bgctrl.obj
 0003:00094180       _FadeOutPat                0059c180   Bgctrl.obj
 0003:000943c8       _int_min                   0059c3c8   mabiki.obj
 0003:00094420       _WaitFlag                  0059c420   mabiki.obj
 0003:00094428       _B_blk_forest              0059c428   Mbforest.obj
 0003:00095ec8       _mbforest                  0059dec8   Mbforest.obj
 0003:00099f18       _ExTextureCnt              005a1f18   Texture.obj
 0003:00099f1c       _ExTextureSize             005a1f1c   Texture.obj
 0003:00099f20       _ExTextureBPP              005a1f20   Texture.obj
 0003:00099f28       _GameTextureTbl            005a1f28   Texture.obj
 0003:00099f98       _Animal2TextureTbl         005a1f98   Texture.obj
 0003:00099fa8       _SelectTextureTbl          005a1fa8   Texture.obj
 0003:0009a000       _EndingTextureTbl          005a2000   Texture.obj
 0003:0009a010       _StaffTextureTbl           005a2010   Texture.obj
 0003:0009a020       _Game2pTextureTbl1         005a2020   Texture.obj
 0003:0009a060       _Game2pTextureTbl2         005a2060   Texture.obj
 0003:0009a088       _texttbl_tbl               005a2088   Texture.obj
 0003:0009a098       _texttbl2p_tbl             005a2098   Texture.obj
 0003:0009a0a8       _id_tbl_00                 005a20a8   Texture.obj
 0003:0009a0e8       _id_tbl_2p                 005a20e8   Texture.obj
 0003:0009a128       _side_t_lamp_new           005a2128   Texture.obj
 0003:0009a1a8       _KEYCODENAMES              005a21a8   Keydlg.obj
 0003:0009a4d8       _JOYCODENAMES              005a24d8   Keydlg.obj
 0003:0009aa20       _DefaultKeyType1           005a2a20   Keydlg.obj
 0003:0009aa70       _DefaultKeyType2           005a2a70   Keydlg.obj
 0003:0009aac0       _DefaultJoyType1           005a2ac0   Keydlg.obj
 0003:0009ab10       _DefaultJoyType2           005a2b10   Keydlg.obj
 0003:0009ab70       _rally_level               005a2b70   Prgdata2.obj
 0003:0009ab80       _rally_esy_lap             005a2b80   Prgdata2.obj
 0003:0009abb8       _rally_nml_lap             005a2bb8   Prgdata2.obj
 0003:0009abf0       _rally_hard_lap            005a2bf0   Prgdata2.obj
 0003:0009ac28       _prac_level                005a2c28   Prgdata2.obj
 0003:0009ac38       _prac_esy_lap              005a2c38   Prgdata2.obj
 0003:0009ac70       _prac_nml_lap              005a2c70   Prgdata2.obj
 0003:0009aca8       _prac_hard_lap             005a2ca8   Prgdata2.obj
 0003:0009ace0       _start_spldata             005a2ce0   Prgdata2.obj
 0003:0009ad10       _start_spldata2p           005a2d10   Prgdata2.obj
 0003:0009ad40       _goal_posi_tbl             005a2d40   Prgdata2.obj
 0003:0009add0       _goal_posi1p_tbl           005a2dd0   Prgdata2.obj
 0003:0009ae60       _goal_posi2p_tbl           005a2e60   Prgdata2.obj
 0003:0009aef0       _pinit_tbl                 005a2ef0   Prgdata2.obj
 0003:0009af30       _pinit1p_tbl               005a2f30   Prgdata2.obj
 0003:0009af70       _pinit2p_tbl               005a2f70   Prgdata2.obj
 0003:0009afb0       _B_blk_mount               005a2fb0   Mbmount.obj
 0003:0009c948       _mbmount                   005a4948   Mbmount.obj
 0003:000a0948       _net_initflag              005a8948   CS_BATTLE_2P.obj
 0003:000a094c       _battle_scroll_flag        005a894c   CS_BATTLE_2P.obj
 0003:000a0950       _battle_2pscroll_flag      005a8950   CS_BATTLE_2P.obj
 0003:000a0954       _battle_scroll_mode        005a8954   CS_BATTLE_2P.obj
 0003:000a0958       _battle_2pscroll_mode      005a8958   CS_BATTLE_2P.obj
 0003:000a095c       _battle_scroll_delay       005a895c   CS_BATTLE_2P.obj
 0003:000a0960       _battle_2pscroll_delay     005a8960   CS_BATTLE_2P.obj
 0003:000a0964       _SubModeFlag1              005a8964   CS_BATTLE_2P.obj
 0003:000a0968       _SubModeFlag2              005a8968   CS_BATTLE_2P.obj
 0003:000a096c       _bt_ms13                   005a896c   CS_BATTLE_2P.obj
 0003:000a0970       _bt_ms23                   005a8970   CS_BATTLE_2P.obj
 0003:000a0974       _start1                    005a8974   CS_BATTLE_2P.obj
 0003:000a0978       _start2                    005a8978   CS_BATTLE_2P.obj
 0003:000a097c       _tuned1                    005a897c   CS_BATTLE_2P.obj
 0003:000a0980       _tuned2                    005a8980   CS_BATTLE_2P.obj
 0003:000a0984       _lap_flg                   005a8984   CS_BATTLE_2P.obj
 0003:000a0988       _cancel_flg1               005a8988   CS_BATTLE_2P.obj
 0003:000a098c       _END_flg                   005a898c   CS_BATTLE_2P.obj
 0003:000a0990       _hande                     005a8990   CS_BATTLE_2P.obj
 0003:000a0994       _scrl_carname1_1p_flg      005a8994   CS_BATTLE_2P.obj
 0003:000a0998       _scrl_carname1_2p_flg      005a8998   CS_BATTLE_2P.obj
 0003:000a099c       _lscrl_p1_part1_0_flg      005a899c   CS_BATTLE_2P.obj
 0003:000a09a0       _lscrl_p2_part1_0_flg      005a89a0   CS_BATTLE_2P.obj
 0003:000a09a4       _crs_flg                   005a89a4   CS_BATTLE_2P.obj
 0003:000a09a8       _title_2pscroll_flag       005a89a8   CS_BATTLE_2P.obj
 0003:000a09b0       _battle_s_lap_out          005a89b0   CS_BATTLE_2P.obj
 0003:000a09f0       _battle_s_lap_in           005a89f0   CS_BATTLE_2P.obj
 0003:000a0a30       _battle_cource_dx_out      005a8a30   CS_BATTLE_2P.obj
 0003:000a0a80       _battle_cource_dx_in       005a8a80   CS_BATTLE_2P.obj
 0003:000a0ad0       _battle_car1_dx_out        005a8ad0   CS_BATTLE_2P.obj
 0003:000a0b10       _battle_car1_dx_in         005a8b10   CS_BATTLE_2P.obj
 0003:000a0b50       _battle_car2_dx_out        005a8b50   CS_BATTLE_2P.obj
 0003:000a0b90       _battle_car2_dx_in         005a8b90   CS_BATTLE_2P.obj
 0003:000a0bd0       _battle_standard_car1_out  005a8bd0   CS_BATTLE_2P.obj
 0003:000a0c90       _battle_standard_car1_in   005a8c90   CS_BATTLE_2P.obj
 0003:000a0d50       _battle_standard_car2_out  005a8d50   CS_BATTLE_2P.obj
 0003:000a0e10       _battle_standard_car2_in   005a8e10   CS_BATTLE_2P.obj
 0003:000a0ed0       _battle_tuned_car1_in      005a8ed0   CS_BATTLE_2P.obj
 0003:000a0f90       _battle_tuned_car1_out     005a8f90   CS_BATTLE_2P.obj
 0003:000a1050       _battle_tuned_car2_in      005a9050   CS_BATTLE_2P.obj
 0003:000a1110       _battle_tuned_car2_out     005a9110   CS_BATTLE_2P.obj
 0003:000a11d0       _battle_car_select_out     005a91d0   CS_BATTLE_2P.obj
 0003:000a14a0       _battle_car_select_in      005a94a0   CS_BATTLE_2P.obj
 0003:000a1770       _battle_cource_select_out  005a9770   CS_BATTLE_2P.obj
 0003:000a1970       _battle_cource_select_in   005a9970   CS_BATTLE_2P.obj
 0003:000a1b70       _battle_cource_in          005a9b70   CS_BATTLE_2P.obj
 0003:000a1c60       _battle_cource_out         005a9c60   CS_BATTLE_2P.obj
 0003:000a1d10       _battle_lap_select_in      005a9d10   CS_BATTLE_2P.obj
 0003:000a1dd0       _battle_lap_select_out     005a9dd0   CS_BATTLE_2P.obj
 0003:000a1e90       _battle_lap_in             005a9e90   CS_BATTLE_2P.obj
 0003:000a1f50       _battle_lap_out            005a9f50   CS_BATTLE_2P.obj
 0003:000a1fe0       _battle_d_start_out        005a9fe0   CS_BATTLE_2P.obj
 0003:000a2140       _battle_d_start_in         005aa140   CS_BATTLE_2P.obj
 0003:000a22a0       _battle_boost_out          005aa2a0   CS_BATTLE_2P.obj
 0003:000a2300       _battle_boost_in           005aa300   CS_BATTLE_2P.obj
 0003:000a2360       _battle_lag_out            005aa360   CS_BATTLE_2P.obj
 0003:000a2490       _battle_lag_in             005aa490   CS_BATTLE_2P.obj
 0003:000a25c0       _battle_scroll_list        005aa5c0   CS_BATTLE_2P.obj
 0003:000a2630       _battle_2pscroll_list      005aa630   CS_BATTLE_2P.obj
 0003:000a2654       _ghost_disp_mode           005aa654   record.obj
 0003:000a2658       _lank_disp_mode            005aa658   record.obj
 0003:000a265c       _lank_up_disp              005aa65c   record.obj
 0003:000a2660       _lank_down_disp            005aa660   record.obj
 0003:000a2678       _record_select_cource      005aa678   record.obj
 0003:000a26a8       _record_s                  005aa6a8   record.obj
 0003:000a26c8       _timeattack_s              005aa6c8   record.obj
 0003:000a26e8       _record_e                  005aa6e8   record.obj
 0003:000a2818       _a_c_p_s                   005aa818   record.obj
 0003:000a2948       _a_c_p_e                   005aa948   record.obj
 0003:000a2a58       _a_c_lc_s                  005aaa58   record.obj
 0003:000a2b68       _a_c_lc_e                  005aab68   record.obj
 0003:000a2c78       _a_p_cc_s                  005aac78   record.obj
 0003:000a2d48       _a_p_cc_e                  005aad48   record.obj
 0003:000a2e18       _a_p_c_s                   005aae18   record.obj
 0003:000a2f28       _a_p_c_e                   005aaf28   record.obj
 0003:000a3058       _a_c_t_s                   005ab058   record.obj
 0003:000a31c8       _a_c_t_e                   005ab1c8   record.obj
 0003:000a3338       _timeattack_e              005ab338   record.obj
 0003:000a3428       _a_p_t_s                   005ab428   record.obj
 0003:000a35b8       _a_p_t_e                   005ab5b8   record.obj
 0003:000a36e8       _a_t_c_s                   005ab6e8   record.obj
 0003:000a3868       _a_t_c_e                   005ab868   record.obj
 0003:000a39d8       _a_t_p_s                   005ab9d8   record.obj
 0003:000a3b38       _a_t_p_e                   005abb38   record.obj
 0003:000a3c48       _a_t_csc_s                 005abc48   record.obj
 0003:000a3cf8       _a_t_csc_e                 005abcf8   record.obj
 0003:000a3da8       _a_t_cc_s                  005abda8   record.obj
 0003:000a3e48       _a_t_cc_e                  005abe48   record.obj
 0003:000a3ee8       _a_t_tc_s                  005abee8   record.obj
 0003:000a3f58       _a_t_tc_e                  005abf58   record.obj
 0003:000a3fc8       _line_scroll_list          005abfc8   record.obj
 0003:000a41a8       _B_blk_lake                005ac1a8   Mblake.obj
 0003:000a5c78       _mblake                    005adc78   Mblake.obj
 0003:000a9c78       _SubModeFlag               005b1c78   tm_attck.obj
 0003:000a9c7c       _start_flag                005b1c7c   tm_attck.obj
 0003:000a9c80       _cancel_flg                005b1c80   tm_attck.obj
 0003:000a9c84       _TM_END                    005b1c84   tm_attck.obj
 0003:000a9c88       _rec_flag                  005b1c88   tm_attck.obj
 0003:000a9c8c       _lay1_flag                 005b1c8c   tm_attck.obj
 0003:000a9c90       _title_scroll_flag         005b1c90   tm_attck.obj
 0003:000a9c94       _tm_scroll_flag            005b1c94   tm_attck.obj
 0003:000a9c98       _tm_scroll_mode            005b1c98   tm_attck.obj
 0003:000a9c9c       _tm_scroll_delay           005b1c9c   tm_attck.obj
 0003:000a9ca0       _tm_cource_dx_out          005b1ca0   tm_attck.obj
 0003:000a9cf0       _tm_cource_dx_in           005b1cf0   tm_attck.obj
 0003:000a9d40       _tm_car_dx_out             005b1d40   tm_attck.obj
 0003:000a9d80       _tm_car_dx_in              005b1d80   tm_attck.obj
 0003:000a9dc0       _tm_standard_car_out       005b1dc0   tm_attck.obj
 0003:000a9e80       _tm_standard_car_in        005b1e80   tm_attck.obj
 0003:000a9f40       _tm_tuned_car_in           005b1f40   tm_attck.obj
 0003:000aa000       _tm_tuned_car_out          005b2000   tm_attck.obj
 0003:000aa0c0       _tm_car_select_out         005b20c0   tm_attck.obj
 0003:000aa230       _tm_car_select_in          005b2230   tm_attck.obj
 0003:000aa3a0       _tm_cource_select_in       005b23a0   tm_attck.obj
 0003:000aa520       _tm_cource_select_out      005b2520   tm_attck.obj
 0003:000aa6a0       _tm_cource_in              005b26a0   tm_attck.obj
 0003:000aa750       _tm_cource_out             005b2750   tm_attck.obj
 0003:000aa800       _tm_lap_select_in          005b2800   tm_attck.obj
 0003:000aa870       _tm_lap_select_out         005b2870   tm_attck.obj
 0003:000aa8e0       _tm_scroll_list            005b28e0   tm_attck.obj
 0003:000aa958       _B_cli_forest              005b2958   Mcforest.obj
 0003:000e9eb0       _mcforest                  005f1eb0   Mcforest.obj
 0003:000edeb0       _cg_desertbg               005f5eb0   Cgdesert.obj
 0003:000fad50       _B_btl_mount               00602d50   Mlmount.obj
 0003:000fdbe0       _mlmount                   00605be0   Mlmount.obj
 0003:000fdde0       _B_cli_mount               00605de0   Mcmount.obj
 0003:0012b2c8       _mcmount                   006332c8   Mcmount.obj
 0003:0012f2c8       _bTransDest                006372c8   ddraw.obj
 0003:0012f2d0       _B_btl_lake                006372d0   Mllake.obj
 0003:00132140       _mllake                    0063a140   Mllake.obj
 0003:00132360       _LIMUX                     0063a360   Fchatex.obj
 0003:00132364       _LIMUY                     0063a364   Fchatex.obj
 0003:00132368       _LIMUX1                    0063a368   Fchatex.obj
 0003:0013236c       _LIMUY1                    0063a36c   Fchatex.obj
 0003:00132398       _time2                     0063a398   Keyctrl.obj
 0003:0013239c       _LinkCheckTime             0063a39c   Keyctrl.obj
 0003:001323a0       _LinkCountTime             0063a3a0   Keyctrl.obj
 0003:001323a4       _LinkCount                 0063a3a4   Keyctrl.obj
 0003:001323a8       _Time                      0063a3a8   Keyctrl.obj
 0003:001323ac       _LinkTimeAvg               0063a3ac   Keyctrl.obj
 0003:001323b0       _LinkTime                  0063a3b0   Keyctrl.obj
 0003:001323b4       _send_flag                 0063a3b4   Keyctrl.obj
 0003:001323b8       _test_buf                  0063a3b8   Keyctrl.obj
 0003:00132530       __fltused                  0063a530   LIBC:fpinit.obj
 0003:00132534       __ldused                   0063a534   LIBC:fpinit.obj
 0003:00132538       ___fastflag                0063a538   LIBC:fpinit.obj
 0003:0013253c       __adjust_fdiv              0063a53c   LIBC:fpinit.obj
 0003:00132540       __FPinit                   0063a540   LIBC:fpinit.obj
 0003:00132544       __FPmtinit                 0063a544   LIBC:fpinit.obj
 0003:00132548       __FPmtterm                 0063a548   LIBC:fpinit.obj
 0003:0013254c       _errno                     0063a54c   LIBC:crt0dat.obj
 0003:00132550       __doserrno                 0063a550   LIBC:crt0dat.obj
 0003:00132554       __umaskval                 0063a554   LIBC:crt0dat.obj
 0003:00132558       __osver                    0063a558   LIBC:crt0dat.obj
 0003:0013255c       __winver                   0063a55c   LIBC:crt0dat.obj
 0003:00132560       __winmajor                 0063a560   LIBC:crt0dat.obj
 0003:00132564       __winminor                 0063a564   LIBC:crt0dat.obj
 0003:00132568       ___argc                    0063a568   LIBC:crt0dat.obj
 0003:0013256c       ___argv                    0063a56c   LIBC:crt0dat.obj
 0003:00132570       ___wargv                   0063a570   LIBC:crt0dat.obj
 0003:00132574       __environ                  0063a574   LIBC:crt0dat.obj
 0003:00132578       ___initenv                 0063a578   LIBC:crt0dat.obj
 0003:0013257c       __wenviron                 0063a57c   LIBC:crt0dat.obj
 0003:00132580       ___winitenv                0063a580   LIBC:crt0dat.obj
 0003:00132584       __pgmptr                   0063a584   LIBC:crt0dat.obj
 0003:00132588       __wpgmptr                  0063a588   LIBC:crt0dat.obj
 0003:0013258c       __exitflag                 0063a58c   LIBC:crt0dat.obj
 0003:00132590       __C_Termination_Done       0063a590   LIBC:crt0dat.obj
 0003:00132594       __NLG_Destination          0063a594   LIBC:exsup.obj
 0003:001325a4       __aenvptr                  0063a5a4   LIBC:wincrt0.obj
 0003:001325a8       __wenvptr                  0063a5a8   LIBC:wincrt0.obj
 0003:001325ac       __aexit_rtn                0063a5ac   LIBC:wincrt0.obj
 0003:001325b0       ___error_mode              0063a5b0   LIBC:wincrt0.obj
 0003:001325b4       ___app_type                0063a5b4   LIBC:wincrt0.obj
 0003:001325b8       ??_C@_0BB@JPOE@GetCurrentThread?$AA@ 0063a5b8   LIBC:testfdiv.obj
 0003:001325cc       ??_C@_0BG@PMJE@SetThreadAffinityMask?$AA@ 0063a5cc   LIBC:testfdiv.obj
 0003:001325e4       ??_C@_0BC@CFOG@GetCurrentProcess?$AA@ 0063a5e4   LIBC:testfdiv.obj
 0003:001325f8       ??_C@_0BH@KAJB@GetProcessAffinityMask?$AA@ 0063a5f8   LIBC:testfdiv.obj
 0003:00132610       ??_C@_08OBID@KERNEL32?$AA@ 0063a610   LIBC:testfdiv.obj
 0003:00132620       __cfltcvt_tab              0063a620   LIBC:cmiscdat.obj
 0003:00132644       ??_C@_05OFLO@e?$CL000?$AA@ 0063a644   LIBC:cvt.obj
 0003:00132650       __stdbuf                   0063a650   LIBC:_sftbuf.obj
 0003:00132658       ??_C@_1O@POHA@?$AA?$CI?$AAn?$AAu?$AAl?$AAl?$AA?$CJ?$AA?$AA?$AA?$AA?$AA?$AD?$AA?$AA?$AA?$AA?$AA?$AAã?$<I?$ADi@ 0063a658   LIBC:output.obj
 0003:00132668       ??_C@_06ONKE@?$CInull?$CJ?$AA@ 0063a668   LIBC:output.obj
 0003:00132670       ___nullstring              0063a670   LIBC:output.obj
 0003:00132674       ___wnullstring             0063a674   LIBC:output.obj
 0003:00132692       __OP_SINjmptab             0063a692   LIBC:87trig.obj
 0003:001326b2       __OP_COSjmptab             0063a6b2   LIBC:87trig.obj
 0003:001326d2       __OP_TANjmptab             0063a6d2   LIBC:87trig.obj
 0003:001326fc       ??_C@_01A@?$AA?$AA@        0063a6fc   LIBC:aw_map.obj
 0003:00132700       ??_C@_13A@?$AA?$AA?$AA?$AA?$AA?$AD?$AA?$AA@ 0063a700   LIBC:aw_map.obj
 0003:00132708       ___lc_handle               0063a708   LIBC:nlsdata2.obj
 0003:00132720       ___lc_codepage             0063a720   LIBC:nlsdata2.obj
 0003:00132728       __pctype                   0063a728   LIBC:ctype.obj
 0003:0013272c       __pwctype                  0063a72c   LIBC:ctype.obj
 0003:00132730       __ctype                    0063a730   LIBC:ctype.obj
 0003:00132934       ___mb_cur_max              0063a934   LIBC:nlsdata1.obj
 0003:00132938       ___decimal_point           0063a938   LIBC:nlsdata1.obj
 0003:0013293c       ___decimal_point_length    0063a93c   LIBC:nlsdata1.obj
 0003:0013294c       ?__pSETranslator@@3P6AXIPAU_EXCEPTION_POINTERS@@@ZA 0063a94c   LIBC:hooks.obj
 0003:00132950       ?__pTerminate@@3P6AXXZA    0063a950   LIBC:hooks.obj
 0003:00132954       ?__pUnexpected@@3P6AXXZA   0063a954   LIBC:hooks.obj
 0003:00132958       ?__pInconsistency@@3P6AXXZA 0063a958   LIBC:hooks.obj
 0003:00132960       __XcptActTab               0063a960   LIBC:winxfltr.obj
 0003:001329d8       __First_FPE_Indx           0063a9d8   LIBC:winxfltr.obj
 0003:001329dc       __Num_FPE                  0063a9dc   LIBC:winxfltr.obj
 0003:001329e0       __XcptActTabCount          0063a9e0   LIBC:winxfltr.obj
 0003:001329e4       __fpecode                  0063a9e4   LIBC:winxfltr.obj
 0003:001329e8       __pxcptinfoptrs            0063a9e8   LIBC:winxfltr.obj
 0003:001329f8       __mbctype                  0063a9f8   LIBC:mbctype.obj
 0003:00132afc       ___mbcodepage              0063aafc   LIBC:mbctype.obj
 0003:00132b00       ___mblcid                  0063ab00   LIBC:mbctype.obj
 0003:00132b08       ___mbulinfo                0063ab08   LIBC:mbctype.obj
 0003:00132c10       ___badioinfo               0063ac10   LIBC:ioinit.obj
 0003:00132c18       __amblksiz                 0063ac18   LIBC:heapinit.obj
 0003:00132c1c       ??_C@_0P@GGKG@runtime?5error?5?$AA@ 0063ac1c   LIBC:crt0msg.obj
 0003:00132c2c       ??_C@_02PIMC@?$AN?6?$AA@   0063ac2c   LIBC:crt0msg.obj
 0003:00132c30       ??_C@_0O@DELO@TLOSS?5error?$AN?6?$AA@ 0063ac30   LIBC:crt0msg.obj
 0003:00132c40       ??_C@_0N@OMLL@SING?5error?$AN?6?$AA@ 0063ac40   LIBC:crt0msg.obj
 0003:00132c50       ??_C@_0P@OJAK@DOMAIN?5error?$AN?6?$AA@ 0063ac50   LIBC:crt0msg.obj
 0003:00132c60       ??_C@_0DF@ECGN@R6027?$AN?6?9?5not?5enough?5space?5for?5lo@ 0063ac60   LIBC:crt0msg.obj
 0003:00132c98       ??_C@_0DF@FKAC@R6026?$AN?6?9?5not?5enough?5space?5for?5st@ 0063ac98   LIBC:crt0msg.obj
 0003:00132cd0       ??_C@_0CG@DPMN@R6025?$AN?6?9?5pure?5virtual?5function?5c@ 0063acd0   LIBC:crt0msg.obj
 0003:00132cf8       ??_C@_0DF@CKIP@R6024?$AN?6?9?5not?5enough?5space?5for?5_o@ 0063acf8   LIBC:crt0msg.obj
 0003:00132d30       ??_C@_0CJ@GGOE@R6019?$AN?6?9?5unable?5to?5open?5console?5@ 0063ad30   LIBC:crt0msg.obj
 0003:00132d5c       ??_C@_0CB@LBOB@R6018?$AN?6?9?5unexpected?5heap?5error?$AN?6@ 0063ad5c   LIBC:crt0msg.obj
 0003:00132d80       ??_C@_0CN@FPEG@R6017?$AN?6?9?5unexpected?5multithread?5@ 0063ad80   LIBC:crt0msg.obj
 0003:00132db0       ??_C@_0CM@OBIC@R6016?$AN?6?9?5not?5enough?5space?5for?5th@ 0063adb0   LIBC:crt0msg.obj
 0003:00132ddc       ??_C@_0CB@HPAL@?$AN?6abnormal?5program?5termination?$AN?6@ 0063addc   LIBC:crt0msg.obj
 0003:00132e00       ??_C@_0CM@JOOB@R6009?$AN?6?9?5not?5enough?5space?5for?5en@ 0063ae00   LIBC:crt0msg.obj
 0003:00132e2c       ??_C@_0CK@OIBL@R6008?$AN?6?9?5not?5enough?5space?5for?5ar@ 0063ae2c   LIBC:crt0msg.obj
 0003:00132e58       ??_C@_0CF@LKPB@R6002?$AN?6?9?5floating?5point?5not?5load@ 0063ae58   LIBC:crt0msg.obj
 0003:00132f08       __adbgmsg                  0063af08   LIBC:crt0msg.obj
 0003:00132f0c       ??_C@_0CF@JPDF@Microsoft?5Visual?5C?$CL?$CL?5Runtime?5Lib@ 0063af0c   LIBC:crt0msg.obj
 0003:00132f34       ??_C@_02JJJH@?6?6?$AA@     0063af34   LIBC:crt0msg.obj
 0003:00132f38       ??_C@_0BK@DEOK@Runtime?5Error?$CB?6?6Program?3?5?$AA@ 0063af38   LIBC:crt0msg.obj
 0003:00132f54       ??_C@_03NAME@?4?4?4?$AA@   0063af54   LIBC:crt0msg.obj
 0003:00132f58       ??_C@_0BH@NNCD@?$DMprogram?5name?5unknown?$DO?$AA@ 0063af58   LIBC:crt0msg.obj
 0003:00133108       __iob                      0063b108   LIBC:_file.obj
 0003:00133388       __cflush                   0063b388   LIBC:_file.obj
 0003:0013338c       __commode                  0063b38c   LIBC:ncommode.obj
 0003:00133390       __indefinite               0063b390   LIBC:87disp.obj
 0003:0013339a       __piby2                    0063b39a   LIBC:87disp.obj
 0003:001333ac       __cpower                   0063b3ac   LIBC:87disp.obj
 0003:001333c0       __infinity                 0063b3c0   LIBC:87tran.obj
 0003:001333ca       __minfinity                0063b3ca   LIBC:87tran.obj
 0003:001333d4       __logemax                  0063b3d4   LIBC:87tran.obj
 0003:00133404       __OP_POWjmptab             0063b404   LIBC:87tran.obj
 0003:00133454       __OP_LOG10jmptab           0063b454   LIBC:87tran.obj
 0003:00133474       __OP_LOGjmptab             0063b474   LIBC:87tran.obj
 0003:00133494       __OP_EXPjmptab             0063b494   LIBC:87tran.obj
 0003:001334b4       __newmode                  0063b4b4   LIBC:_newmode.obj
 0003:001334cc       ??_C@_0BD@NJFP@GetLastActivePopup?$AA@ 0063b4cc   LIBC:crtmbox.obj
 0003:001334e0       ??_C@_0BA@GILI@GetActiveWindow?$AA@ 0063b4e0   LIBC:crtmbox.obj
 0003:001334f0       ??_C@_0M@PKCK@MessageBoxA?$AA@ 0063b4f0   LIBC:crtmbox.obj
 0003:001334fc       ??_C@_0L@HKL@user32?4dll?$AA@ 0063b4fc   LIBC:crtmbox.obj
 0003:00133508       ??_C@_06PAPI@1?$CDQNAN?$AA@ 0063b508   LIBC:x10fout.obj
 0003:00133510       ??_C@_05BGNL@1?$CDINF?$AA@ 0063b510   LIBC:x10fout.obj
 0003:00133518       ??_C@_05EDPF@1?$CDIND?$AA@ 0063b518   LIBC:x10fout.obj
 0003:00133520       ??_C@_06LKFM@1?$CDSNAN?$AA@ 0063b520   LIBC:x10fout.obj
 0003:00133528       __fmode                    0063b528   LIBC:txtmode.obj
 0003:0013352c       ??_C@_03GAFO@_yn?$AA@      0063b52c   LIBC:fpexcept.obj
 0003:00133530       ??_C@_03GNLD@_y1?$AA@      0063b530   LIBC:fpexcept.obj
 0003:00133534       ??_C@_03MHCE@_y0?$AA@      0063b534   LIBC:fpexcept.obj
 0003:00133538       ??_C@_05PAK@frexp?$AA@     0063b538   LIBC:fpexcept.obj
 0003:00133540       ??_C@_04JKCH@fmod?$AA@     0063b540   LIBC:fpexcept.obj
 0003:00133548       ??_C@_06GGHF@_hypot?$AA@   0063b548   LIBC:fpexcept.obj
 0003:00133550       ??_C@_05JNMC@_cabs?$AA@    0063b550   LIBC:fpexcept.obj
 0003:00133558       ??_C@_05MEKH@ldexp?$AA@    0063b558   LIBC:fpexcept.obj
 0003:00133560       ??_C@_04KAOJ@modf?$AA@     0063b560   LIBC:fpexcept.obj
 0003:00133568       ??_C@_04EHAJ@fabs?$AA@     0063b568   LIBC:fpexcept.obj
 0003:00133570       ??_C@_05MFBN@floor?$AA@    0063b570   LIBC:fpexcept.obj
 0003:00133578       ??_C@_04JJMP@ceil?$AA@     0063b578   LIBC:fpexcept.obj
 0003:00133580       ??_C@_03JLPI@tan?$AA@      0063b580   LIBC:fpexcept.obj
 0003:00133584       ??_C@_03DLFL@cos?$AA@      0063b584   LIBC:fpexcept.obj
 0003:00133588       ??_C@_03JAMN@sin?$AA@      0063b588   LIBC:fpexcept.obj
 0003:0013358c       ??_C@_04LMBE@sqrt?$AA@     0063b58c   LIBC:fpexcept.obj
 0003:00133594       ??_C@_05BFPO@atan2?$AA@    0063b594   LIBC:fpexcept.obj
 0003:0013359c       ??_C@_04EAGN@atan?$AA@     0063b59c   LIBC:fpexcept.obj
 0003:001335a4       ??_C@_04OAMO@acos?$AA@     0063b5a4   LIBC:fpexcept.obj
 0003:001335ac       ??_C@_04ELFI@asin?$AA@     0063b5ac   LIBC:fpexcept.obj
 0003:001335b4       ??_C@_04LFAD@tanh?$AA@     0063b5b4   LIBC:fpexcept.obj
 0003:001335bc       ??_C@_04PFKD@cosh?$AA@     0063b5bc   LIBC:fpexcept.obj
 0003:001335c4       ??_C@_04NPAI@sinh?$AA@     0063b5c4   LIBC:fpexcept.obj
 0003:001335cc       ??_C@_05IJHH@log10?$AA@    0063b5cc   LIBC:fpexcept.obj
 0003:001335d4       ??_C@_03BGKD@log?$AA@      0063b5d4   LIBC:fpexcept.obj
 0003:001335d8       ??_C@_03EGFG@pow?$AA@      0063b5d8   LIBC:fpexcept.obj
 0003:001335dc       ??_C@_03CDGJ@exp?$AA@      0063b5dc   LIBC:fpexcept.obj
 0003:001336b8       __matherr_flag             0063b6b8   LIBC:matherr.obj
 0003:001336dc       ??_C@_01BJG@?6?$AA@        0063b6dc   LIBC:assert.obj
 0003:00133728       __d_inf                    0063b728   LIBC:util.obj
 0003:00133730       __d_ind                    0063b730   LIBC:util.obj
 0003:00133738       __d_max                    0063b738   LIBC:util.obj
 0003:00133740       __d_min                    0063b740   LIBC:util.obj
 0003:00133748       __d_mzero                  0063b748   LIBC:util.obj
 0003:00133750       __pow10pos                 0063b750   LIBC:constpow.obj
 0003:001338b0       __pow10neg                 0063b8b0   LIBC:constpow.obj
 0003:001342d8       ?buf@@3PADA                0063c2d8   LoadScrollBmp.obj
 0003:00134330       _ScrollBitmapTable         0063c330   LoadScrollBmp.obj
 0003:00135c88       ?_pnhHeap@@3P6AHI@ZA       0063dc88   LIBC:handler.obj
 0003:00135c90       _UserKey                   0063dc90   <common>
 0003:00135ce0       _InvY_l16                  0063dce0   <common>
 0003:0013dce0       _InvY_l8                   00645ce0   <common>
 0003:00145ce0       _nNext_scan                0064dce0   <common>
 0003:00146460       _MulAB                     0064e460   <common>
 0003:001c6460       _InvY                      006ce460   <common>
 0003:001ce460       _nBufferCount              006d6460   <common>
 0003:001ce464       _bUseSysMem                006d6464   <common>
 0003:001ce470       _gddpf                     006d6470   <common>
 0003:001ce490       _bColorFill                006d6490   <common>
 0003:001ce4a0       _PalSave                   006d64a0   <common>
 0003:001ce8a0       _bUseEmulation             006d68a0   <common>
 0003:001ce8a4       _net_continue_cur          006d68a4   <common>
 0003:001ce8a6       _LilkResultTimer           006d68a6   <common>
 0003:001ce8a8       _lpVRAM                    006d68a8   <common>
 0003:001ce8ac       _tm_scroll                 006d68ac   <common>
 0003:001ce8b0       _tm_scroll_all             006d68b0   <common>
 0003:001ce8b4       _tm_mode                   006d68b4   <common>
 0003:001ce8b8       _tm_scroll_back            006d68b8   <common>
 0003:001ce8bc       _bnum0                     006d68bc   <common>
 0003:001ce8bd       _bnum1                     006d68bd   <common>
 0003:001ce8be       _bnum2                     006d68be   <common>
 0003:001ce8bf       _bnum3                     006d68bf   <common>
 0003:001ce8c0       _bnum4                     006d68c0   <common>
 0003:001ce8c1       _fnum0                     006d68c1   <common>
 0003:001ce8c2       _fnum1                     006d68c2   <common>
 0003:001ce8c3       _fnum2                     006d68c3   <common>
 0003:001ce8c4       _fnum3                     006d68c4   <common>
 0003:001ce8c5       _fnum4                     006d68c5   <common>
 0003:001ce8c8       _ghost_flag                006d68c8   <common>
 0003:001ce8cc       _lank_disp_time            006d68cc   <common>
 0003:001ce8d0       _special_flag              006d68d0   <common>
 0003:001ce8d4       _ghost_cartype             006d68d4   <common>
 0003:001ce8d5       _ghost_setting             006d68d5   <common>
 0003:001ce8d8       _vs_stratos_flag           006d68d8   <common>
 0003:001ce8dc       _mirror_mode_flag          006d68dc   <common>
 0003:001ce8e0       _ghost_disp_time           006d68e0   <common>
 0003:001ce8e4       _ghost_mission             006d68e4   <common>
 0003:001ce8e8       _ghost_time                006d68e8   <common>
 0003:001ce8ec       _stratos_mode_flag         006d68ec   <common>
 0003:001ce8f0       _battle_scroll_all         006d68f0   <common>
 0003:001ce8f4       _battle_scroll             006d68f4   <common>
 0003:001ce8f8       _battle_scroll_back        006d68f8   <common>
 0003:001ce900       _line_2pscroll             006d6900   <common>
 0003:001cf260       _battle_mode               006d7260   <common>
 0003:001cf270       _ExTextureBuf              006d7270   <common>
 0003:005cf270       _ExTextureTbl              00ad7270   <common>
 0003:005d11b0       _AveCalcCount              00ad91b0   <common>
 0003:005d11b4       _AveDrawCount              00ad91b4   <common>
 0003:005d11b8       _mode_req                  00ad91b8   <common>
 0003:005d11bc       _GameOverCnt               00ad91bc   <common>
 0003:005d11c0       _PalTexture                00ad91c0   <common>
 0003:005d21c0       _option_mode               00ada1c0   <common>
 0003:005d21c4       _sup                       00ada1c4   <common>
 0003:005d21c6       _sdown                     00ada1c6   <common>
 0003:005d21c8       _option_scroll             00ada1c8   <common>
 0003:005d21cc       _option_scroll_back        00ada1cc   <common>
 0003:005d21d0       _option_scroll_all         00ada1d0   <common>
 0003:005d21d4       _staff_vpos_max            00ada1d4   <common>
 0003:005d21d8       _staff_vpos                00ada1d8   <common>
 0003:005d21dc       _staff_stop_wait           00ada1dc   <common>
 0003:005d21e0       _timecmp_laps_vs_save      00ada1e0   <common>
 0003:005d21e4       _scrobj_extend_wk          00ada1e4   <common>
 0003:005d21e8       _timecmp_vs_save           00ada1e8   <common>
 0003:005d21ec       _vs_cmpchk_sav             00ada1ec   <common>
 0003:005d21f0       _hTrack                    00ada1f0   <common>
 0003:005d21f4       _uCDDeviceID               00ada1f4   <common>
 0003:005d21f8       _dwParam1Play              00ada1f8   <common>
 0003:005d21fc       _TrackCnt                  00ada1fc   <common>
 0003:005d2200       _mciPP                     00ada200   <common>
 0003:005d2210       _logon_name                00ada210   <common>
 0003:005d2230       _gameok                    00ada230   <common>
 0003:005d2240       _machine_name              00ada240   <common>
 0003:005d2250       _player_name               00ada250   <common>
 0003:005d2270       _select_player             00ada270   <common>
 0003:005d2280       _ReceiveBuff               00ada280   <common>
 0003:007d2280       _nBytes                    00cda280   <common>
 0003:007d2290       _p2swdatabuf               00cda290   <common>
 0003:008d2290       _disp_flag                 00dda290   <common>
 0003:008d22a0       _enemy_name                00dda2a0   <common>
 0003:008d22c0       _dcoID                     00dda2c0   <common>
 0003:008d22c4       _gSWDTSize                 00dda2c4   <common>
 0003:008d22c8       _fromID                    00dda2c8   <common>
 0003:008d22d0       _DpGameName                00dda2d0   <common>
 0003:008d22f0       _g_lpGuid                  00dda2f0   <common>
 0003:008d2300       _p1swdatabuf               00dda300   <common>
 0003:009d2300       _cBuf                      00eda300   <common>
 0003:009d2700       _dphEvent                  00eda700   <common>
 0003:009d2704       _ghInst                    00eda704   <common>
 0003:009d2708       _dcoReceiveID              00eda708   <common>
 0003:009d270c       _org_gInputDevice          00eda70c   <common>
 0003:009d2710       _JoyConnect                00eda710   <common>
 0003:009d2720       _JoyInfoEx                 00eda720   <common>
 0003:009d2790       _load_buff                 00eda790   <common>
 0003:00afe7dc       _lpPauseBitmapBits         010067dc   <common>
 0003:00afe7e0       _lpPauseBitmapInfo         010067e0   <common>
 0003:00afe7e4       _CmdPtr                    010067e4   <common>
 0003:00afe7e8       _wGouraud                  010067e8   <common>
 0003:00afe7ec       _fxClientPerSuturn         010067ec   <common>
 0003:00afe7f0       _EVENT_STS_NET             010067f0   <common>
 0003:00b167f0       _VDP2_SYSREGS              0101e7f0   <common>
 0003:00b16910       _alpha_color_sav           0101e910   <common>
 0003:00b16920       _VDP1_VRAM                 0101e920   <common>
 0003:00bd6920       _SOUND_RAM                 010de920   <common>
 0003:00bd6928       _fyClientPerSuturn         010de928   <common>
 0003:00bd692c       _lpColor                   010de92c   <common>
 0003:00bd6930       _VDP1_SYSREGS              010de930   <common>
 0003:00bd6950       _fyPolyBase                010de950   <common>
 0003:00bd6960       _VDP2_VRAM1                010de960   <common>
 0003:00c56960       _VDP2_VRAM2                0115e960   <common>
 0003:00c57960       _WORK_RAM_H                0115f960   <common>
 0003:00d57960       _WORK_RAM_L                0125f960   <common>
 0003:00e57960       _lpFrameBuffCurrent        0135f960   <common>
 0003:00e57964       _wBankNo                   0135f964   <common>
 0003:00e57968       _fxPolyBase                0135f968   <common>
 0003:00e5796c       _bMaskPtn                  0135f96c   <common>
 0003:00e57970       _DummyTex4x4               0135f970   <common>
 0003:00e57990       _lpConvertBuf              0135f990   <common>
 0003:00e7d190       _CmdStack                  01385190   <common>
 0003:00e7d1e0       _Div_Rem                   013851e0   <common>
 0003:00e7d1e4       _bColorMode                013851e4   <common>
 0003:00e7d1f0       _ClipFramePoly             013851f0   <common>
 0003:00e7d240       _PalHist                   01385240   <common>
 0003:00e7d640       _Div_Quo                   01385640   <common>
 0003:00e7d644       _lpLookUp                  01385644   <common>
 0003:00e7d648       _result_sub_mode           01385648   <common>
 0003:00e7d64c       _menu_loop                 0138564c   <common>
 0003:00e7d650       _glpFrameBuff              01385650   <common>
 0003:00e7d654       _hBuffer                   01385654   <common>
 0003:00e7d658       _DATASIZE                  01385658   <common>
 0003:00e7d65c       _ACC                       0138565c   <common>
 0003:00e7d660       _lpDSBENG                  01385660   <common>
 0003:00e7d780       _WAVELIST                  01385780   <common>
 0003:00e7d898       _gWaveStatus               01385898   <common>
 0003:00e7d8a0       _lpDSB                     013858a0   <common>
 0003:00e7d9b8       _RPM                       013859b8   <common>
 0003:00e7d9bc       _pwavebank                 013859bc   <common>
 0003:00e7d9c0       _hWaveBuffer               013859c0   <common>
 0003:00e7d9c4       _AveFrameRateCount         013859c4   <common>
 0003:00e7d9c8       _lpClipper                 013859c8   <common>
 0003:00e7d9cc       _dwColorKey                013859cc   <common>
 0003:00e7d9d0       _FrameRateX                013859d0   <common>
 0003:00e7d9d4       _FullScreenBPP             013859d4   <common>
 0003:00e7d9d8       _gInputDevice              013859d8   <common>
 0003:00e7d9e0       _rcWindow                  013859e0   <common>
 0003:00e7d9f0       _lpBackBuffer              013859f0   <common>
 0003:00e7d9f4       _gMenuNo                   013859f4   <common>
 0003:00e7d9f8       _AveFrameRate              013859f8   <common>
 0003:00e7d9fc       _dwFrameCount              013859fc   <common>
 0003:00e7da00       _OrgBPP                    01385a00   <common>
 0003:00e7da04       _PixelShiftB               01385a04   <common>
 0003:00e7da08       _lpFrameRate               01385a08   <common>
 0003:00e7da0c       _PixelShiftG               01385a0c   <common>
 0003:00e7da10       _PixelShiftR               01385a10   <common>
 0003:00e7da20       _szFrameRate               01385a20   <common>
 0003:00e7daa0       _lpStretchBuffer           01385aa0   <common>
 0003:00e7daa8       _GameMode                  01385aa8   <common>
 0003:00e7dab0       _dwFrameTime               01385ab0   <common>
 0003:00e7dac0       _gszRallyEXEFullPath       01385ac0   <common>
 0003:00e7dbc0       _ScreenMode                01385bc0   <common>
 0003:00e7dbd0       _szInfo                    01385bd0   <common>
 0003:00e7dc50       _OrgWidth                  01385c50   <common>
 0003:00e7dc54       _OrgHeight                 01385c54   <common>
 0003:00e7dc58       _lpFrontBuffer             01385c58   <common>
 0003:00e7dc60       _GameRect                  01385c60   <common>
 0003:00e7dc70       _lpPalette                 01385c70   <common>
 0003:00e7dc74       _bPaused                   01385c74   <common>
 0003:00e7dc78       _dubugFlags                01385c78   <common>
 0003:00e7dc80       _GameSize                  01385c80   <common>
 0003:00e7dc88       _GameBPP                   01385c88   <common>
 0003:00e7dc8c       _bIsActive                 01385c8c   <common>
 0003:00e7dc90       _hWndMain                  01385c90   <common>
 0003:00e7dc98       _sizeINFO                  01385c98   <common>
 0003:00e7dca0       _dwFramesLast              01385ca0   <common>
 0003:00e7dca4       _lpInfo                    01385ca4   <common>
 0003:00e7dca8       _lpDD                      01385ca8   <common>
 0003:00e7dcac       _dwFrames                  01385cac   <common>
 0003:00e7dcb0       _bStretch                  01385cb0   <common>
 0003:00e7dcb8       _sizeFPS                   01385cb8   <common>
 0003:00e7dcc0       _GamePitch                 01385cc0   <common>
 0003:00e7dcc4       _pre_mis                   01385cc4   <common>
 0003:00e7dcc8       _setting_scroll_all        01385cc8   <common>
 0003:00e7dccc       _setting_mode              01385ccc   <common>
 0003:00e7dcd0       _pre_save                  01385cd0   <common>
 0003:00e7dcd4       _setting_scroll_back       01385cd4   <common>
 0003:00e7dcd8       _pre_tire                  01385cd8   <common>
 0003:00e7dce0       _TL                        01385ce0   <common>
 0003:00e7dd20       _pre_rsus                  01385d20   <common>
 0003:00e7dd24       _car_offset1               01385d24   <common>
 0003:00e7dd28       _car_offset2               01385d28   <common>
 0003:00e7dd30       _nFre                      01385d30   <common>
 0003:00e7dd70       _line_scroll               01385d70   <common>
 0003:00e7eb80       _pre_fsus                  01386b80   <common>
 0003:00e7eb84       _obj_offset                01386b84   <common>
 0003:00e7eb90       _PCM_TBL                   01386b90   <common>
 0003:00e7f390       _pre_blv                   01387390   <common>
 0003:00e7f394       _setting_scroll            01387394   <common>
 0003:00e7f398       _pre_hdl                   01387398   <common>
 0003:00e7f3a0       _MasterWaveFreq            013873a0   <common>
 0003:00e7f3e0       _NumModes                  013873e0   <common>
 0003:00e7f3e4       _scroll_num                013873e4   <common>
 0003:00e7f3f0       _OffBuffer                 013873f0   <common>
 0003:00e806b0       _ScrollBitmapTable16bit    013886b0   <common>
 0003:00e80730       _ModeList                  01388730   <common>
 0003:00e80be0       _sprite_window             01388be0   <common>
 0003:00e81540       _scroll_x                  01389540   <common>
 0003:00e817a0       _scroll_y                  013897a0   <common>
 0003:00e81a00       _cchange_color             01389a00   <common>
 0003:00e81c00       __nstream                  01389c00   <common>
 0003:00e81c04       ___piob                    01389c04   <common>
 0003:00e81c10       __bufin                    01389c10   <common>
 0003:00e82c10       __crtheap                  0138ac10   <common>
 0003:00e82c14       __nhandle                  0138ac14   <common>
 0003:00e82c20       ___pioinfo                 0138ac20   <common>
 0003:00e82d20       __acmdln                   0138ad20   <common>
 0003:00e82d24       ___onexitend               0138ad24   <common>
 0003:00e82d28       ___onexitbegin             0138ad28   <common>
 0004:00000000       __IMPORT_DESCRIPTOR_KERNEL32 0138b000   kernel32:KERNEL32.dll
 0004:00000014       __IMPORT_DESCRIPTOR_USER32 0138b014   user32:USER32.dll
 0004:00000028       __IMPORT_DESCRIPTOR_GDI32  0138b028   gdi32:GDI32.dll
 0004:0000003c       __IMPORT_DESCRIPTOR_COMCTL32 0138b03c   comctl32:COMCTL32.dll
 0004:00000050       __IMPORT_DESCRIPTOR_ADVAPI32 0138b050   advapi32:ADVAPI32.dll
 0004:00000064       __IMPORT_DESCRIPTOR_WINMM  0138b064   winmm:WINMM.dll
 0004:00000078       __IMPORT_DESCRIPTOR_LZ32   0138b078   lz32:LZ32.dll
 0004:0000008c       __IMPORT_DESCRIPTOR_DDRAW  0138b08c   ddraw:DDRAW.dll
 0004:000000a0       __IMPORT_DESCRIPTOR_DSOUND 0138b0a0   dsound:DSOUND.dll
 0004:000000b4       __IMPORT_DESCRIPTOR_DPLAYX 0138b0b4   dplayx:DPLAYX.dll
 0004:000000c8       __NULL_IMPORT_DESCRIPTOR   0138b0c8   kernel32:KERNEL32.dll
 0004:000003b4       __imp__RegCreateKeyExA@36  0138b3b4   advapi32:ADVAPI32.dll
 0004:000003b8       __imp__RegOpenKeyExA@20    0138b3b8   advapi32:ADVAPI32.dll
 0004:000003bc       __imp__RegQueryValueExA@24 0138b3bc   advapi32:ADVAPI32.dll
 0004:000003c0       \177ADVAPI32_NULL_THUNK_DATA 0138b3c0   advapi32:ADVAPI32.dll
 0004:000003c4       __imp__PropertySheetA@4    0138b3c4   comctl32:COMCTL32.dll
 0004:000003c8       __imp__InitCommonControls@0 0138b3c8   comctl32:COMCTL32.dll
 0004:000003cc       \177COMCTL32_NULL_THUNK_DATA 0138b3cc   comctl32:COMCTL32.dll
 0004:000003d0       __imp__DirectDrawCreate@12 0138b3d0   ddraw:DDRAW.dll
 0004:000003d4       \177DDRAW_NULL_THUNK_DATA  0138b3d4   ddraw:DDRAW.dll
 0004:000003d8       __imp__DirectPlayEnumerateA@8 0138b3d8   dplayx:DPLAYX.dll
 0004:000003dc       __imp__DirectPlayCreate@12 0138b3dc   dplayx:DPLAYX.dll
 0004:000003e0       \177DPLAYX_NULL_THUNK_DATA 0138b3e0   dplayx:DPLAYX.dll
 0004:000003e4       __imp__DirectSoundCreate@12 0138b3e4   dsound:DSOUND.dll
 0004:000003e8       \177DSOUND_NULL_THUNK_DATA 0138b3e8   dsound:DSOUND.dll
 0004:000003ec       __imp__SetBkMode@8         0138b3ec   gdi32:GDI32.dll
 0004:000003f0       __imp__DeleteObject@4      0138b3f0   gdi32:GDI32.dll
 0004:000003f4       __imp__GetDeviceCaps@8     0138b3f4   gdi32:GDI32.dll
 0004:000003f8       __imp__SetPixel@16         0138b3f8   gdi32:GDI32.dll
 0004:000003fc       __imp__StretchBlt@44       0138b3fc   gdi32:GDI32.dll
 0004:00000400       __imp__ExtTextOutA@32      0138b400   gdi32:GDI32.dll
 0004:00000404       __imp__SetBkColor@8        0138b404   gdi32:GDI32.dll
 0004:00000408       __imp__SetTextColor@8      0138b408   gdi32:GDI32.dll
 0004:0000040c       __imp__SelectObject@8      0138b40c   gdi32:GDI32.dll
 0004:00000410       __imp__GetTextExtentPointA@16 0138b410   gdi32:GDI32.dll
 0004:00000414       __imp__TextOutA@20         0138b414   gdi32:GDI32.dll
 0004:00000418       __imp__CreateFontA@56      0138b418   gdi32:GDI32.dll
 0004:0000041c       __imp__GetStockObject@4    0138b41c   gdi32:GDI32.dll
 0004:00000420       __imp__GetPixel@12         0138b420   gdi32:GDI32.dll
 0004:00000424       __imp__Polyline@12         0138b424   gdi32:GDI32.dll
 0004:00000428       __imp__SetDIBitsToDevice@48 0138b428   gdi32:GDI32.dll
 0004:0000042c       __imp__SetStretchBltMode@8 0138b42c   gdi32:GDI32.dll
 0004:00000430       __imp__StretchDIBits@52    0138b430   gdi32:GDI32.dll
 0004:00000434       __imp__Polygon@12          0138b434   gdi32:GDI32.dll
 0004:00000438       \177GDI32_NULL_THUNK_DATA  0138b438   gdi32:GDI32.dll
 0004:0000043c       __imp__LocalFree@4         0138b43c   kernel32:KERNEL32.dll
 0004:00000440       __imp__LocalAlloc@8        0138b440   kernel32:KERNEL32.dll
 0004:00000444       __imp___lwrite@12          0138b444   kernel32:KERNEL32.dll
 0004:00000448       __imp__OpenFile@12         0138b448   kernel32:KERNEL32.dll
 0004:0000044c       __imp___lread@12           0138b44c   kernel32:KERNEL32.dll
 0004:00000450       __imp___llseek@12          0138b450   kernel32:KERNEL32.dll
 0004:00000454       __imp__WriteFile@20        0138b454   kernel32:KERNEL32.dll
 0004:00000458       __imp__GetFileSize@8       0138b458   kernel32:KERNEL32.dll
 0004:0000045c       __imp__GetLogicalDrives@0  0138b45c   kernel32:KERNEL32.dll
 0004:00000460       __imp__GetDriveTypeA@4     0138b460   kernel32:KERNEL32.dll
 0004:00000464       __imp__lstrcpyA@8          0138b464   kernel32:KERNEL32.dll
 0004:00000468       __imp__WritePrivateProfileStringA@16 0138b468   kernel32:KERNEL32.dll
 0004:0000046c       __imp__SetFilePointer@16   0138b46c   kernel32:KERNEL32.dll
 0004:00000470       __imp__FlushFileBuffers@4  0138b470   kernel32:KERNEL32.dll
 0004:00000474       __imp__SetStdHandle@8      0138b474   kernel32:KERNEL32.dll
 0004:00000478       __imp__HeapCreate@12       0138b478   kernel32:KERNEL32.dll
 0004:0000047c       __imp__GetStdHandle@4      0138b47c   kernel32:KERNEL32.dll
 0004:00000480       __imp__GetFileType@4       0138b480   kernel32:KERNEL32.dll
 0004:00000484       __imp__SetHandleCount@4    0138b484   kernel32:KERNEL32.dll
 0004:00000488       __imp__GetOEMCP@0          0138b488   kernel32:KERNEL32.dll
 0004:0000048c       __imp__GetACP@0            0138b48c   kernel32:KERNEL32.dll
 0004:00000490       __imp__GetCPInfo@8         0138b490   kernel32:KERNEL32.dll
 0004:00000494       __imp__GetEnvironmentStringsW@0 0138b494   kernel32:KERNEL32.dll
 0004:00000498       __imp__FreeEnvironmentStringsW@4 0138b498   kernel32:KERNEL32.dll
 0004:0000049c       __imp__GetEnvironmentStrings@0 0138b49c   kernel32:KERNEL32.dll
 0004:000004a0       __imp__FreeEnvironmentStringsA@4 0138b4a0   kernel32:KERNEL32.dll
 0004:000004a4       __imp__GetModuleFileNameA@12 0138b4a4   kernel32:KERNEL32.dll
 0004:000004a8       __imp__UnhandledExceptionFilter@4 0138b4a8   kernel32:KERNEL32.dll
 0004:000004ac       __imp__LCMapStringW@24     0138b4ac   kernel32:KERNEL32.dll
 0004:000004b0       __imp__WideCharToMultiByte@32 0138b4b0   kernel32:KERNEL32.dll
 0004:000004b4       __imp__LCMapStringA@24     0138b4b4   kernel32:KERNEL32.dll
 0004:000004b8       __imp__MultiByteToWideChar@24 0138b4b8   kernel32:KERNEL32.dll
 0004:000004bc       __imp__HeapAlloc@12        0138b4bc   kernel32:KERNEL32.dll
 0004:000004c0       __imp__GetLastError@0      0138b4c0   kernel32:KERNEL32.dll
 0004:000004c4       __imp__HeapFree@12         0138b4c4   kernel32:KERNEL32.dll
 0004:000004c8       __imp__LoadLibraryA@4      0138b4c8   kernel32:KERNEL32.dll
 0004:000004cc       __imp__GetProcAddress@8    0138b4cc   kernel32:KERNEL32.dll
 0004:000004d0       __imp__GetVersion@0        0138b4d0   kernel32:KERNEL32.dll
 0004:000004d4       __imp__GetCommandLineA@0   0138b4d4   kernel32:KERNEL32.dll
 0004:000004d8       __imp__GetStartupInfoA@4   0138b4d8   kernel32:KERNEL32.dll
 0004:000004dc       __imp__GetModuleHandleA@4  0138b4dc   kernel32:KERNEL32.dll
 0004:000004e0       __imp__RtlUnwind@16        0138b4e0   kernel32:KERNEL32.dll
 0004:000004e4       __imp__ExitProcess@4       0138b4e4   kernel32:KERNEL32.dll
 0004:000004e8       __imp__GlobalUnlock@4      0138b4e8   kernel32:KERNEL32.dll
 0004:000004ec       __imp__GlobalFree@4        0138b4ec   kernel32:KERNEL32.dll
 0004:000004f0       __imp__lstrlenA@4          0138b4f0   kernel32:KERNEL32.dll
 0004:000004f4       __imp__GlobalLock@4        0138b4f4   kernel32:KERNEL32.dll
 0004:000004f8       __imp__GlobalAlloc@8       0138b4f8   kernel32:KERNEL32.dll
 0004:000004fc       __imp__OutputDebugStringA@4 0138b4fc   kernel32:KERNEL32.dll
 0004:00000500       __imp__CloseHandle@4       0138b500   kernel32:KERNEL32.dll
 0004:00000504       __imp__RaiseException@16   0138b504   kernel32:KERNEL32.dll
 0004:00000508       __imp__GetStringTypeA@20   0138b508   kernel32:KERNEL32.dll
 0004:0000050c       __imp__GetStringTypeW@16   0138b50c   kernel32:KERNEL32.dll
 0004:00000510       __imp__SetUnhandledExceptionFilter@4 0138b510   kernel32:KERNEL32.dll
 0004:00000514       __imp__IsBadReadPtr@8      0138b514   kernel32:KERNEL32.dll
 0004:00000518       __imp__IsBadWritePtr@8     0138b518   kernel32:KERNEL32.dll
 0004:0000051c       __imp__GlobalHandle@4      0138b51c   kernel32:KERNEL32.dll
 0004:00000520       __imp__IsBadCodePtr@4      0138b520   kernel32:KERNEL32.dll
 0004:00000524       __imp__SetEndOfFile@4      0138b524   kernel32:KERNEL32.dll
 0004:00000528       __imp___lclose@4           0138b528   kernel32:KERNEL32.dll
 0004:0000052c       __imp__HeapReAlloc@16      0138b52c   kernel32:KERNEL32.dll
 0004:00000530       __imp__HeapSize@12         0138b530   kernel32:KERNEL32.dll
 0004:00000534       __imp___lopen@8            0138b534   kernel32:KERNEL32.dll
 0004:00000538       __imp__lstrcatA@8          0138b538   kernel32:KERNEL32.dll
 0004:0000053c       __imp__ReadFile@20         0138b53c   kernel32:KERNEL32.dll
 0004:00000540       __imp__CreateFileA@28      0138b540   kernel32:KERNEL32.dll
 0004:00000544       __imp__lstrcmpA@8          0138b544   kernel32:KERNEL32.dll
 0004:00000548       __imp__GetPrivateProfileStringA@24 0138b548   kernel32:KERNEL32.dll
 0004:0000054c       \177KERNEL32_NULL_THUNK_DATA 0138b54c   kernel32:KERNEL32.dll
 0004:00000550       __imp__LZSeek@12           0138b550   lz32:LZ32.dll
 0004:00000554       __imp__LZRead@12           0138b554   lz32:LZ32.dll
 0004:00000558       __imp__LZOpenFileA@12      0138b558   lz32:LZ32.dll
 0004:0000055c       __imp__LZClose@4           0138b55c   lz32:LZ32.dll
 0004:00000560       \177LZ32_NULL_THUNK_DATA   0138b560   lz32:LZ32.dll
 0004:00000564       __imp__IsIconic@4          0138b564   user32:USER32.dll
 0004:00000568       __imp__SetWindowLongA@12   0138b568   user32:USER32.dll
 0004:0000056c       __imp__DefWindowProcA@16   0138b56c   user32:USER32.dll
 0004:00000570       __imp__GetWindowRect@8     0138b570   user32:USER32.dll
 0004:00000574       __imp__DestroyMenu@4       0138b574   user32:USER32.dll
 0004:00000578       __imp__GetDC@4             0138b578   user32:USER32.dll
 0004:0000057c       __imp__PostMessageA@16     0138b57c   user32:USER32.dll
 0004:00000580       __imp__WinHelpA@16         0138b580   user32:USER32.dll
 0004:00000584       __imp__wsprintfA           0138b584   user32:USER32.dll
 0004:00000588       __imp__SystemParametersInfoA@16 0138b588   user32:USER32.dll
 0004:0000058c       __imp__BeginPaint@8        0138b58c   user32:USER32.dll
 0004:00000590       __imp__ClientToScreen@8    0138b590   user32:USER32.dll
 0004:00000594       __imp__GetClientRect@8     0138b594   user32:USER32.dll
 0004:00000598       __imp__GetSystemMetrics@4  0138b598   user32:USER32.dll
 0004:0000059c       __imp__PostQuitMessage@4   0138b59c   user32:USER32.dll
 0004:000005a0       __imp__GetWindowLongA@8    0138b5a0   user32:USER32.dll
 0004:000005a4       __imp__AdjustWindowRectEx@16 0138b5a4   user32:USER32.dll
 0004:000005a8       __imp__SetWindowPos@28     0138b5a8   user32:USER32.dll
 0004:000005ac       __imp__SetRect@20          0138b5ac   user32:USER32.dll
 0004:000005b0       __imp__SetCursor@4         0138b5b0   user32:USER32.dll
 0004:000005b4       __imp__ShowCursor@4        0138b5b4   user32:USER32.dll
 0004:000005b8       __imp__EndPaint@8          0138b5b8   user32:USER32.dll
 0004:000005bc       __imp__GetAsyncKeyState@4  0138b5bc   user32:USER32.dll
 0004:000005c0       __imp__CheckDlgButton@12   0138b5c0   user32:USER32.dll
 0004:000005c4       __imp__IsDlgButtonChecked@8 0138b5c4   user32:USER32.dll
 0004:000005c8       __imp__GetDlgItemTextA@16  0138b5c8   user32:USER32.dll
 0004:000005cc       __imp__SendDlgItemMessageA@20 0138b5cc   user32:USER32.dll
 0004:000005d0       __imp__SendMessageA@16     0138b5d0   user32:USER32.dll
 0004:000005d4       __imp__SetTimer@16         0138b5d4   user32:USER32.dll
 0004:000005d8       __imp__SetDlgItemTextA@12  0138b5d8   user32:USER32.dll
 0004:000005dc       __imp__GetDlgItem@8        0138b5dc   user32:USER32.dll
 0004:000005e0       __imp__EnableWindow@8      0138b5e0   user32:USER32.dll
 0004:000005e4       __imp__KillTimer@8         0138b5e4   user32:USER32.dll
 0004:000005e8       __imp__EndDialog@8         0138b5e8   user32:USER32.dll
 0004:000005ec       __imp__DialogBoxParamA@20  0138b5ec   user32:USER32.dll
 0004:000005f0       __imp__LoadMenuA@8         0138b5f0   user32:USER32.dll
 0004:000005f4       __imp__SetMenu@8           0138b5f4   user32:USER32.dll
 0004:000005f8       __imp__CheckMenuItem@12    0138b5f8   user32:USER32.dll
 0004:000005fc       __imp__GetWindowThreadProcessId@8 0138b5fc   user32:USER32.dll
 0004:00000600       __imp__GetWindowTextA@12   0138b600   user32:USER32.dll
 0004:00000604       __imp__CharUpperBuffA@8    0138b604   user32:USER32.dll
 0004:00000608       __imp__MessageBoxA@16      0138b608   user32:USER32.dll
 0004:0000060c       __imp__GetMenu@4           0138b60c   user32:USER32.dll
 0004:00000610       __imp__GetSubMenu@8        0138b610   user32:USER32.dll
 0004:00000614       __imp__ModifyMenuA@20      0138b614   user32:USER32.dll
 0004:00000618       __imp__EnableMenuItem@12   0138b618   user32:USER32.dll
 0004:0000061c       __imp__DrawMenuBar@4       0138b61c   user32:USER32.dll
 0004:00000620       __imp__EnumWindows@8       0138b620   user32:USER32.dll
 0004:00000624       __imp__LoadIconA@8         0138b624   user32:USER32.dll
 0004:00000628       __imp__LoadCursorA@8       0138b628   user32:USER32.dll
 0004:0000062c       __imp__RegisterClassA@4    0138b62c   user32:USER32.dll
 0004:00000630       __imp__CreateWindowExA@48  0138b630   user32:USER32.dll
 0004:00000634       __imp__UpdateWindow@4      0138b634   user32:USER32.dll
 0004:00000638       __imp__SetFocus@4          0138b638   user32:USER32.dll
 0004:0000063c       __imp__GetMessageA@16      0138b63c   user32:USER32.dll
 0004:00000640       __imp__TranslateMessage@4  0138b640   user32:USER32.dll
 0004:00000644       __imp__PeekMessageA@20     0138b644   user32:USER32.dll
 0004:00000648       __imp__DispatchMessageA@4  0138b648   user32:USER32.dll
 0004:0000064c       __imp__WaitMessage@0       0138b64c   user32:USER32.dll
 0004:00000650       __imp__InvalidateRect@12   0138b650   user32:USER32.dll
 0004:00000654       __imp__GetForegroundWindow@0 0138b654   user32:USER32.dll
 0004:00000658       __imp__ReleaseDC@8         0138b658   user32:USER32.dll
 0004:0000065c       \177USER32_NULL_THUNK_DATA 0138b65c   user32:USER32.dll
 0004:00000660       __imp__mmioOpenA@12        0138b660   winmm:WINMM.dll
 0004:00000664       __imp__mciSendCommandA@16  0138b664   winmm:WINMM.dll
 0004:00000668       __imp__joyGetPosEx@8       0138b668   winmm:WINMM.dll
 0004:0000066c       __imp__joyGetNumDevs@0     0138b66c   winmm:WINMM.dll
 0004:00000670       __imp__joyGetDevCapsA@12   0138b670   winmm:WINMM.dll
 0004:00000674       __imp__mmioDescend@16      0138b674   winmm:WINMM.dll
 0004:00000678       __imp__mmioAscend@12       0138b678   winmm:WINMM.dll
 0004:0000067c       __imp__mmioRead@12         0138b67c   winmm:WINMM.dll
 0004:00000680       __imp__mmioClose@8         0138b680   winmm:WINMM.dll
 0004:00000684       __imp__timeGetTime@0       0138b684   winmm:WINMM.dll
 0004:00000688       \177WINMM_NULL_THUNK_DATA  0138b688   winmm:WINMM.dll

 entry point at        0001:000fd5e0

 Static symbols

 0001:000fb798       $$$$$$00001                004fc798 f PHOTOCTRL.obj
 0001:000faf90       $$$$$$00001                004fbf90 f REC_R.obj
 0001:000f97a0       $$$$$$00001                004fa7a0 f ANIMAL.obj
 0001:000f4fd8       $$$$$$00001                004f5fd8 f CS_MD_SELECT.obj
 0001:000f4b24       $$$$$$00001                004f5b24 f SOUND.obj
 0001:000efd80       $$$$$$00001                004f0d80 f PLAYER.obj
 0001:000ed7e4       $$$$$$00001                004ee7e4 f REC_MAIN.obj
 0001:000ebee4       $$$$$$00001                004ecee4 f GAME.obj
 0001:000e9684       $$$$$$00001                004ea684 f GAMESD.obj
 0001:000e8ae8       $$$$$$00001                004e9ae8 f CLROFFSET.obj
 0001:000e7384       $$$$$$00001                004e8384 f CS_SETTING_PSET.obj
 0001:000e7238       $$$$$$00001                004e8238 f SLAVE.obj
 0001:000e6988       $$$$$$00001                004e7988 f SWITCH.obj
 0001:000e0720       $$$$$$00001                004e1720 f LAPTIME.obj
 0001:000df568       $$$$$$00001                004e0568 f EXTRACT.obj
 0001:000dd2fc       $$$$$$00001                004de2fc f HELI.obj
 0001:000dd0f4       $$$$$$00001                004de0f4 f ERROR.obj
 0001:000dcb00       $$$$$$00001                004ddb00 f scroll.obj
 0001:000d9898       $$$$$$00001                004da898 f AC_C_SELECT.obj
 0001:000d947c       $$$$$$00001                004da47c f REC_RTXX.obj
 0001:000d8ea0       $$$$$$00001                004d9ea0 f NEXT.obj
 0001:000d85b0       $$$$$$00001                004d95b0 f TITLEwatanabe.obj
 0001:000d7b70       $$$$$$00001                004d8b70 f REC_CHANGE.obj
 0001:000d5788       $$$$$$00001                004d6788 f DEBUG.obj
 0001:000d428c       $$$$$$00001                004d528c f PAD.obj
 0001:000d3600       $$$$$$00001                004d4600 f LIGHT.obj
 0001:000d2ef0       $$$$$$00001                004d3ef0 f blinkle.obj
 0001:000d01ec       $$$$$$00001                004d11ec f PHOTO.obj
 0001:000cfad4       $$$$$$00001                004d0ad4 f timer.obj
 0001:000cf578       $$$$$$00001                004d0578 f BUP_MELT.obj
 0001:000cf0b0       $$$$$$00001                004d00b0 f REC_RT.obj
 0001:000ce854       $$$$$$00001                004cf854 f CS_CAR_SET.obj
 0001:000ca0b0       $$$$$$00001                004cb0b0 f CS_TM_ATTCK.obj
 0001:000c8ff4       $$$$$$00001                004c9ff4 f LINE_SCRL.obj
 0001:000c8fec       $$$$$$00001                004c9fec f CACHE.obj
 0001:000c6378       $$$$$$00001                004c7378 f OTHERCAR.obj
 0001:000c5f94       $$$$$$00001                004c6f94 f REC_RAP.obj
 0001:000c5550       $$$$$$00001                004c6550 f CS_PICT_SET.obj
 0001:000c3850       $$$$$$00001                004c4850 f NAME_EXIT.obj
 0001:000c0280       $$$$$$00001                004c1280 f AC_CRS_SELECT.obj
 0001:000bd850       $$$$$$00001                004be850 f REC_MARKACT.obj
 0001:000b96c0       $$$$$$00001                004ba6c0 f MATRIX.obj
 0001:000b749c       $$$$$$00001                004b849c f OTHERCTRL.obj
 0001:000b5478       $$$$$$00001                004b6478 f COPRO.obj
 0001:000b4efc       $$$$$$00001                004b5efc f REC_RTX.obj
 0001:000b363c       $$$$$$00001                004b463c f MATH.obj
 0001:000b3350       $$$$$$00001                004b4350 f REC_RACX.obj
 0001:000b2a7c       $$$$$$00001                004b3a7c f REC_RAC.obj
 0001:000b0e44       $$$$$$00001                004b1e44 f CS_TM_ATT_PSET.obj
 0001:000acb94       $$$$$$00001                004adb94 f OTHERSET.obj
 0001:000aa1d0       $$$$$$00001                004ab1d0 f CARCTRL.obj
 0001:000a4fc0       $$$$$$00001                004a5fc0 f MOTION.obj
 0001:000a3300       $$$$$$00001                004a4300 f ZSORT.obj
 0001:000a3288       $$$$$$00001                004a4288 f SHADING.obj
 0001:000a3260       $$$$$$00001                004a4260 f NAME_DISP.obj
 0001:000a27b0       $$$$$$00001                004a37b0 f NAME_MOJI.obj
 0001:0009c438       $$$$$$00001                0049d438 f GCTRL.obj
 0001:0009c0d4       $$$$$$00001                0049d0d4 f REC_MODEDISP.obj
 0001:00099114       $$$$$$00001                0049a114 f INIT.obj
 0001:000974c0       $$$$$$00001                004984c0 f TITLEhori.obj
 0001:00096174       $$$$$$00001                00497174 f GENERATOR.obj
 0001:00095000       $$$$$$00001                00496000 f RES_MAIN.obj
 0001:00093038       $$$$$$00001                00494038 f REC_ASORT.obj
 0001:00091d8c       $$$$$$00001                00492d8c f INT.obj
 0001:0008fc34       $$$$$$00001                00490c34 f PUBLIC.obj
 0001:0008f5a8       $$$$$$00001                004905a8 f REC_MOJIACT.obj
 0001:0008e5c8       $$$$$$00001                0048f5c8 f CS_POLY_SET.obj
 0001:0008e0e0       $$$$$$00001                0048f0e0 f REC_CMARKACT.obj
 0001:0008d324       $$$$$$00001                0048e324 f REC_MENU.obj
 0001:0008d02c       $$$$$$00001                0048e02c f REC_CORACT.obj
 0001:0008cb54       $$$$$$00001                0048db54 f RES2_TIMEACT.obj
 0001:0008c2b0       $$$$$$00001                0048d2b0 f STARTwatanabe.obj
 0001:00089298       $$$$$$00001                0048a298 f CAMERA.obj
 0001:00089230       $$$$$$00001                0048a230 f TITLEtoya.obj
 0001:00087cd0       $$$$$$00001                00488cd0 f SPLASH.obj
 0001:00086f2c       $$$$$$00001                00487f2c f VARIETY.obj
 0001:00086f10       $$$$$$00001                00487f10 f APPINIT.obj
 0001:000824bc       $$$$$$00001                004834bc f NAME_SELMOJI.obj
 0001:000802f0       $$$$$$00001                004812f0 f ADVCTRL.obj
 0001:0007ba08       $$$$$$00001                0047ca08 f ETCSUB.obj
 0001:0007a384       $$$$$$00001                0047b384 f BUP_FREEZE.obj
 0001:0007907c       $$$$$$00001                0047a07c f OPT_DISP.obj
 0001:00076ab4       $$$$$$00001                00477ab4 f DISPCAR.obj
 0001:0006eff0       $$$$$$00001                0046fff0 f MKPOLY.obj
 0001:000682e0       _put_time                  004692e0 f Scrlobj.obj
 0001:0006d910       _put_time_result           0046e910 f Scrlobj.obj
 0001:0006ef00       _put_pause                 0046ff00 f Scrlobj.obj
 0001:00065ea0       $$$$$$00001                00466ea0 f REC_RTXXX.obj
 0001:000621c4       $$$$$$00001                004631c4 f x_result.obj
 0001:00060050       $$$$$$00001                00461050 f ADV.obj
 0001:0005d981       $$$$$$00001                0045e981 f CINTF.obj
 0001:0005d2f8       $$$$$$00001                0045e2f8 f REC_SCRACT.obj
 0001:000598c4       $$$$$$00001                0045a8c4 f NAME_MAIN.obj
 0001:00054230       $$$$$$00001                00455230 f display2.obj
 0001:00052fd8       $$$$$$00001                00453fd8 f POLY_SET.obj
 0001:00052ca4       $$$$$$00001                00453ca4 f EVENT.obj
 0001:00052870       $$$$$$00001                00453870 f VDP.obj
 0001:000519e4       $$$$$$00001                004529e4 f REC_DATASET.obj
 0001:0005143c       $$$$$$00001                0045243c f REC_MENU2.obj
 0001:0004ff0c       $$$$$$00001                00450f0c f AC_PICT_SET.obj
 0001:0004fae0       $$$$$$00001                00450ae0 f ACTION.obj
 0001:0004f074       $$$$$$00001                00450074 f GF_SUB.obj
 0001:0004d0f4       $$$$$$00001                0044e0f4 f AC_G_SELECT.obj
 0001:0004cdc0       $$$$$$00001                0044ddc0 f BOOT.obj
 0001:0004965c       $$$$$$00001                0044a65c f CEREMONY.obj
 0001:00048ce4       $$$$$$00001                00449ce4 f STARThattori.obj
 0001:000477f8       $$$$$$00001                004487f8 f DSP.obj
 0001:00045690       $$$$$$00001                00446690 f POWER.obj
 0001:0004464c       $$$$$$00001                0044564c f STEER.obj
 0001:00043134       $$$$$$00001                00444134 f BALLDEMO.obj
 0001:000416fc       $$$$$$00001                004426fc f CARCOLI.obj
 0001:00040a00       $$$$$$00001                00441a00 f RES2_MAIN.obj
 0001:0003a420       $$$$$$00001                0043b420 f CLIP2D.obj
 0001:00039770       $$$$$$00001                0043a770 f REC_DISP.obj
 0001:00033700       $$$$$$00001                00434700 f SCRLMOVE.obj
 0001:0002ec80       $$$$$$00001                0042fc80 f REC_REQUEST.obj
 0001:0002d9d4       $$$$$$00001                0042e9d4 f REC_TSORT.obj
 0001:0002af18       $$$$$$00001                0042bf18 f CS_BATTLE_2P_PSET.obj
 0001:0002a520       $$$$$$00001                0042b520 f EXTDATA.obj
 0001:0002649c       $$$$$$00001                0042749c f CAR.obj
 0001:00022a44       $$$$$$00001                00423a44 f OTHERSUB.obj
 0001:0001d258       $$$$$$00001                0041e258 f display3.obj
 0001:0001b238       $$$$$$00001                0041c238 f REC_CONNECT.obj
 0001:0001aa70       $$$$$$00001                0041ba70 f SPRITE.obj
 0001:0001a3ac       $$$$$$00001                0041b3ac f ETC.obj
 0001:00019c3c       $$$$$$00001                0041ac3c f RES_TIMEACT.obj
 0001:00019a04       $$$$$$00001                0041aa04 f RES2_PLAYER.obj
 0001:00010014       $$$$$$00001                00411014 f ENDING.obj
 0001:0000e070       $$$$$$00001                0040f070 f display.obj
 0001:0000ac90       $$$$$$00001                0040bc90 f SAMPLE.obj
 0001:00008d5c       $$$$$$00001                00409d5c f tmp.obj
 0001:00008bf4       $$$$$$00001                00409bf4 f NAME_CAR.obj
 0001:00005b4c       $$$$$$00001                00406b4c f CS_SETTING.obj
 0001:000053a8       $$$$$$00001                004063a8 f REC_RA.obj
 0001:00004aac       $$$$$$00001                00405aac f RES_CMARKACT.obj
 0001:00000000       $$$$$$00001                00401000 f PLCTRL.obj
 0001:00105080       _siglookup                 00506080 f LIBC:winsig.obj
 0001:001032e0       _$E2                       005042e0 f LIBC:unhandld.obj
 0001:001032f0       _$E1                       005042f0 f LIBC:unhandld.obj
 0001:00101380       __abstract_cw              00502380 f LIBC:ieee87.obj
 0001:00101430       __hw_cw                    00502430 f LIBC:ieee87.obj
 0001:00100d20       _getSystemCP               00501d20 f LIBC:mbctype.obj
 0001:00100d70       _CPtoLCID                  00501d70 f LIBC:mbctype.obj
 0001:00100dd0       _setSBCS                   00501dd0 f LIBC:mbctype.obj
 0001:001007c0       _parse_cmdline             005017c0 f LIBC:stdargv.obj
 0001:00100600       _x_ismbbtype               00501600 f LIBC:ismbbyte.obj
 0001:001005b0       _xcptlookup                005015b0 f LIBC:winxfltr.obj
 0001:000ff960       ?FindHandler@@YAXPAUEHExceptionRecord@@PAUEHRegistrationNode@@PAU_CONTEXT@@PAXPBU_s_FuncInfo@@EH1@Z 00500960 f LIBC:frame.obj
 0001:000ffc00       ?FindHandlerForForeignException@@YAXPAUEHExceptionRecord@@PAUEHRegistrationNode@@PAU_CONTEXT@@PAXPBU_s_FuncInfo@@HH1@Z 00500c00 f LIBC:frame.obj
 0001:000ffce0       ?GetRangeOfTrysToCheck@@YAPBU_s_TryBlockMapEntry@@PBU_s_FuncInfo@@HHPAI1@Z 00500ce0 f LIBC:frame.obj
 0001:000ffe50       ?FrameUnwindFilter@@YAHPAU_EXCEPTION_POINTERS@@@Z 00500e50 f LIBC:frame.obj
 0001:000ffe70       ?CatchIt@@YAXPAUEHExceptionRecord@@PAUEHRegistrationNode@@PAU_CONTEXT@@PAXPBU_s_FuncInfo@@PBU_s_HandlerType@@PBU_s_CatchableType@@PBU_s_TryBlockMapEntry@@H1@Z 00500e70 f LIBC:frame.obj
 0001:000fff10       ?CallCatchBlock@@YAPAXPAUEHExceptionRecord@@PAUEHRegistrationNode@@PAU_CONTEXT@@PBU_s_FuncInfo@@PAXHK@Z 00500f10 f LIBC:frame.obj
 0001:00100020       ?ExFilterRethrow@@YAHPAU_EXCEPTION_POINTERS@@@Z 00501020 f LIBC:frame.obj
 0001:00100050       ?BuildCatchObject@@YAXPAUEHExceptionRecord@@PAUEHRegistrationNode@@PBU_s_HandlerType@@PBU_s_CatchableType@@@Z 00501050 f LIBC:frame.obj
 0001:00100250       ?DestructExceptionObject@@YAXPAUEHExceptionRecord@@E@Z 00501250 f LIBC:frame.obj
 0001:001002d0       ?AdjustPointer@@YAPAXPAXABUPMD@@@Z 005012d0 f LIBC:frame.obj
 0001:000ff7d0       _strncnt                   005007d0 f LIBC:aw_map.obj
 0001:000ff190       _write_char                00500190 f LIBC:output.obj
 0001:000ff1e0       _write_multi_char          005001e0 f LIBC:output.obj
 0001:000ff220       _write_string              00500220 f LIBC:output.obj
 0001:000ff260       _get_int_arg               00500260 f LIBC:output.obj
 0001:000ff270       _get_int64_arg             00500270 f LIBC:output.obj
 0001:000ff290       _get_short_arg             00500290 f LIBC:output.obj
 0001:000fe060       _flsall                    004ff060 f LIBC:fflush.obj
 0001:000fdd60       __cftoe_g                  004fed60 f LIBC:cvt.obj
 0001:000fdd90       __cftof_g                  004fed90 f LIBC:cvt.obj
 0001:000fde30       __shift                    004fee30 f LIBC:cvt.obj
 0001:000fd460       ?CatchGuardHandler@@YA?AW4_EXCEPTION_DISPOSITION@@PAUEHExceptionRecord@@PAUCatchGuardRN@@PAX2@Z 004fe460 f LIBC:trnsctrl.obj
 0001:000fd570       ?TranslatorGuardHandler@@YA?AW4_EXCEPTION_DISPOSITION@@PAUEHExceptionRecord@@PAUTranslatorGuardRN@@PAX2@Z 004fe570 f LIBC:trnsctrl.obj
 0001:000fd208       __unwind_handler           004fe208 f LIBC:exsup.obj
 0001:000fcfa0       _doexit                    004fdfa0 f LIBC:crt0dat.obj
 0001:000fd020       __initterm                 004fe020 f LIBC:crt0dat.obj

FIXUPS: fe1ad ffffff4b ffffffee ffffffa0 18 ffffffab 15 c fffffedc 12 12
FIXUPS: fdf8a 6b 12 fffffeda 1c 20 ffffff29 1a fffffee4 b c 1b ffffff3b
FIXUPS: fdcb6 a 10bc 2b 3c 1d 1d 34 fffff9c7 d5 fffffebe fffffe97 c 5 10
FIXUPS: fe67c 8 5 5 31 5a 6 19 10 32 a fffffbf4 60 64 45 12e 13 fffffc3a
FIXUPS: fe13a 1279 fffffd55 1b fffffe79 b 1d 4b 44 35 19 fffffec4 ffffff5f
FIXUPS: feed0 d 20 d fffffa31 21 d9 22 50 15 33 10d 28 20 18 2e 37 36 48
FIXUPS: fed54 c94 81 e 73 4e 26 76 81 3e 16 1d 13 db 1c 113 b2 1f 2c 28
FIXUPS: 100027 24 28 144 48 46 fffff486 4f 5a 2c fffffedf ffffff10 fffffd06
FIXUPS: 1011aa d f 10 1b e f e 7 10 61 12 fffff5c7 fffffda9 85 82 9 17
FIXUPS: 1007b4 9 fffffd6f 33 11 fffffd7c 3d 49 132 31 fffffdf2 fffff5fb
FIXUPS: ff915 aa 1218 10 4d 2b 56 6c 46 64 2d b 2f 2d 2e 1f 18 29 e 89
FIXUPS: 100fd3 a d 17 b5 13 1d 20 13 19 21 1e 13 1c a7f 77 6a 103 fffffc5a
FIXUPS: 101a82 68 fffffc74 14 10 1c fffffed9 15 2e 10 3c fffffee4 fffffe6e
FIXUPS: 1013be 80 fffffee1 1e fffff571 29 77 33 49 c 26 45 12a 2d 1dae
FIXUPS: 102957 14 18 19 28 6c 20 2b 12 2e 12 fffffa3d 73 ffffff46 fffffe6c
FIXUPS: 102348 28 fffffd9d 18 e4 bd fffffda5 d 11 2f 25 fffffd40 10 94
FIXUPS: 101b4d 20 1ca1 51 20 22 15 e 1a e fffffbdc 4a ffffff3f ffffff31
FIXUPS: 1033a1 13 6d e fffffd64 11e fffffe28 fffffdeb fffffcba 20 fffffacc
FIXUPS: 102685 77 12 197 1c 20 15 20 22 1aab a a fffffeea 15 39 1d ffffff3a
FIXUPS: 1042c2 fffffdf7 5f 12 18 f fffffd3f 12 1d 5 55 3c 7 2f b2 15 fffffb4e
FIXUPS: 103bad 2c 47 1f fffffb16 5f 2e 1b78 10 9 36 fffffe87 1c ffffff91
FIXUPS: 105008 1d 6d 1e 33 d 12 d fffff740 bf 87 119 4d d4 5a fffff8b9
FIXUPS: 1044f7 1a 1b d9 b e 9 26 42 1fed ffffff80 27 fffffbbf 50 47 160
FIXUPS: 105f2e 4a fffffe9f 21 13 4b 20 13 fffff919 15a 119 21 26 16e b1
FIXUPS: 105cda fffff8a9 cb 1c 2b fffffbf1 40 19 33 1c fff06415 2e 26 1b
FIXUPS: b7d8 27 1b 26 27 2e 3d 1b2 28 28 2d 21 1d 21 21 20 24 24 34 32
FIXUPS: 650e 1d9 1ea b3 106 ffcd7 11 37 fff03743 2a 237 32 d5 3f 289 11a
FIXUPS: a85c 28 5c 63 40 6a e 2a1 2f1 1b0 dc 14 12 12 14 14 14 14 93 112
FIXUPS: b69c 24 29 2d 32f1 1b d 12 c c 1b d 12 c c 1b d 21 23 26 22 14
FIXUPS: eb91 d 21 14 1a c c 17 23 26 22 c8 56 bd fffff971 1e d 12 c c 1b
FIXUPS: e857 1a c c 1f d 12 c c 14 1e d 12 c c 1f d 12 c c 14 1e d 12 c
FIXUPS: e590 c c 3e b b b b b b b 2e 20 43 15 9 14 c c c c c c c c c c
FIXUPS: e77a a 18 10 7 fffffa0b c 18 36 15 23 1f 15 15 15 3d 15 15 15 59
FIXUPS: e3b7 34 34 34 30 30 54 9 14 c c c c c c c c fffffa99 c c 15 c c
FIXUPS: e06e c c c 15 c c c c c c 15 c c c c c c 12 c c c c c c c fffffa9d
FIXUPS: dc58 8 9 8 9 8 16 9 10 24 14 1c 10 bd 143 12 12 13 12 13 9 14 c
FIXUPS: dfa6 c c c 23 c c c fffff6af 1b 16 23 b c c 10 a4 63 5f 5f 5f 5f
FIXUPS: da0d 35 48 33 89 49 12 33 8 27 8 9 8 9 8 9 8 9 fffff5b3 31 59 12
FIXUPS: d2a7 19 2a f 16 7 f 5 f 5 16f 54 15 5 1d 8 1b 11 58 c c c a 6e
FIXUPS: d68e 5 10 14 320d d2 41 1a5 6b 142 67 ffffc1a1 12 12 30 37 29 12
FIXUPS: d01a 5 7 14 2e 17 8f 5 9 c c c c c c 16 5c 12 9269 11 11 11 11
FIXUPS: 164db 34 11 15 11 11 11 11 11 11 4c ffff9c15 b f 110 5 b 19 b a5
FIXUPS: 10404 b 10c 84 f5 84 16c 5632 19 8 12 18 8 13 16 d 5 5 5 1e 3e
FIXUPS: 160b2 14 ab 5 38 2c 1f 32 116 2c 2c 2c 1e 11 15 15 11 11 fffff311
FIXUPS: 15823 50 68 6c 1f 2b 37 20 34 8 9 13 1a 18 16d 17 5 5 145 5 c 1f
FIXUPS: 15d9c 43 2c 2c 2c 8 5 e 20 fffff08c 5 17 1c 27 7 12 45 8 23 11
FIXUPS: 15049 11 a2 2c 19 8 19 11 26 11 27 48 4d 30 39 6b 213 138 40 a
FIXUPS: 15736 fffff320 5 19 84 5 11 5 5 62 3a 3a 1f 36 19 22 10 2b 45 2e
FIXUPS: 14d5b 33 3f 37 37 26 1a 26 1b 26 1b 21 7 fffff29c 24 5 18 15 cc
FIXUPS: 142ea 2b 14 18 144 1a 5 5 5 5 29 7 b7 e8 5 43 2f 7 42 fe 51 fd
FIXUPS: 149c9 72 5 11 fffff471 5 e 5 17 5 14 5 25 5 12 6c 5 23 6e 5 5 14
FIXUPS: 140b5 5 1e 5c 5 5 27 5 20 5 12 5 11 5 1b9bb 23 29 19 c 23 29 19
FIXUPS: 2fc59 19 ffff0b10 ffff2449 5 90 5 26 1a ab 5 3a e7e 15 8 50 2c
FIXUPS: 13cd2 2c 96 2c 2c 2c a5 1b9d7 c c 15 c c c 19 15 15 15 31 15 15
FIXUPS: 2f9ad 2a 9 18 d 1f 15 22 29 19 c 23 29 19 c 1d 9 18 fffffaa6 15
FIXUPS: 2f625 c 15 16 14 14 15 25 15 15 15 15 15 27 15 15 15 31 15 c 15
FIXUPS: 2f800 c 15 c c c 19 15 c fffff9f1 c c 15 c 1a 14 11 14 15 c 61
FIXUPS: 2f393 15 15 4c 15 15 15 66 15 15 15 4c 15 15 15 2d c 15 16 11 370f
FIXUPS: 32d35 c 3a 39 c 3a 39 c 115 c 1e 39 c f7 19 35 4b 1b 99 ffffbfc0
FIXUPS: 2f1d0 15 9 14 c 1a c c c c c 2d0b 329 f 10c 17 1c 71 f 1c 14 14
FIXUPS: 32525 89 9 17 f 16 1e 21 c d4 c 2d ea 42 20 19 2a 52 4d 15 339
FIXUPS: 346b3 f 1c ffffbfdc 3d 22b e1 bdc 1e 28 20 3ec 7 4c 7 6b 4d 41
FIXUPS: 31ba6 12a 7 47 7 6a 4d 42 23 ca 1b 9 1c 1b 20f8 97 10 7 5 5 f 23
FIXUPS: 341cd 10 7 5 5 f 23 35 51 10 7 5 5 f 21 6b 3e 4c ec 2b 36 a 10d
FIXUPS: 346a4 ffffeb9e a 1c 3c a 2f 36 a 1b 38 a 27 5 129 2bd 5 21 211
FIXUPS: 339c8 21 233 5c 5 20 23 1ee 5c 5 20 23 a9 27 226a 5 6c 5 5 9 1c
FIXUPS: 36333 13 6e 5 5 5 5 9 8 19 7 13 6e 5 9 8 19 7 13 65 5 5 11 5 5
FIXUPS: 35fb9 65 5 5 9 11 5 5 5 1b 65 5 5 5 5 9 1b 11 11 5 11 5 5 79 5
FIXUPS: 36249 5 5 5 19 5 f fffffa3e 78 5 9 21 19 65 9 11 5 5 5 5 11 7 5
FIXUPS: 35e38 6f 5 5 e 11 20 5 78 5 5 9 11 5 5 5 fffff77b 5 77 5 a 5 98
FIXUPS: 35848 5 b 5 5 9 11 5 5 5 19 5 18 332 f 5 10 5 5 6a 9 11 5 5 5 fffff6ca
FIXUPS: 353e6 5 a 5 68 5 5 5 1a 5 68 5 10 5 a f 5 68 5 a 5 68 5 a 5 68
FIXUPS: 35695 a 5 68 5 fffffa4e 9 8 5 5 18 5 5 13 16 5 5 6c 1c 5 9 8 5
FIXUPS: 35277 19 5 5 13 14 63 5 5 5 5 5 1e 1e fffffb3f 11 89 5 5 5 5 22
FIXUPS: 34f8d 5 9 8 5 5 13 a 6c 5 5 34 5 9 8 5 5 5 5 5 13 a 6c 2e 46b1
FIXUPS: 3985a 20 b 63 29 1b5 28a 59 3c 30 db 1f 18 11 6a 2b 1d 18 11 34
FIXUPS: 3a375 2b a3 59 3c 30 42 19c 39 2b ffffa6f5 3b5a 9 14 6d 39 39 39
FIXUPS: 38b07 39 39 39 37 d 29 d 2c3 12 2e 12 1af 1ff f 1f5 20 b 55 20
FIXUPS: 39598 4e d 1ed 20 ffffeb01 aa 64 1c 48 3e b 12 1e 27 54 1c 40 4e
FIXUPS: 3861c 12 1e 27 41 22 20 16 20 19 60 3a 35 34 35 35 34 35 14b3c
FIXUPS: 4d56b 102 20 1c 22 41 17 3f0 33 12e ffff7b9c 29a 39 12 26 139 195
FIXUPS: 460f9 5d 18 ffffb593 8 14 286 20 30 ffff9f5e 190 1aa ffffc652 12
FIXUPS: 5a8b9 ffffb009 228 39 54 1e9 39 39 196 68 131 ffffe6dd 192 1d 39
FIXUPS: 54a93 ba 1d 3e 49 3bc ffffdfb0 bd 128 92 441 ffffd338 38 df 5 4d
FIXUPS: 50abb 827a 225 10 18b 105 58 19c 8e 217 8 146 8 36 31 5d 11f 8
FIXUPS: 599f7 5 88 43 5 88 58 15 49 51d 53 526 10d 2a dd ffffd4b3 bd 6b
FIXUPS: 57ea0 1e 17 c2 2b 8 1e0 c e 32 8 1b 7a 15 23 3a 2b 8 1b c8 235
FIXUPS: 58665 114 b3 8 f7 4e 267 10 62f2 18 18 18 18 18 18 18 18 18 18
FIXUPS: 5efea 18 18 18 18 18 f 5 5 5 5 ffff8a19 5 2b f5 3b 14 41 23 6c
FIXUPS: 57cea 6ef8 18 18 18 18 18 18 18 18 18 18 18 18 18 18 18 18 18 18
FIXUPS: 5edaa 18 18 18 18 18 18 18 18 18 18 18 18 250f ebc 6b4 ffffda6c
FIXUPS: 60b8d 2c0 46 ffffdaef 5 18 18 33 18 18 18 18 18 18 18 18 18 18
FIXUPS: 5eaf2 18 18 18 18 18 18 18 18 18 11105 f 5 7 5 5 14 8 5 5 5 7 28
FIXUPS: 6fd55 7 11 13 2c 36 2b 1e 23 22 1b f e b1 20 57 ffff6fc6 10c 74
FIXUPS: 6fb17 55 3a 4a 8 5 5 5 a 8 5 5 5 13 8 5 a 8 5 5 5 5 13 8 5 a 8
FIXUPS: 6fca5 5 5 5 13 fffff7b8 2f 19 2f 41 19 8 11 19 37 31 10 b1 41 2e
FIXUPS: 6f7a7 4f 2e 1c 16 38 1b 13 2e c 9 9 9 10e 13 6f 5 fffff451 13 22
FIXUPS: 6ef61 2b 78 3f 13 22 35 2b 78 3f 19 38 14 19 21 14 19 17 d1 14
FIXUPS: 6f36c 2b 14 13 27 42 1b 8 1c fffff3b2 1f 59 42 2c d9 45 26 6d 3f
FIXUPS: 6eb14 63 38 30 49 23 d 33 69 17 3a 2a 16 2e 10 11 67 13 22 14 13
FIXUPS: 6eeb9 fffff42a 13 1b 14 13 22 3c 25 31 53 2b a2 34 13 22 14 13
FIXUPS: 6e5bf 14 13 22 14 13 23 14 19 38 19 6e 1e 6f 29 fffff460 1b 2f
FIXUPS: 6dd31 59 32 14 59 32 21 59 32 14 59 32 40 19 fa 3c 1d 14 13 22
FIXUPS: 6e1af 13 5e 2c 13 27 14 13 22 fffff564 36 29 24 21 22 1a 15 14
FIXUPS: 6d951 14 6b 19 21 b 8 30 19 21 1d 1a 2f 1b 19 2f 36 19 14 22 1d
FIXUPS: 6dc0c 2f fffff46a 33 1b 2f 1b 2f 1b 2f 19 31 1b 2f 1b 2f 19 43
FIXUPS: 6d313 35 21 bb 35 1c 65 39 1c 5b 31 1f 33 39 1a3 29 fffff3b6 5
FIXUPS: 6cbd4 5 5 68 13 23 8 55 68 d7 31 8 5 5c 8 5 36 5f 3e 19 23 8 e
FIXUPS: 6cfe9 8 5 22 19 21 3a fffff4fa 35 91 1e 68 49 3d 22 14 11 14 2d
FIXUPS: 6c7f4 1f 29 1e ed 1d 22 2a 22 b4 1d 22 14 11 2a 22 2e 22 2b 8 fffff5e7
FIXUPS: 6c1b3 22 1a 13 11 14 13 22 14 13 2b 14 13 22 14 13 22 14 13 11
FIXUPS: 6c3dc 13 23 3b 19 23 42 13 23 49 19 fffff810 22 14 2d 2b 14 2f
FIXUPS: 6be66 14 2d 22 14 2d 22 14 2d 15 69 13 21 1e 23 2f 1b 25 14 13
FIXUPS: 6c118 14 13 15 d fffff85d 2b 22 13 31 25 14 13 2e 2d 2f 1b 27 2b
FIXUPS: 6bba5 22 14 13 2b 14 13 22 14 13 22 14 13 22 14 13 15 30 fffff7fb
FIXUPS: 6b56e 23 14 27 8 42 13 2b 1e 23 14 1d 2e 1e 27 40 13 4b 14 13 31
FIXUPS: 6b864 3f 13 24 25 14 13 21 2d 2f fffff81b 5f 8 5 5 21 8 5 a 39
FIXUPS: 6b2ff a 5 3d 13 23 14 27 14 13 22 14 13 15 1f 8 5 a 39 5f a 5 fffff863
FIXUPS: 6ada3 14 13 15 20 13 22 14 13 15 14 13 22 14 13 15 14 13 22 14
FIXUPS: 6af65 15 27 8 5 5 55 68 d7 31 d fffff6a9 2e 46 1e 14 13 22 14 13
FIXUPS: 6a953 8 11 23 21 14 15 ca 75 40 1b 43 19 40 1b 43 19 5b 13 23 14
FIXUPS: 6ad52 1c fffff6d7 17 29 19 1c 50 16 2e 1c 14 41 2e 4f 21 14 13
FIXUPS: 6a6a6 14 13 23 14 13 28 14 13 11 14 13 22 14 13 15 fffff89c 23
FIXUPS: 6a0c3 44 50 1e 14 13 22 14 13 25 29 19 14 13 22 14 13 18 50 1e
FIXUPS: 6a356 13 22 14 13 23 14 13 22 14 fffff742 13 15 3d 38 4d 22 da
FIXUPS: 69d73 1c 13 22 14 13 22 14 13 29 68 2b 1c 36 22 2a 1c 49 13 22
FIXUPS: 6a03c 13 22 14 fffff59f 55 13 22 14 13 22 16 1b 29 d1 13 2c 21
FIXUPS: 69895 1c 7b 44 2e 2c 25 12 2e 13 22 14 13 2e 23 59 15 15 fffff516
FIXUPS: 690b9 26 13 22 14 13 3d 20 1a 13 22 33 13 2d 16 13 38 104 3b 1c
FIXUPS: 69475 31 1c 55 2a 2e 1e 1e 1e 1e 21 fffff47e 1a 13 87 31 14 13
FIXUPS: 68bb4 14 13 68 3c 69 68 35 6f 31 78 31 47 13 22 14 13 15 14 13
FIXUPS: 68fcf 33 13 37 16 fffff34e 25 2b 23 33 29 23 5a a7 39 2b 36 2a
FIXUPS: 686e9 4b 75 38 82 42 62 23 8 1a 2d e 24 e 31 23 8 3a 13 ffffedff
FIXUPS: 67897 e4 5 54 5 3e c6 464 23 39 23 3c 23 39 23 35 23 66 23 22 2e
FIXUPS: 681ce d 23 22 44 5f 57 23 23 23 18df8 c e 4d 25 9 14 11 c c c 11
FIXUPS: 81287 9 14 11 c c c e ffffd065 76 11 5d 2d ffff4890 15d ffff4595
FIXUPS: 67410 2d0 29 d6 19539 c c c e a 6b 177 14 3f 8 10 63 14 1c 9 15
FIXUPS: 8105b 15 f c c c 11 4d 14 1a 7 9 15 f c fffff9df c c 11 a 8 1b
FIXUPS: 80bab 9 14 11 c c c e a 20 9 15 9 14 11 c c c 11 a 8 1b 7 9 14
FIXUPS: 80640 1f 23 43 29 26 2d 29 2d 14 13 5 7 9 c 73 14 5c 8 15 38 18
FIXUPS: 80a05 14 6d 8 68 9 15 9 14 11 fffff7d9 15 a 1b 16 c c 42 b 16 b
FIXUPS: 80422 c e 17 27 c e 17 27 c e 17 30 c e 17 17 17 17 59 1f fffff468
FIXUPS: 7fa95 19 19 19 431 19 41 19 41 19 4e 19 41 19 41 19 62 19 41 19
FIXUPS: 8020f 19 3c 12 c 23 16 c c 1e 15 fffff4a1 19 1b 8 d a a a 5f 2e
FIXUPS: 7f8e8 11 11 11 11 11 11 15 13 1f 1f 14 c c c 15 19 19 19 19 c c
FIXUPS: 7f4a9 1f c c c c 1c 16 c c c 1e c 29 14 25 c 2d 25 38 15 15 16
FIXUPS: 7f6cf 19 19 19 19 19 19 19 21 fffffa4d 15 19 36 17 15 15 19 36
FIXUPS: 7f2ea 15 15 19 37 a c 17 c 2a c c c c 29 c c c c 29 c c c fffff769
FIXUPS: 7ec49 12 13 1b e 15 21 8a 1ec 4a a 15 15 19 36 17 15 15 19 36 17
FIXUPS: 7f0cc 15 19 36 17 15 15 19 36 17 fffff724 c c c c c c c c c c c
FIXUPS: 7e98b c c c c 1a 19 19 19 19 19 19 16 19 13 70 12 12 42 32 fffffb91
FIXUPS: 7e752 c c 1d 9 14 c c c c c c c 2b c c c c c c c c c c c c c c
FIXUPS: 7e8d7 c c 8136 78 8f 83 ab ffffa7fa ffffd08d 12 12 44 2e 4d 45
FIXUPS: 7e61b 2f 7 14 28 5 13 9 14 c c c c c c c c c c 92e8 245 118 13
FIXUPS: 87dbf 4b 8 32 2c 1c 48 8 17 ffffe3e0 19 10 83 29 1d 20 22 2c 37
FIXUPS: 866cd 2d 39 48 9d 36 1b6 8 d f410 38 58 19 34 98 37 ffff2b70 e7
FIXUPS: 86e5b 192 43 44 27 53 89 4e 40 23 ea 1c1 68 27 2d 16 8e a1 cf 123
FIXUPS: 87900 9 b5 dc90 5b 13 13 19 2d 96 39 37 98 38 46 19 34 98 38 3e
FIXUPS: 95ac9 19 34 96 38 77 13 13 4b 13 14 18 3b 19 34 fffff2dc 39 2b
FIXUPS: 950ec 34 13 3c 37 4e 5 2c 13 13 39 8 1e 19 2e 13 12 b 48 13 13
FIXUPS: 953e0 96 38 5b 13 13 51 96 fffff56d 3c 39 31 13 16 15 3f 28 13
FIXUPS: 94cf4 13 21 f 33 13 13 4b 13 14 17 47 3f 1a 2a 19 34 13 3c 37 93
FIXUPS: 9505c 4d6c 36 1e 15 ffffa678 7 77 30 3a a1 38 12c 5d 3d 1c 47 3f
FIXUPS: 948ec 47 3d 1c 47 3d 1c 4b 3f 1a 34 13 13 19 2d ea00 ffff5b1b 10
FIXUPS: 991ae 14 3b 1e8 15 cb ec 2d 17 2c 1d 17 2c 99 1af d 89 d9 2d 17
FIXUPS: 99ae3 23 18 17 67 23 11 22 1c1 8eda c 13 f 19 c e4 3f 87 37 121
FIXUPS: a2fe9 17e c c 66 18 3f 28 16 4d 28 16 15 17 41 b 12 41 b 9a 58
FIXUPS: a29dc 13 14 c 11 c 1e 1c 1e 1c c 19 19 c 1a c 1a 11 14 c 1e 1f
FIXUPS: a2bb6 1f c 19 19 c 1f c 1e 11 fffffac3 a c 11 c 1e 1c 1e 1c c 19
FIXUPS: a2821 c 1a c 1a 11 14 c 1e 1f 1e 1f c 19 19 c 1f c 1e 11 14 fffffaeb
FIXUPS: a24ce 11 c 1c 11 c 1e 23 29 19 c 23 29 19 c 19 16 c c 15 c c 19
FIXUPS: a26bd c 1a c c c 13 11 fffffaf2 15 c 25 16 1a 25 16 17 a 15 13
FIXUPS: a232d f 8 10 f 8 9 7 9 12 c 1e 23 29 19 c 23 29 19 c fffffaec 9
FIXUPS: a1fa7 c 1a c c c c 11 1a 18 1e 13 7 9 10 11 c 1e 15 22 29 19 c
FIXUPS: a2174 29 19 c e c c fffffa19 f 41 f0 5 5 5 5 5 5 5 5 14 5a 16 34
FIXUPS: a1e28 9 10 1a c 1e 15 22 29 19 c 23 29 19 c c fffff53f 12 14 c
FIXUPS: a1683 13 13 1d 35 13 16 31 39 1d 25 142 4d c 14 c c c 15 15 1e
FIXUPS: a1a0e 17 40 2d 1e 27 f9 fffff569 1d 2e 13 a7 1d 18 c a 28 1d 1e
FIXUPS: a1309 c 25 d 1b c 1a 12 14 c 1e 20 1e 20 c 19 18 d 20 c fffff78c
FIXUPS: a0c4c 5c 36 46 28 7 30 41 18 7 b1 1b a 40 26 50 1d 92 1f c c 15
FIXUPS: a1076 c 15 c c 15 a 2f 1d fffff7f2 c 14 19 c 21 c 14 15 c 14 15
FIXUPS: a09e8 14 5c 2d 70 32 c 14 15 c 14 19 c 21 c 14 15 c 14 15 fffff43b
FIXUPS: a0089 41 17e 11 46 1a 3a 98 96 b9 3b 16 1e a 36 7 1d 2c c5 3b 16
FIXUPS: a0713 3a 5a 7 51 33 73 32 c 14 ffffee4a 1c 1d 19 1d 18 1d eb c
FIXUPS: 9f91c c 215 22 ff 46 3e 16 c d 46 16 c d a2 47 7 10 14f 11 46 15
FIXUPS: a004b fffff2a1 c 16 1a c 15 c 40 a c 20 e 63 1f 12 2f 74 12 48
FIXUPS: 9f578 7 1f 1f 1f 1f 1f 49 20 7 60 24 7 b4c0 21 db 18b 14 1a e 9b
FIXUPS: aaf3f 58 2a 40 125 ffff3dce 1f 12 30 4a b 31 12 39 5 5 14 3b 5
FIXUPS: 9f0fe 5 f 3a 164 b58d c 17 26 27 20 5e f c c c 2f 11 a a a 8 f
FIXUPS: aa9d8 1e 11 a a a 8 f 5 6a 1c 5 5 ae fffff81d c 11 20 66 16 39
FIXUPS: aa4b8 24 32 26 27 20 5e f c c c 17 26 27 20 66 16 11 2e 26 27 20
FIXUPS: aa816 f c fffff795 5c 1b 2b 26 2c 2e 26 2a 25 c 18 c 14 14 a 14
FIXUPS: aa1fa 5e f c c c 17 26 2f c 14 14 a 1b 2a fffff870 63 55 16 25
FIXUPS: a9cf9 c 3e a e a e a a c c c 11 2e 1f 40 20 20 54 f c c c 17 29
FIXUPS: a9f70 16 fffff7f9 12 18 2c 61 23 33 20 16 40 54 f c c c 8 4e e
FIXUPS: a99f7 a c c a a a a 4c cd 36 14 26 b fffff8cf c c 8 22 a a a 23
FIXUPS: a953b 14 21 20 56 f c c c 8 14 14 22 14 30 48 f c c c 14 12 14
FIXUPS: a90ef 14 12 1e 30 3b 22 12 18 1e a 20 a 58 f c c c 8 14 1b 36 11
FIXUPS: a93b9 f c c c 17 11 75 f fffff997 1a 56 f c c c 8 2d 11 c c c 39
FIXUPS: a8f7f e a e a a c c c a 14 35 14 30 48 f c c fffff83d c c c 53
FIXUPS: a89a6 c c c 3a 12 14 1d 7 7 1b 18 55 149 21 c 1a 21 c 11 c 11 c
FIXUPS: a8ce6 dc 36 14 fffff6df a a 13 19 a a a 50 1c 16 c c 11 79 c 11
FIXUPS: a86d2 f c c c c 6c 74 12 12 18 42 18 34 56 fffffa58 16 11 16 20
FIXUPS: a83d0 a a a a a a a a a a a a a a a a a a a a a 11 c c c a fffffcdd
FIXUPS: a81cc a e a a e a a a 1f a e a e a a 18 a a a 14 e a 16 c c c c
FIXUPS: a8345 c c fffffc2b a a 14 e a 57 c c c c c 18 a a a 14 e a 46 c
FIXUPS: a811b c c c c 16 14 a c c c fffffb54 c c 39 12 3b 8 5 14 8 14 b4
FIXUPS: a7e8e 6 a a d f 1f a a e a a e a a e a a a 17 fffff83b 8 c 18 e
FIXUPS: a77fb 5 b 8 b 4b 2a 40 8 e7 7d 51 b 99 12 12 18 49 18 34 52 f c
FIXUPS: a7c7e c 52 f fffff729 4b 2a 40 8 b 4b 2a 44 e 4b 2a 40 8 b 4b 2a
FIXUPS: a7720 11 18 e 8 5 b 8 5 b 8 5 b 8 5 fffff984 c e c d 28 20 11 c
FIXUPS: a71eb 18 18 18 18 1b 21 a c 10 a a c c c c 32 4b 2a 40 11 11 c
FIXUPS: a6f60 c 14 c c 2c a a a c c c c c 16 11 18 c c e c d 18 a a a c
FIXUPS: a70ea c c c 16 fffffc7a c c 1b e a e a a e a a a c c c 16 11 c
FIXUPS: a6e9a c 17 e c d 2a a c 10 a a c fffffb4f c c 14b c c c c 16 c
FIXUPS: a6c64 c 16 e c d 2a a c 10 a a c c c 14 c c 13 a a a d834 fffff8a8
FIXUPS: b3e8f 39 10 2a 8 b5 2f a 6 f 6 b0 3a 40 ae 38 c 21 1b 2a 43 3a
FIXUPS: b433a fffff7c2 7a 1ce a5 ffff9f78 ffff8d27 f 17819 c c a 1b 10
FIXUPS: be309 c 1d 14 c 15 1b 14 14 c5 6f 37 11c 7 ffffb8f3 15 285 ffffbdb7
FIXUPS: b5ff6 1ce ce 74 ce 52 ffffe020 10c 9ad3 10 8 c c c 45 c a 16 17
FIXUPS: be0f3 16 30 2a a 16 24 c a 15 19 a 16 1b 1b 15 c 15 c c 15 fffffa3e
FIXUPS: bdd12 1b 38 2a 16 16 c 1b ab 12 13 12 10 8 14 7 12 10 12 23 11
FIXUPS: bdf7a 15 c 15 c c 15 c c c fffffa5e 15 15 16 15 15 2c b 1d 13 13
FIXUPS: bdb56 13 15 15 15 15 15 15 d d d 13 13 13 13 13 13 13 13 13 17
FIXUPS: bd74b 16 9d 15 c 15 c c 15 c c c 10 c 1d 14 c 15 1a 83 d d d d
FIXUPS: bd9d3 f f f 13 13 13 13 fffff9f9 16 16 4d 16 16 16 3c c 14 16 c
FIXUPS: bd592 1a c 14 17 c 14 16 c 14 16 c 14 20 16 16 16 2d 21 16 fffff8b3
FIXUPS: bd017 a 22 15 4c 2c 26 33 3a 29 20 40 36 2d a 2f 31 2c c c c c
FIXUPS: bd321 c 1d 14 c 15 33 17 66 fffff5fb 16 1d a 13 49 94 d6 14 22
FIXUPS: bcc79 16 16 37 a 20 29 7 1e 41 77 4c 10 32 c a 1b 3c 8c 13 16 16
FIXUPS: bc4af 1c 5c 12 12 31 63 12 30 7 22 f 12 f 12 5 12 5 11 5 2c 6f
FIXUPS: bc765 f1 5 ef e 55 c 16 16 16 7c2e 30 12 ffff7b46 12 12 30 41 29
FIXUPS: bc281 35 5 7 14 e 5 5 5 5 1e 5d 5 5 5 7 12 e 37 14 2f 37 49 df69
FIXUPS: ca8f6 60a a da ffffcbeb 7fc ffffecbf 14f 74 b6 ffffd3d0 c 1f 3b
FIXUPS: c477a 1d 1d 1c fffff714 1e 34 63 37 42 18f c b b 48 1a 8b 1ced7
FIXUPS: e11ba 1d 31 1d 1f 1d 1d 1a 21b 41 b0 ffff8f58 7a 1e8 74 74 ffffbfa9
FIXUPS: d680f ffffbb51 20 22 ffffeef6 2a 81f 653 ffffdffc 7a 1dc 74 b6
FIXUPS: d0524 20d2f 1e9 12e4 5d 5d 264 546 c58 bad 2bb 59 83 4e8 20 f ffffa443
FIXUPS: efbc6 92 f48 92 ffffc735 ffff379f 26 3be 91 1d 31 1d 1f 1d 1d 1a
